:020000040000FA
:04000000B6EF00F067
:100008005482D9CF05F0DACF06F00F0112A91CD01F
:100018008EBC02D0839483928EA802D083A20FD084
:10002800899425EE04F0010EDBBE08D0000EDE5CDC
:10003800020EDE58D8A002D0899201D089828EB8EB
:1000480083B201D08984129912A184D08EB883B268
:1000580089929050FF0A096E8E50FF0A086E04C5F7
:100068000AF005C50BF00BBE04D0020E0B5CD8B02D
:100078002CD00A4A0B2A0AC004F50BC005F502C5A4
:100088000AF003C50BF0060E0A24D96E050E0B20E4
:10009800DA6E09C0DFFF060E0A24D96E070E0B20A0
:1000A800DA6E08C0DFFF0A4A0B2AFF0E016E010E46
:1000B800026E0AC003F00BC004F001500316025090
:1000C800041603C002F504C003F58EB883B2898410
:1000D80089848EA0FED78EA802D083A202D08994EC
:1000E80001D0898425EE04F0010EDBBE08D0000E95
:1000F800DE5C020EDE58D8A002D0899201D0898237
:1001080008B80CD025D0838202D0838405D083948C
:100118001FD083A21DD0839483921AD00950016EF8
:10012800026A0250000AD8A413D00150040AD8B4B5
:10013800F0D7100AD8B4EDD7340AD8B4E4D71F0AD8
:10014800D8B4EAD77F0AD8B4E0D71F0AD8B4DFD723
:100158000F0112910E01CA9906C0DAFF05C0D9FF36
:1001680054921100B5EF4BF084C0D9FF85C0DAFF77
:10017800000EDE6E000EDD6E86C00CF087C00DF03E
:1001880097EC46F00CC0C1F00DC0C2F00001C2AF40
:1001980002D00B0E1200D890C135D96EC235DA6E76
:1001A8008A0ED926010EDA22DECFDBF0DDCFDCF0B5
:1001B800DB51DC11D8A402D00C0E120084C0D9FF88
:1001C80085C0DAFFDBC0DEFFDCC0DDFFDBC0D9FFA6
:1001D800DCC0DAFFDF50D8B415D020EE01F0DB51D7
:1001E800D926DC51DA22DF5086EC5BF00001CD6FB6
:1001F800CDB108D08851D8A4CDA502D00A0E1200DE
:10020800000E1200DBC0D9FFDCC0DAFF000EDF6E83
:1002180020EE01F0DB51D926DC51DA22C1C0DFFF24
:1002280020EE01F0DB51D926DC51DA22DF5089ECCF
:1002380040F00001CD6FCDA102D0030E120088510D
:10024800D8B402D0CDB5DAD7000ED46F000ED56F72
:10025800000ED66F000ED76FDBC060F0DCC061F017
:10026800000E626F000E636F000E646F000E656F04
:100278000BEC36F00001DA6FDA05D8A4FAD0000EDC
:10028800D96F000ED86FD95105E1040ED85DD8B0EA
:10029800A2D001D0A0D0D8C089F0D9C08AF0893BBB
:1002A8008A3BF00E8A1789510F0B8A13F00E8917B3
:1002B800DBC08BF0DCC08CF089518B278A518C23F2
:1002C800EC0E8B25CE6F010E8C21CF6F20EE04F043
:1002D800CE51D926CF51DA22DF50D8A408D0000E4B
:1002E800B36F000EB46F000EB56F000E58D020EE3D
:1002F80009F0CE51D926CF51DA22DF50896F8951C2
:100308008B6F8A6B20EE0AF0CE51D926CF51DA22B4
:10031800DF508C6F8CC08DF08E6B8F6B906B8EC0A6
:1003280090F08DC08FF08E6B8D6B20EE0BF0CE5160
:10033800D926CF51DA22DF50916F91C092F0936B9A
:10034800946B956B92C095F0946B936B926B8D51F7
:100358009211966F8E519311976F8F519411986FD8
:1003680090519511996F8A5196119A6F8B519711E7
:100378009B6F000E98119C6F000E99119D6F20EED7
:1003880008F0CE51D926CF51DA22DF509E6F9E5108
:100398009A11B36F9B51B46F9C51B56F9D51B66F55
:1003A800A30E896F000E8A6FD890D835D96ED935CB
:1003B800DA6ED890D936DA368951D9268A51DA22B6
:1003C800B3C0DEFFB4C0DEFFB5C0DEFFB6C0DEFFDF
:1003D800D84BD92B58D7000ED96F000ED86FD851EB
:1003E800D911D8B403D0D807D8A0D907A30E896FDC
:1003F800000E8A6FD890D835D96ED935DA6ED89074
:10040800D936DA368951D9268A51DA22DECFD4F0A4
:10041800DECFD5F0DECFD6F0DECFD7F0D451D51170
:10042800D611D711D8A405D0000EB86F020EB76F39
:1004380013D0DBC060F0DCC061F0D4C062F0D5C07E
:1004480063F0D6C064F0D7C065F00BEC36F000015D
:10045800896F8951B76FB86BB7C0DAF0DA51D8B481
:1004680008D0D84BD92BD95104E1040ED85DD8A0B7
:10047800BDD7030EDA19D8A402D0010E1200DA5142
:10048800D8B402D00D0E120020EE3AF0DB51D92676
:10049800DC51DA22DF50896F89518B6F8A6B20EE2D
:1004A80039F0DB51D926DC51DA22DF508C6F8C51C0
:1004B8008A13000E8B13020E8B198A11D8A4E2D767
:1004C80020EE45F0DB51D926DC51DA22DF50896F66
:1004D80089518B6F8A6B20EE44F0DB51D926DC51B1
:1004E800DA22DF508C6F8C518A13000E8B138AC06E
:1004F800D0F08BC0D1F0D26BD36BD051D111D211C7
:10050800D311D8A459D020EE53F0DB51D926DC51B1
:10051800DA22DF50896F89518B6F8A6B20EE54F095
:10052800DB51D926DC51DA22DF508C6F8CC08DF07C
:100538008E6B8F6B906B8EC090F08DC08FF08E6B32
:100548008D6B20EE55F0DB51D926DC51DA22DF50D5
:10055800916F91C092F0936B946B956B92C095F0EC
:10056800946B936B926B8D519211966F8E51931180
:10057800976F8F519411986F90519511996F8A5177
:1005880096119A6F8B5197119B6F000E98119C6F63
:10059800000E99119D6F20EE52F0DB51D926DC51E7
:1005A800DA22DF509E6F9E519A11D06F9B51D16F06
:1005B8009C51D26F9D51D36F20EE16F0DB51D92696
:1005C800DC51DA22D0C0DEFFD1C0DEFFD2C0DEFFB0
:1005D800D3C0DEFF20EE3EF0DB51D926DC51DA2213
:1005E80010EE03F0DB51E126DC51E222DFCFE7FF1A
:1005F80020EE03F0DB51D926DC51DA22DE04D8B430
:100608000AD020EE03F0DB51D926DC51DA22020EA3
:10061800DE18D8A437D7D0C00CF0D1C00DF0D2C0A6
:100628000EF0D3C00FF020EE03F0DB51D926DC51D9
:10063800DA22DF50896F8951106E116A126A136AC3
:1006480007EC57F00CC0D0F00DC0D1F00EC0D2F0BE
:100658000FC0D3F0000120EE3BF0DB51D926DC516E
:10066800DA2210EE02F0DB51E126DC51E222DFCF84
:10067800E7FF20EE02F0DB51D926DC51DA22DF5009
:10068800D8B400D7FF0E896FFF0E8A6F20EE02F0F4
:10069800DB51D926DC51DA22DF508B6F8C6B895104
:1006A8008B278A518C2320EE02F0DB51D926DC51AE
:1006B800DA22DF508D6F8D518B17000E8C178B51FE
:1006C8008C11D8A4DFD620EE40F0DB51D926DC51BE
:1006D800DA22DF50896F89518B6F8A6B20EE3FF0E9
:1006E800DB51D926DC51DA22DF508C6F8C518A130A
:1006F800000E8B1320EE08F0DB51D926DC51DA22EC
:100708008AC0DEFF8BC0DDFF20EE08F0DB51D92662
:10071800DC51DA22DECF89F0DDCF8AF00F0E89179F
:10072800000E8A1789518A11D8A4ACD620EE42F05F
:10073800DB51D926DC51DA22DF50896F89518B6F62
:100748008A6B20EE41F0DB51D926DC51DA22DF50EA
:100758008C6F8C518A13000E8B138AC0C5F08BC026
:10076800C6F0C76BC86BC551C611C711C811D8A44C
:1007780059D020EE4FF0DB51D926DC51DA22DF5078
:10078800896F89518B6F8A6B20EE50F0DB51D92627
:10079800DC51DA22DF508C6F8CC08DF08E6B8F6B42
:1007A800906B8EC090F08DC08FF08E6B8D6B20EEAD
:1007B80051F0DB51D926DC51DA22DF50916F91C01C
:1007C80092F0936B946B956B92C095F0946B936BCE
:1007D800926B8D519211966F8E519311976F8F5125
:1007E8009411986F90519511996F8A5196119A6F3B
:1007F8008B5197119B6F000E98119C6F000E9911E9
:100808009D6F20EE4EF0DB51D926DC51DA22DF5005
:100818009E6F9E519A11C56F9B51C66F9C51C76FB1
:100828009D51C86F20EE3CF0DB51D926DC51DA220D
:10083800DF50896F20EE3DF0DB51D926DC51DA22FA
:10084800DF508A6F8951C36F8AC0C4F0C351C41185
:10085800D8B418D620EE08F0DB51D926DC51DA22BC
:10086800DECF89F0DDCF8AF0040E8B6FD8908A3303
:1008780089338B2FFBD7C35189258C6FC4518A21AB
:100888008D6F8E6BD8B08E2B8F6BD0518C25BD6F32
:10089800D1518D21BE6FD2518E21BF6FD3518F217F
:1008A800C06FBD51C55DBE51C659BF51C759C05172
:1008B800C859D8A0E7D5BD51C55D0C6EBE51C65903
:1008C8000D6EBF51C7590E6EC051C8590F6E20EE3C
:1008D80002F0DB51D926DC51DA22DF50896F8951C9
:1008E800106E116A126A136ACFEC52F00CC0C9F08C
:1008F8000DC0CAF00EC0CBF00FC0CCF00001C9513A
:10090800CA11CB11CC11D8B4BDD5010EDA6FCC51B8
:10091800CB1106E1F60EC95D0F0ECA59D8A002D058
:10092800020EDA6FCC51CB1106E1F60EC95DFF0E4F
:10093800CA59D8A002D0030EDA6F020EC925896FF2
:10094800000ECA218A6F000ECB218B6F000ECC21BE
:100958008C6F20EE12F0DB51D926DC51DA2289C0E7
:10096800DEFF8AC0DEFF8BC0DEFF8CC0DEFF20EE1C
:100978001AF0DB51D926DC51DA22D4C0DEFFD5C00B
:10098800DEFFD6C0DEFFD7C0DEFFC351D425896F96
:10099800C451D5218A6F000ED6218B6F000ED72146
:1009A8008C6F20EE1EF0DB51D926DC51DA2289C08B
:1009B800DEFF8AC0DEFF8BC0DEFF8CC0DEFFBD51CC
:1009C800D425896FBE51D5218A6FBF51D6218B6F2F
:1009D800C051D7218C6F20EE26F0DB51D926DC518F
:1009E800DA2289C0DEFF8AC0DEFF8BC0DEFF8CC042
:1009F800DEFF030EDA19D8A490D020EE08F0DB5100
:100A0800D926DC51DA22DE50DE10D8A43BD520EE00
:100A18005BF0DB51D926DC51DA22DF50896F89512E
:100A28008B6F8A6B20EE5CF0DB51D926DC51DA2221
:100A3800DF508C6F8CC08DF08E6B8F6B906B8EC07F
:100A480090F08DC08FF08E6B8D6B20EE5DF0DB51DA
:100A5800D926DC51DA22DF50916F91C092F0936B66
:100A6800946B956B92C095F0946B936B926B8D51D0
:100A78009211966F8E519311976F8F519411986FB1
:100A880090519511996F8A5196119A6F8B519711C0
:100A98009B6F000E98119C6F000E99119D6F20EEB0
:100AA8005AF0DB51D926DC51DA22DF509E6F9E5175
:100AB8009A119F6F9B51A06F9C51A16F9D51A26F7E
:100AC80020EE22F0DB51D926DC51DA229FC0DEFF6E
:100AD800A0C0DEFFA1C0DEFFA2C0DEFF20EE12F044
:100AE800DB51D926DC51DA22DECF89F0DECF8AF05D
:100AF800DECF8BF0DECF8CF0020ED89089378A37A4
:100B08008B378C37E82EF9D789C0B9F08AC0BAF08C
:100B18008BC0BBF08CC0BCF091D020EE08F0DB514C
:100B2800D926DC51DA22DE50DE10D8B4ABD420EE60
:100B38001EF0DB51D926DC51DA22DECF89F0DECF78
:100B48008AF0DECF8BF0DECF8CF0D05189258D6F07
:100B5800D1518A218E6FD2518B218F6FD3518C2125
:100B6800906F20EE22F0DB51D926DC51DA228DC0BD
:100B7800DEFF8EC0DEFF8FC0DEFF90C0DEFF020EFC
:100B8800DA19D8B444D020EE12F0DB51D926DC5162
:100B9800DA22DECF89F0DECF8AF0DECF8BF0DECF2F
:100BA8008CF0010E89158D6F000E8A158E6F000E60
:100BB8008B158F6F000E8C15906F20EE12F0DB51A5
:100BC800D926DC51DA22DECF0CF0DECF0DF0DECFF5
:100BD8000EF0DECF0FF0030E106E000E116E000E39
:100BE800126E000E136E07EC57F0D8900F320E32CB
:100BF8000D320C3200018D510C24B96F8E510D202D
:100C0800BA6F8F510E20BB6F90510F2016D020EE77
:100C180012F0DB51D926DC51DA22DECF89F0DECFA3
:100C28008AF0DECF8BF0DECF8CF0D8908935B96FA3
:100C38008A35BA6F8B35BB6F8C35BC6FFF0EB92503
:100C4800896F010EBA218A6F000EBB218B6F000ECF
:100C5800BC218C6F0A0E05D0D8908C338B338A3325
:100C68008933E82EF9D720EE16F0DB51D926DC516E
:100C7800DA228951DE5C8A51DE588B51DE588C515C
:100C8800DE58D8A046EF02F020EE0EF0DB51D92650
:100C9800DC51DA22FF0EDE6EFF0EDE6EFF0EDE6E18
:100CA800FF0EDD6EDD52DD5210EE0AF0DB51E1265B
:100CB800DC51E222DECFE6FFDECFE6FFDECFE6FF45
:100CC800DECFE6FF20EE05F0DB51D926DC51DA2233
:100CD800800EDF6E030EDA19D8A4F1D120EE5FF092
:100CE800DB51D926DC51DA22DF50896F89518B6FAD
:100CF8008A6B20EE5EF0DB51D926DC51DA22DF5018
:100D08008C6F8C518A13000E8B138A058B11D8A413
:100D1800D6D1DBC03AF0DCC03BF0010ED4253C6EE6
:100D2800000ED5213D6E000ED6213E6E000ED72155
:100D38003F6E84EC4FF00009D8A4C1D1000120EE29
:100D480005F0DB51D926DC51DA22000EDF6E22EEE7
:100D58002DF0DB51D926DC51DA22DF50896F895119
:100D68008B6F8A6B22EE2CF0DB51D926DC51DA220C
:100D7800DF508C6F8C518A13000E8B13550E8A1915
:100D880003E1AA0E8B19D8A49AD120EE2FF0DB51DB
:100D9800D926DC51DA22DF50896F89518B6F8A6B33
:100DA80020EE30F0DB51D926DC51DA22DF508C6F8F
:100DB8008CC08DF08E6B8F6B906B8EC090F08DC059
:100DC8008FF08E6B8D6B20EE31F0DB51D926DC5124
:100DD800DA22DF50916F91C092F0936B946B956B10
:100DE80092C095F0946B936B926B8D519211966FA4
:100DF8008E519311976F8F519411986F905195114F
:100E0800996F8A5196119A6F8B5197119B6F000EAB
:100E180098119C6F000E99119D6F20EE2EF0DB51FA
:100E2800D926DC51DA22DF509E6F9E519A119F6FAE
:100E38009B51A06F9C51A16F9D51A26F520E9F199B
:100E480009E1520EA01906E1610EA11903E1410E54
:100E5800A219D8A434D122EE13F0DB51D926DC51E3
:100E6800DA22DF50896F89518B6F8A6B22EE14F07A
:100E7800DB51D926DC51DA22DF508C6F8CC08DF023
:100E88008E6B8F6B906B8EC090F08DC08FF08E6BD9
:100E98008D6B22EE15F0DB51D926DC51DA22DF50BA
:100EA800916F91C092F0936B946B956B92C095F093
:100EB800946B936B926B8D519211966F8E51931127
:100EC800976F8F519411986F90519511996F8A511E
:100ED80096119A6F8B5197119B6F000E98119C6F0A
:100EE800000E99119D6F22EE12F0DB51D926DC51CC
:100EF800DA22DF509E6F9E519A119F6F9B51A06F0F
:100F08009C51A16F9D51A26F720E9F1909E1720E3B
:100F1800A01906E1410EA11903E1610EA219D8A496
:100F2800CED022EE17F0DB51D926DC51DA22DF5081
:100F3800896F89518B6F8A6B22EE18F0DB51D926A5
:100F4800DC51DA22DF508C6F8CC08DF08E6B8F6B8A
:100F5800906B8EC090F08DC08FF08E6B8D6B22EEF3
:100F680019F0DB51D926DC51DA22DF50916F91C09C
:100F780092F0936B946B956B92C095F0946B936B16
:100F8800926B8D519211966F8E519311976F8F516D
:100F98009411986F90519511996F8A5196119A6F83
:100FA8008B5197119B6F000E98119C6F000E991131
:100FB8009D6F22EE16F0DB51D926DC51DA22DF5084
:100FC8009E6F9E519A119F6F9B51A06F9C51A16F6C
:100FD8009D51A26F20EE0EF0DB51D926DC51DA22AA
:100FE8009FC0DEFFA0C0DEFFA1C0DEFFA2C0DEFF03
:100FF80022EE1BF0DB51D926DC51DA22DF50896F53
:1010080089518B6F8A6B22EE1CF0DB51D926DC519B
:10101800DA22DF508C6F8CC08DF08E6B8F6B906BEB
:101028008EC090F08DC08FF08E6B8D6B22EE1DF010
:10103800DB51D926DC51DA22DF50916F91C092F052
:10104800936B946B956B92C095F0946B936B926BCA
:101058008D519211966F8E519311976F8F519411F4
:10106800986F90519511996F8A5196119A6F8B517B
:1010780097119B6F000E98119C6F000E99119D6F30
:1010880022EE1AF0DB51D926DC51DA22DF509E6FAE
:101098009E519A119F6F9B51A06F9C51A16F9D51BA
:1010A800A26F20EE0AF0DB51D926DC51DA229FC06C
:1010B800DEFFA0C0DEFFA1C0DEFFA2C0DEFFDBC0F6
:1010C800D9FFDCC0DAFFDAC0DFFF0101884B892BCA
:1010D800000120EE06F0DB51D926DC51DA2288C166
:1010E800DEFF89C1DDFF04EF01F0000E0D6E000E7A
:1010F8000C6E52EC5BF00F0B0101E86F000E9E6F57
:10110800070E8C6E010EE76F000EA36F0F0E0F0116
:10111800596F000E116F000E196F000E216F000E2F
:10112800266F000E2E6F886889688A688A8E889074
:1011380088928382020E536EE8EC59F08894838477
:10114800889C839C889E838E8B688968860E0001A4
:101158008A6FFB0E8B6FA60E8C6FFF0E8D6FF70ECE
:101168008E6FFE0E8F6F2D0E906FFF0E916F35EC08
:101178005BF0CDEC59F017D0B80E00018A6FFE0E67
:101188008B6F8FCF8CF08D6B35EC5BF0290E0101E6
:10119800E46F960EE36F7F0EE82EFED7E32FFCD7A1
:1011A800E42FFAD704008FB2E7D796EC49F0010193
:1011B800E86F9F0E00018A6FFC0E8B6FE8C18CF000
:1011C8008D6B35EC5BF00400290E0101E46F960E7F
:1011D800E36F7F0EE82EFED7E32FFCD7E42FFAD774
:1011E800D250F00B0109D26ED09E0E01C691CF0EDF
:1011F800CF16CF82CF80C2890F011381138914893A
:10120800F28E0E01BA8929EC50F083928394AFECE8
:101218004CF0AFEC4CF0000E0C6E340E86EC57F030
:10122800480E106EFF0E116E8DEC53F0A60E106E68
:10123800FF0E116E8DEC53F0000E0C6E390E86EC1D
:1012480057F0838004002BEC32F0D6EC43F0FEEC30
:1012580051F0000E0C6E800E86EC57F07BEC5AF0C5
:10126800000E0C6E800E86EC57F00101E8510F0D50
:10127800340EF324106E0D0EF420116E8DEC53F025
:1012880001019D51D8B4EED0D40E00018A6FFD0E35
:101298008B6F35EC5BF010EC53F010C0AAF311C063
:1012A800ABF312C0ACF313C0ADF30301AA51AB11F9
:1012B800AC11AD11D8A419D0FC0E00018A6FFC0E38
:1012C8008B6FAAC38CF0ABC38DF0ACC38EF0ADC3EB
:1012D8008FF035EC5BF00A0E0F6E000E106E000EEC
:1012E800116E000E126EAEEC56F0000E0301AF6FD9
:1012F800000EAE6FAFBF06D0AF511DE1040EAE5D5C
:10130800D8B019D0DB0E00018A6FFF0E8B6FAA0EC2
:101318000301AE25D96E030EAF21DA6EDF5001014D
:10132800E36FE35100018C6F8D6B35EC5BF00301CB
:10133800AE4BAF2BDFD7B40E00018A6FFB0E8B6F5D
:1013480035EC5BF0540E00018A6FFC0E8B6F35ECA8
:101358005BF022EE14F000EECBF01F0EDBCFEBFFBC
:10136800E806FCE2D30E0001EB6FFF0EEC6F80EC99
:1013780033F0CBC06CF1CCC06DF1CDC06EF1CEC0F6
:101388006FF101016C516D116E116F11D8B46AD0F3
:101398003A0E00018A6FFC0E8B6F6CC18CF06DC128
:1013A8008DF06EC18EF06FC18FF035EC5BF0140ECE
:1013B8000001A46F020EA56F6CC1E4F16DC1E5F1E7
:1013C8006EC1E6F10101E36B000EE3250001A66F93
:1013D800010E0101E4210001A76F000E0101E521C2
:1013E8000001A86F000E0101E6210001A96F02ECBF
:1013F80010F0140E00018C6F020E8D6F340E8E6F7C
:101408000B0E8F6F000E916F080E906FA80E926FE3
:10141800030E936F09EC13F0000E0301B16F000E79
:10142800B06FB1BF06D0B1511DE1080EB05DD8B0A4
:1014380019D0D70E00018A6FFF0E8B6F340E03018F
:10144800B025D96E0B0EB121DA6EDF500101E36FC2
:10145800E35100018C6F8D6B35EC5BF00301B04BF1
:10146800B12BDFD70101A3AF12D08A6883928382A0
:10147800290E0101E46F960EE36F7F0EE82EFED76A
:10148800E32FFCD7E42FFAD7A7EC3EF0EFD7E751CC
:10149800D8B40CD0F40E00018A6FFD0E8B6F35ECBA
:1014A8005BF0020E0101A26F220E0BD0E40E0001C8
:1014B8008A6FFD0E8B6F35EC5BF0010E0101A26F98
:1014C800040EA16F000E0301A56F000EA46F000E9D
:1014D800B56F000EB46F010EB36FB4BF06D0B45130
:1014E8006EE1040EB35DD8B06AD0B3C30CF0B4C3D8
:1014F8000DF0000E0F6E0F0E0E6EE2EC5AF0240E79
:101508000C24126E0E0E0D20136E3AEC58F0135088
:1015180004E1030E125CD8A04ED0B3C30CF0B4C3E0
:101528000DF0000E0F6E0F0E0E6EE2EC5AF0240E48
:101538000C240301A16F0E0E0D20A26F420E0001B4
:101548008A6FFE0E8B6FA1C38CF0A2C38DF035ECB1
:101558005BF0B3C3E3F1B4C3E4F1050ED890010125
:10156800E337E437E82EFAD7140EE3250001DD6FE0
:10157800020E0101E4210001DE6FB3C30CF0B4C315
:101588000DF0000E0F6E0F0E0E6EE2EC5AF0240EE8
:101598000C240001DF6F0E0E0D20E06F030EE16FCB
:1015A80001EC1BF00101E56FE5510301A66FA76B84
:1015B800A651F0EC55F00301B34BB42B8ED7020EB5
:1015C80001019F19D8A404D00F01108B070E2D6FAD
:1015D800839E000E0C6EC00E86EC57F07BEC5AF022
:1015E800000E0C6EC00E86EC57F0940E106EFF0EB7
:1015F800116E8DEC53F020D18EA8899416EC5BF017
:101608000C500D10D8B4F7D0B5C3A3F3B20E0C6EBE
:10161800030E0D6E44EC52F00301B56F350EB5198B
:10162800D8A407D0B40E00018A6FFB0E8B6F35EC7F
:101638005BF0360E00018A6FFF0E8B6FB5C38CF01E
:101648008D6B8DA004D00101E36BE32B02D0010167
:10165800E36BE35100018E6F8F6B35EC5BF0030198
:10166800B2A927D0600EB519D8A423D05F0EA3194C
:10167800D8A41FD053500209536E2BEE34F0A2C1E8
:10168800DFFF2BEE35F0A1C1DFFF8384000E246E4F
:10169800020E236E8EEC3AF083945350FD0B536E7A
:1016A800000E0101A96FBCEC5AF0000E0301B56FE2
:1016B800C3D00101E751D8B44AD00301B251100B8D
:1016C8000001B06F000EB16F0301B551CDEC34F0DD
:1016D800B0C0B6F3B1C0B7F3080E0301B619B7111D
:1016E800D8B400F0070E0301B619B711D8B4EDEC61
:1016F80054F00301B605B711D8B443EC54F0020E08
:101708000301B619B711D8B4ABEC3DF0030E0301D1
:10171800B619B711D8A406D047EC2CF0E2C0A4F350
:10172800E3C0A5F3050E0301B619B711D8A406D076
:101738005CEC38F0EDC0A4F3EEC0A5F3090E03018C
:10174800B619B711D8A478D08EEC5BF075D0030128
:10175800B251100B0C6E000E0D6EB55105EC22F057
:101768000CC0B6F30DC0B7F3070E0301B619B711D5
:10177800D8B47EEC54F0020E0301B619B711D8B4F0
:10178800DBEC56F00301B605B711D8B495EC44F07C
:10179800030E0301B619B711D8B48AEC52F0040E3F
:1017A8000301B619B711D8B495EC59F0050E030129
:1017B800B619B711D8B400EC49F0060E0301B619F2
:1017C800B711D8B49CEC5BF0080E0301B619B71139
:1017D800D8B498EC3FF0090E0301B619B711D8B484
:1017E80031EC4BF00A0E0301B619B711D8A424D076
:1017F800ABEC4AF021D096EC49F001019E6F9F5165
:10180800D8B41AD0E8519E19D8B416D0838E000ED9
:101818000C6EC00E86EC57F07BEC5AF0000E0C6E86
:10182800C00E86EC57F0030E106EFF0E116E8DEC95
:1018380053F09EC1E8F132D08FB230D0050E0301CB
:10184800A419A511D8B42AD0D7D6B80E00018A6F2A
:10185800FE0E8B6F8FCF8CF08D6B35EC5BF0290E05
:101868000101E46F960EE36F7F0EE82EFED7E32F9B
:10187800FCD7E42FFAD70400000E0C6EC00E86ECDD
:1018880057F07BEC5AF0000E0C6EC00E86EC57F049
:10189800500E106EFF0E116E8DEC53F08FB2D5D72F
:1018A800290E0101E46F960EE36F7F0EE82EFED736
:1018B800E32FFCD7E42FFAD783948392000E00011C
:1018C800DD6F000EDE6FB60EDF6FFB0EE06F000EF1
:1018D800E16F2AEC4FF0B6D4A6C0B9F0A7C0BAF0B1
:1018E800AAC0D9FFABC0DAFF000EDE6E000EDD6EB7
:1018F800A4C00DF0A5C00EF0B4EC51F00001B86F13
:10190800B851D8B402D0B851120020EE05F0A45155
:10191800D926A551DA22DF50D8B408D020EE05F038
:10192800A451D926A551DA22DF50120020EE04F086
:10193800A451D926A551DA22DFB202D0070E12002F
:1019480020EE06F0A451D926A551DA2210EE06F0B1
:10195800A451E126A551E222E6CFB0F0E6CFB1F0DE
:10196800E6CFB2F0E6CFB3F0A851B025B46FA951D5
:10197800B121B56F000EB221B66F000EB321B76F5B
:10198800DE50B45DDE50B559DE50B659DE50B75959
:10199800D8B0FCD2000EA96F000EA86FF7D220EEC7
:1019A80006F0A451D926A551DA22FF0EDE14AC6F39
:1019B800010EDE14AD6F000EDE14AE6F000EDE14E5
:1019C800AF6FAC51AD11AE11AF11D8A445D220EE16
:1019D80006F0A451D926A551DA22DECFACF0DECF2D
:1019E800ADF0DECFAEF0DECFAFF00A0E05D0D89066
:1019F800AF33AE33AD33AC33E82EF9D7A4C0D9FF3B
:101A0800A5C0DAFF10EE02F0DE50E126DD50E2223A
:101A1800E750B06FB005AC15BB6FBB51D8A4A5D0CB
:101A280020EE06F0A451D926A551DA22DE50DE10A8
:101A3800DE10DE10D8A427D020EE0EF0A451D9264F
:101A4800A551DA22DECFC2F0DECFC3F0DECFC4F07C
:101A5800DECFC5F0C251C311C411C511D8A433D00B
:101A6800A4C0D9FFA5C0DAFFDECF91F0DDCF92F098
:101A7800000E936F000E946F000E956F000E966F18
:101A8800DFEC2DF018D0A4C0D9FFA5C0DAFFDECF57
:101A980091F0DDCF92F020EE12F0A451D926A55195
:101AA800DA22DECF93F0DECF94F0DECF95F0DECFF2
:101AB80096F0DFEC2DF091C0C2F092C0C3F093C055
:101AC800C4F094C0C5F00001C251C311C411C511BE
:101AD800D8B460D2C205C311C411C511D8A40AD0A4
:101AE80020EE05F0A451D926A551DA22020EDF6EA8
:101AF800020E1200C22911E1C3290FE1C4290DE128
:101B0800C529D8A40AD020EE05F0A451D926A5519C
:101B1800DA22010EDF6E010E120020EE12F0A4513F
:101B2800D926A551DA22C2C0DEFFC3C0DEFFC4C079
:101B3800DEFFC5C0DEFF20EE0EF0A451D926A55168
:101B4800DA22DE50DE10DE10DE10D8A40ED020EE31
:101B58000EF0A451D926A551DA22C2C0DEFFC3C0B7
:101B6800DEFFC4C0DEFFC5C0DEFF20EE16F0A451C4
:101B7800D926A551DA22A4C0E1FFA5C0E2FF00EEF4
:101B88002AF0E650E926E550EA22DE50EE1817E181
:101B9800DE50EE1814E1DE50EE1811E1DE50EE18BA
:101BA800D8A40DD0A4C0D9FFA5C0DAFFDECF25F098
:101BB800DDCF26F047EC45F00009D8A48CD1A4C0AD
:101BC800D9FFA5C0DAFFDECF18F0DDCF19F000018C
:101BD80020EE12F0A451D926A551DA22DECF1AF050
:101BE800DECF1BF0DECF1CF0DECF1DF0CDEC4EF0CB
:101BF80018C0BEF019C0BFF01AC0C0F01BC0C1F0B9
:101C08000001BE51BF11C011C111D8B469D7BB5171
:101C1800BE27000EBF23C023C123A8C0ACF0A9C0B3
:101C2800ADF0090EAE6FD890AD33AC33AE2FFBD705
:101C3800ACC0BCF0ADC0BDF0BC51BD11D8B4C8D06B
:101C4800BB51BC25AC6F000EBD21AD6FA4C0D9FF40
:101C5800A5C0DAFF10EE02F0DE50E126DD50E222E8
:101C6800E750AE6FAF6BAC51AE5DAD51AF59D8B068
:101C780012D0A4C0D9FFA5C0DAFF10EE02F0DE50E2
:101C8800E126DD50E222E750AC6FBB51AC5DBC6F82
:101C9800BD6BD8A0BD07B9C01BF0BAC01CF0BEC050
:101CA8001DF0BFC01EF0C0C01FF0C1C020F0BCC0F6
:101CB80021F0BDC022F0A4C0D9FFA5C0DAFF10EE04
:101CC80001F0DE50E126DD50E222E75024EC4AF034
:101CD8000009D8A400D10001BC51AC6FBD51AD6F53
:101CE800AE6BAF6BA4C0D9FFA5C0DAFF10EE2AF027
:101CF800DE50E126DD50E222E6CFB0F0E6CFB1F0CB
:101D0800E6CFB2F0E6CFB3F0BE51B05DB46FBF51CD
:101D1800B159B56FC051B259B66FC151B359B76F08
:101D2800AC51B45DAD51B559AE51B659AF51B75973
:101D3800D8B03ED0A4C0D9FFA5C0DAFFDECFACF042
:101D4800DDCFADF02E0EAC250C6E000EAD210D6E64
:101D5800A4C0D9FFA5C0DAFF10EE2AF0DE50E126B4
:101D6800DD50E222E6CFAEF0E5CFAFF0BE51AE5F78
:101D7800BF51AF5B090ED890AE37AF37E82EFBD70F
:101D8800AE51B9250E6EAF51BA210F6E020E116E0B
:101D9800000E106EBEEC58F0A4C0D9FFA5C0DAFF43
:101DA80010EE04F0DE50E126DD50E222000EE76E70
:101DB800BCC0ACF0BDC0ADF0090ED8900001AC3786
:101DC800AD37E82EFAD7ACC0C6F0ADC0C7F0C0D06A
:101DD80020EE0AF0A451D926A551DA2210EE06F019
:101DE800A451E126A551E222DE50E65CDE50E65819
:101DF800DE50E658DE50E658D8A01FD0A4C0D9FF60
:101E0800A5C0DAFFDECF25F0DDCF26F047EC45F0A0
:101E18000009D8A460D0A4C0D9FFA5C0DAFF10EE8D
:101E28002AF0DE50E126DD50E222BEC0E6FFBFC048
:101E3800E6FFC0C0E6FFC1C0E6FF000120EE16F0D5
:101E4800A451D926A551DA22BEC0DEFFBFC0DEFFED
:101E5800C0C0DEFFC1C0DEFFFF0EAC6F010EAD6F6C
:101E680020EE06F0A451D926A551DA22DECFAEF035
:101E7800DDCFAFF0AC51AE17AD51AF17AE51000882
:101E8800C66FAF51D8A0E82A0208C76FC651A85D2F
:101E9800C751A959D8B004D0A8C0C6F0A9C0C7F086
:101EA800A4C0D9FFA5C0DAFFDECF3AF0DDCF3BF002
:101EB80020EE16F0A451D926A551DA22DECF3CF047
:101EC800DECF3DF0DECF3EF0DECF3FF084EC4FF0CA
:101ED8000009D8B402D0000116D6FF0E0001AC6F7D
:101EE800010EAD6F20EE06F0A451D926A551DA22D5
:101EF800DECFAEF0DDCFAFF0AC51AE17AD51AF17BE
:101F0800A4C0D9FFA5C0DAFFDECFB0F0DDCFB1F0B5
:101F1800AE51B027AF51B1232E0EB0250C6E000E76
:101F2800B1210D6EB9C00EF0BAC00FF0C6C010F0E6
:101F3800C7C011F0BEEC58F0A4C0D9FFA5C0DAFFA5
:101F480010EE04F0DE50E126DD50E222010EE76ECD
:101F58000001C651B927C751BA2320EE06F0A45193
:101F6800D926A551DA22C651DE26C751DE22000E37
:101F7800DE22DE22AAC0D9FFABC0DAFFC651DE26B8
:101F8800C751DD22C651A85FC751A95BA851A91145
:101F9800D8A405D520EE06F0A451D926A551DA22F9
:101FA80010EE0AF0A451E126A551E222DE50E65CCB
:101FB800DE50E658DE50E658DE50E658D8B014D069
:101FC80020EE06F0A451D926A551DA2210EE0AF027
:101FD800A451E126A551E222DECFE6FFDECFE6FFDF
:101FE800DECFE6FFDECFE6FF20EE04F0A451D926CF
:101FF800A551DA22000EDB8A000E1200A4C00DF0F3
:10200800A5C00EF0B4EC51F00001BE6FBE51D8B4BB
:1020180002D0BE51120020EE05F0A451D926A551D8
:10202800DA22DF50D8B408D020EE05F0A451D92622
:10203800A551DA22DF50120020EE0AF0A451D92669
:10204800A551DA22A651DE5CA751DE58A851DE5808
:10205800A951DE58D8B016D020EE04F0A451D926E4
:10206800A551DA22DFB20ED020EE0AF0A451D9260B
:10207800A551DA22DECFA6F0DECFA7F0DECFA8F09A
:10208800DECFA9F020EE06F0A451D926A551DA2218
:10209800DECFBAF0DECFBBF0DECFBCF0DECFBDF0D6
:1020A800000EBF6F000EC06F000EC16F000EC26F32
:1020B80020EE06F0A451D926A551DA22BFC0DEFFD2
:1020C800C0C0DEFFC1C0DEFFC2C0DEFFA651A7113F
:1020D800A811A911D8B42DD2A4C0D9FFA5C0DAFF80
:1020E80010EE02F0DE50E126DD50E222E750AA6F42
:1020F800AAC0ABF0AC6BAD6BAE6B090ED890AB372A
:10210800AC37AD37AE37E82EF9D7ABC0C3F0ACC0AB
:10211800C4F0ADC0C5F0AEC0C6F0BA51BB11BC1119
:10212800BD11D8B497D0FF0EA6250C6EFF0EA721BF
:102138000D6EFF0EA8210E6EFF0EA9210F6EC3C0F3
:1021480010F0C4C011F0C5C012F0C6C013F0CFEC37
:1021580052F00CC0AAF00DC0ABF00EC0ACF00FC02E
:10216800ADF0FF0E0001BA250C6EFF0EBB210D6EFF
:10217800FF0EBC210E6EFF0EBD210F6EC3C010F006
:10218800C4C011F0C5C012F0C6C013F0CFEC52F0B5
:102198000C500001AA5D0D50AB590E50AC590F50B0
:1021A800AD59D8A057D0FF0EC325AA6FFF0EC42182
:1021B800AB6FFF0EC521AC6FFF0EC621AD6FAA1D18
:1021C800AE6FAB1DAF6FAC1DB06FAD1DB16FFF0E25
:1021D800BA25B26FFF0EBB21B36FFF0EBC21B46FDF
:1021E800FF0EBD21B56FAE51B215B66FAF51B31525
:1021F800B76FB051B415B86FB151B515B96F20EEBE
:1022080006F0A451D926A551DA22B6C0DEFFB7C020
:10221800DEFFB8C0DEFFB9C0DEFF20EE06F0A45135
:10222800D926A551DA22DE50A65FDE50A75BDE5024
:10223800A85BDD50A95B20EE12F0A451D926A55168
:10224800DA22DECFC7F0DECFC8F0DECFC9F0DECFAE
:10225800CAF06ED020EE0EF0A451D926A551DA228C
:10226800DECFC7F0DECFC8F0DECFC9F0DECFCAF0D0
:10227800C751C811C911CA11D8A44CD0A4C0D9FFDC
:10228800A5C0DAFFDECF91F0DDCF92F0000E936F9C
:10229800000E946F000E956F000E966FDFEC2DF018
:1022A80091C0C7F092C0C8F093C0C9F094C0CAF0FA
:1022B8000001C705C811C911CA11D8A40AD020EE57
:1022C80005F0A451D926A551DA22020EDF6E020EBE
:1022D8001200C72911E1C8290FE1C9290DE1CA294E
:1022E800D8A40AD020EE05F0A451D926A551DA22A7
:1022F800010EDF6E010E120020EE0EF0A451D92659
:10230800A551DA22C7C0DEFFC8C0DEFFC9C0DEFFA4
:10231800CAC0DEFF20EE12F0A451D926A551DA2258
:10232800C7C0DEFFC8C0DEFFC9C0DEFFCAC0DEFF0F
:10233800C751C811C911CA11D8A497D0FAD020EE34
:1023480004F0A451D926A551DA22DFA22AD0A4C0CC
:10235800D9FFA5C0DAFFDECF91F0DDCF92F0C7C07C
:1023680093F0C8C094F0C9C095F0CAC096F0DFECED
:102378002DF091C0C7F092C0C8F093C0C9F094C0C6
:10238800CAF00001C751C811C911CA11D8A423D075
:10239800C3C0A6F0C4C0A7F0C5C0A8F0C6C0A9F0C5
:1023A8006ED0A4C0D9FFA5C0DAFFDECF60F0DDCFC4
:1023B80061F0C7C062F0C8C063F0C9C064F0CAC0A9
:1023C80065F03EEC24F060C0C7F061C0C8F062C0A0
:1023D800C9F063C0CAF00001C72907E1C82905E1AF
:1023E800C92903E1CA29D8B47DD7CA51C911C8116E
:1023F80004E1020EC75DD8A062D7A4C0D9FFA5C06A
:10240800DAFF10EE12F0DE50E126DD50E222E6504F
:10241800C75DE650C859E650C959E650CA59D8B000
:102428004ED720EE12F0A451D926A551DA22C7C002
:10243800DEFFC8C0DEFFC9C0DEFFCAC0DEFF20EE77
:1024480006F0A451D926A551DA22C351DE26C4517B
:10245800DE22C551DE22C651DE22C351A65FC45119
:10246800A75BC551A85BC651A95BA651C35DA7511F
:10247800C459A851C559A951C659D8A060D720EE4A
:1024880006F0A451D926A551DA22A651DE26A75175
:10249800DE22A851DE22A951DE22FF0EA615AA6F60
:1024A800010EA715AB6F000EA815AC6F000EA9158D
:1024B800AD6FAA51AB11AC11AD11D8B43AD0A4C0CC
:1024C800D9FFA5C0DAFFDECF18F0DDCF19F0C7C0FD
:1024D8001AF0C8C01BF0C9C01CF0CAC01DF0CDEC72
:1024E8004EF018C0BFF019C0C0F01AC0C1F01BC030
:1024F800C2F00001BF51C011C111C211D8B4DFD65A
:10250800A6C0AAF0A7C0ABF0A8C0ACF0A9C0ADF0B7
:102518000A0E05D0D890AD33AC33AB33AA33E82ECE
:10252800F9D7AA51BF27AB51C023AC51C123AD5134
:10253800C22320EE06F0A451D926A551DA22FF0EB7
:10254800DE14AA6F010EDE14AB6F000EDE14AC6F42
:10255800000EDE14AD6FAA51AB11AC11AD11D8B499
:1025680021D020EE16F0A451D926A551DA22BF5168
:10257800DE180AE1C051DE1807E1C151DE1804E196
:10258800C251DE18D8B40ED020EE16F0A451D926C8
:10259800A551DA22BFC0DEFFC0C0DEFFC1C0DEFF2A
:1025A800C2C0DEFF20EE06F0A451D926A551DA22DA
:1025B80010EE0AF0A451E126A551E222DE50E65CB5
:1025C800DE50E658DE50E658DE50E658D8B021D541
:1025D80020EE06F0A451D926A551DA2210EE0AF011
:1025E800A451E126A551E222DECFE6FFDECFE6FFC9
:1025F800DECFE6FFDECFE6FF20EE04F0A451D926B9
:10260800A551DA22000EDB8A04D58EC0A9F08FC04E
:10261800AAF092C0D9FF93C0DAFF000EDE6E000E5A
:10262800DD6E8CC00DF08DC00EF0B4EC51F00001E1
:10263800A46FA451D8B402D0A451120020EE05F022
:102648008C51D9268D51DA22DF50D8B408D020EE2B
:1026580005F08C51D9268D51DA22DF50120020EE78
:1026680004F08C51D9268D51DA22DFB002D0070E42
:10267800120020EE06F08C51D9268D51DA22DECFD9
:1026880094F0DECF95F0DECF96F0DECF97F020EE17
:102698000AF08C51D9268D51DA22DECF98F0DECFA0
:1026A80099F0DECF9AF0DECF9BF09451985DA06F41
:1026B80095519959A16F96519A59A26F97519B5963
:1026C800A36F9051946F9151956F966B976B94513E
:1026D800A05D9551A1599651A2599751A359D8B0C7
:1026E8005AD2A0C090F0A1C091F055D220EE06F0C9
:1026F8008C51D9268D51DA22FF0EDE14946F010E0B
:10270800DE14956F000EDE14966F000EDE14976FC0
:102718009451951196119711D8A4AFD120EE06F0D7
:102728008C51D9268D51DA22DECF94F0DECF95F088
:10273800DECF96F0DECF97F00A0E05D0D89097330B
:10274800963395339433E82EF9D78CC0D9FF8DC0D2
:10275800DAFF10EE02F0DE50E126DD50E222E7500B
:10276800986F98059415AB6FAB51D8A46FD020EE35
:1027780006F08C51D9268D51DA22DE50DE10DE109B
:10278800DE10D8A40FD020EE0EF08C51D9268D5132
:10279800DA22DECFA5F0DECFA6F0DECFA7F0DECFBF
:1027A800A8F020D08CC0D9FF8DC0DAFFDECF60F052
:1027B800DDCF61F020EE12F08C51D9268D51DA224E
:1027C800DECF62F0DECF63F0DECF64F0DECF65F0FF
:1027D8003EEC24F060C0A5F061C0A6F062C0A7F08E
:1027E80063C0A8F00001A851A711A6110EE1020EBE
:1027F800A55DD8B00AD020EE05F08C51D9268D51B0
:10280800DA22020EDF6E020E1200A52911E1A629B6
:102818000FE1A7290DE1A829D8A40AD020EE05F0D8
:102828008C51D9268D51DA22010EDF6E010E12006D
:1028380020EE12F08C51D9268D51DA22A5C0DEFF88
:10284800A6C0DEFFA7C0DEFFA8C0DEFF8CC0D9FF90
:102858008DC0DAFFDECF18F0DDCF19F020EE12F0D0
:102868008C51D9268D51DA22DECF1AF0DECF1BF03B
:10287800DECF1CF0DECF1DF0CDEC4EF018C0ACF072
:1028880019C0ADF01AC0AEF01BC0AFF00001AC51DA
:10289800AD11AE11AF11D8B4AED7AB51AC27000E05
:1028A800AD23AE23AF2390C094F091C095F0090EEC
:1028B800966FD89095339433962FFBD794C0B0F089
:1028C80095C0B1F0B051B111D8B4C9D0AB51B02551
:1028D800946F000EB121956F8CC0D9FF8DC0DAFFBF
:1028E80010EE02F0DE50E126DD50E222E750966F4E
:1028F800976B9451965D95519759D8B012D08CC06A
:10290800D9FF8DC0DAFF10EE02F0DE50E126DD506F
:10291800E222E750946FAB51945DB06FB16BD8A0D1
:10292800B107A9C01BF0AAC01CF0ACC01DF0ADC017
:102938001EF0AEC01FF0AFC020F0B0C021F0B1C093
:1029480022F08CC0D9FF8DC0DAFF10EE01F0DE5006
:10295800E126DD50E222E75006EC4EF00009D8A44B
:10296800CBD08CC0D9FF8DC0DAFF10EE04F0DE505A
:10297800E126DD50E222E750D8B461D00001B05121
:10298800946FB151956F966B976B8CC0D9FF8DC0C2
:10299800DAFF10EE2AF0DE50E126DD50E222E6CF23
:1029A80098F0E6CF99F0E6CF9AF0E6CF9BF0AC51DD
:1029B800985D9C6FAD5199599D6FAE519A599E6F14
:1029C800AF519B599F6F94519C5D95519D5996515C
:1029D8009E5997519F59D8B032D08CC0D9FF8DC01D
:1029E800DAFF10EE2AF0DE50E126DD50E222E6CFD3
:1029F80094F0E5CF95F0AC51945FAD51955B090E1D
:102A0800D89094379537E82EFBD79451A9250C6EAA
:102A18009551AA210D6E8CC0D9FF8DC0DAFFDECF8B
:102A280096F0DDCF97F02E0E96250E6E000E9721AC
:102A38000F6E020E116E000E106EBEEC58F0B0C094
:102A480094F0B1C095F0090ED890000194379537ED
:102A5800E82EFAD794C0B2F095C0B3F07ED020EE3D
:102A680016F08C51D9268D51DA22ACC0DEFFADC0EC
:102A7800DEFFAEC0DEFFAFC0DEFFFF0E946F010EBB
:102A8800956F20EE06F08C51D9268D51DA22DECFD3
:102A980096F0DDCF97F09451961795519717965168
:102AA8000008B26F9751D8A0E82A0208B36FB25154
:102AB800905DB3519159D8B004D090C0B2F091C094
:102AC800B3F08CC0D9FF8DC0DAFFDECF3AF0DDCF8E
:102AD8003BF020EE16F08C51D9268D51DA22DECF4C
:102AE8003CF0DECF3DF0DECF3EF0DECF3FF084ECB1
:102AF8004FF00009D8B402D0000190D6A9C00CF05C
:102B0800AAC00DF0FF0E0001946F010E956F20EE24
:102B180006F08C51D9268D51DA22DECF96F0DDCF22
:102B280097F094519617955197178CC0D9FF8DC07F
:102B3800DAFFDECF98F0DDCF99F0965198279751BC
:102B480099232E0E98250E6E000E99210F6EB2C095
:102B580010F0B3C011F0BEEC58F00001B251A92733
:102B6800B351AA2320EE06F08C51D9268D51DA22D2
:102B7800B251DE26B351DE22000EDE22DE2292C0E2
:102B8800D9FF93C0DAFFB251DE26B351DD22B2512C
:102B9800905FB351915B90519111D8A4A7D5000EC5
:102BA8001200296E000E286E2FD22950D8A40DD0FD
:102BB8000001FE51D8B409D0000E286E000E0101A4
:102BC800816F0A0E47D0839091D2020E2918D8A49B
:102BD8000BD00001FE51D8B407D0000E286E000EAD
:102BE8000101816F140E36D01F0E296435D0300EC6
:102BF800296032D00001FE51D8B42ED02950E00F00
:102C0800FF6F000E286EFF51200D1E0EF324D96EA3
:102C1800020EF420DA6EDE50DE10DE10DE10D8B4BC
:102C280003D0030EFF652FD0010E4D6EFF51140D1A
:102C3800130EF324D96E010EF420DA6EFF51140D31
:102C4800130EF324E16E010EF420E26EE75004093E
:102C5800DF6E19D0806FB7D73F0E296419D0500E98
:102C6800296016D00001FE51D8B412D0FF51140DBE
:102C7800000EF324D96E010EF420DA6E2950C00F2D
:102C8800DF6E000E286E000E0101816F000EE2D784
:102C9800340E2918D8A40BD00001FE51D8B407D09F
:102CA800000E0101816F000E806F000EABD1350E52
:102CB8002918D8A40BD00001FE51D8B407D0000EB3
:102CC800286E0D0E0101816FAC0EC4D7370E29187E
:102CD800D8A409D00001FE51D8B405D00E0E0101C8
:102CE800816F750E87D10D0E2918D8A40BD000015D
:102CF800FE51D8B407D0000E286E020E0101816F74
:102D0800BC0EA8D7100E2918D8A409D00001FE516E
:102D1800D8B405D0030E0101816FE90E6BD1180EEE
:102D28002918D8A409D00001FE51D8B405D0070E3F
:102D38000101816F090E5ED13E0E2918D8A4D6D1A3
:102D48000001FE51D8B4D2D10F0E0101816F3D0EA2
:102D580051D10001FF51140D010EF324D96E010E5B
:102D6800F420DA6E29C0DFFF030E0101816FEA0E3D
:102D780041D10001FF51140D020EF324D96E010E4A
:102D8800F420DA6E29C0DFFF030E0101816FEB0E1C
:102D980031D10001FF51140D030EF324D96E010E39
:102DA800F420DA6E29C0DFFF030E0101816FEC0EFB
:102DB80021D10001FF51140D040EF324D96E010E28
:102DC800F420DA6E29C0DFFF030E0101816FED0EDA
:102DD80011D10001FF51140D050EF324D96E010E17
:102DE800F420DA6E29C0DFFF030E0101816FEE0EB9
:102DF80001D10001FF51140D060EF324D96E010E06
:102E0800F420DA6E29C0DFFFFF51140D060EF324FB
:102E1800D96E010EF420DA6EDF500C6E0CC00DF086
:102E28000E6A0F6A106A0FC010F00EC00FF00DC0C6
:102E38000EF00D6AFF51140D050EF324D96E010E24
:102E4800F420DA6EDF50116E11C012F0136A146AA2
:102E5800156A13C015F012C014F0136A126AFF51F4
:102E6800140D040EF324D96E010EF420DA6EDF502F
:102E7800166E16C017F0186A196A1A6A17C01AF07F
:102E8800196A186A176AFF51140D030EF324D96ED4
:102E9800010EF420DA6EDF501B6E1B5017241C6ED7
:102EA800000E18201D6E000E19201E6E000E1A202E
:102EB8001F6E12501C24206E13501D20216E1450BA
:102EC8001E20226E15501F20236E0D502024246EC4
:102ED8000E502120256E0F502220266E10502320E0
:102EE800276EFF51140D070EF324D96E010EF4203E
:102EF800DA6E24C0DEFF25C0DEFF26C0DEFF27C055
:102F0800DEFF000E0101816F000E74D00001FF5139
:102F1800140D120EF324D96E010EF420DA6E29C0B6
:102F2800DFFF070E0101816F0A0E64D00001FF5117
:102F3800140D110EF324D96E010EF420DA6E29C097
:102F4800DFFF070E0101816F0B0E54D00001FF5106
:102F5800140D100EF324D96E010EF420DA6E29C078
:102F6800DFFF070E0101816F0C0E44D00001FF51F5
:102F7800140D0F0EF324D96E010EF420DA6E29C059
:102F8800DFFFBFD729C000F20F0E0101816F3E0E8F
:102F980031D029C001F20F0E0101816F3F0E2AD0F6
:102FA80029C002F20F0E0101816F400E23D029C003
:102FB80003F20F0E0101816F410E1CD029C004F2EB
:102FC8000F0E0101816F420E15D029C005F20F0EB8
:102FD8000101816F430E0ED029C006F20F0E0101C8
:102FE800816F440E07D029C007F28BD70E0E01015E
:102FF800816F760E806F7AD0000E0101816F000E0E
:10300800806F090E286EDFD580C10CF081C10DF0EC
:103018000D50000AD8B416D0030AD8B418D0040A40
:10302800D8B429D00A0AD8B434D0030AD8B437D0CF
:10303800010AD8B43CD0130AD8B453D03B0AD8B448
:1030480053D054D00C50000AD8B4AFD54FD00C5040
:10305800E90AD8B47ED6030AD8B48BD6010AD8B404
:1030680098D6070AD8B4A5D6010AD8B4B2D6030AA6
:10307800D8B4BFD63BD00C50090AD8B447D7030AF6
:10308800D8B454D7010AD8B461D7070AD8B46ED7D0
:103098002DD00C50480AD8B434D7E40A27D00C50A5
:1030A800750AD8B4A3D7030AD8B4A6D71FD00C5032
:1030B8003D0AD8B467D7030AD8B46BD7010AD8B485
:1030C8006FD77F0AD8B473D7010AD8B477D7030A61
:1030D800D8B47BD7010AD8B47FD7070AD8B483D726
:1030E80005D00C502A0A02D00C500F0A28501200A2
:1030F800000165516411631104E1020E625DD8A0FC
:1031080010D020EE12F06051D9266151DA22DE503B
:10311800625DDE506359DE506459DE506559D8A0AF
:1031280054D2020E8E6F67D262C08CF063C08DF0ED
:10313800D8908D316B6F8C316A6F6A518C276B51C7
:103148008D2360C03AF061C03BF020EE1EF0605164
:10315800D9266151DA22DECF6AF0DECF6BF0DECFFE
:103168006CF0DECF6DF08CC06EF08DC06FF0090E84
:10317800706FD8906F336E33702FFBD76E516A25FE
:103188003C6E6F516B213D6E000E6C213E6E000E41
:103198006D213F6E84EC4FF000018E6F8E51D8A4E4
:1031A8002AD2FF0E6A6F010E6B6F8CC06CF08DC057
:1031B8006DF06A516C176B516D1760C06EF061C08D
:1031C8006FF06C516E276D516F232E0E6E258F6F29
:1031D800000E6F21906F8C4B8D2B62B104D066C0AE
:1031E80088F0896B1AD066516A6F6B6B6A3B6B3BD0
:1031F800F00E6B176A510F0B6B13F00E6A178FC026
:10320800D9FF90C0DAFFDF500F0B6C6F6D6B6A51FE
:103218006C11886F6B516D11896F8FC0D9FF90C089
:10322800DAFF88C0DFFF20EE04F06051D926615133
:10323800DA22010EDF6E60C03AF061C03BF020EE8A
:103248001EF06051D9266151DA22DECF6AF0DECF56
:103258006BF0DECF6CF0DECF6DF08CC06EF08DC001
:103268006FF0090E706FD8906F336E33702FFBD7E5
:103278006E516A253C6E6F516B213D6E000E6C21BC
:103288003E6E000E6D213F6E84EC4FF000018E6F94
:103298008E51D8A4B0D1FF0E6A6F010E6B6F8CC02F
:1032A8006CF08DC06DF06A516C176B516D1760C072
:1032B8006EF061C06FF06C516E276D516F232E0E4A
:1032C8006E258F6F000E6F21906F62B11BD066C0A4
:1032D8006AF067C06BF068C06CF069C06DF06BC0D5
:1032E8006AF06CC06BF06DC06CF06D6B0F0E6A17F6
:1032F8008FC0D9FF90C0DAFFDF50F00B6A116E6FF4
:103308006E5112D066C06AF067C06BF068C06CF08E
:1033180069C06DF0050E05D0D8906D336C336B33F2
:103328006A33E82EF9D76A518A6F8B6B8FC0D9FF41
:1033380090C0DAFF8AC0DFFF3FD160C03AF061C0B9
:103348003BF020EE1EF06051D9266151DA22DECF23
:103358006AF0DECF6BF0DECF6CF0DECF6DF062C0CE
:103368006EF063C06FF064C070F065C071F06FC03C
:103378006EF070C06FF071C070F0716B6A516E259D
:103388003C6E6B516F213D6E6C5170213E6E6D51DC
:1033980071213F6E84EC4FF000018E6F8E51D8A4DE
:1033A8002AD1FF0E6A6F010E6B6F62C06CF063C0AA
:1033B8006DF0D8906C376D376A516C176B516D177B
:1033C80060C06EF061C06FF06C516E276D516F2355
:1033D8002E0E6E258F6F000E6F21906F8FC0D9FF54
:1033E80090C0DAFF66C0DFFF20EE01F08F51D926CA
:1033F8009051DA226751DF6EDFD060C03AF061C0C9
:103408003BF020EE1EF06051D9266151DA22DECF62
:103418006AF0DECF6BF0DECF6CF0DECF6DF062C00D
:103428006EF063C06FF064C070F065C071F0080E94
:1034380005D0D890713370336F336E33E82EF9D7D7
:103448006A516E253C6E6B516F213D6E6C51702137
:103458003E6E6D5171213F6E84EC4FF000018E6F0E
:103468008E51D8A4C8D0FF0E6A6F010E6B6F62C070
:103478006CF063C06DF0D8906C376D37D8906C37AE
:103488006D376A516C176B516D1760C06EF061C073
:103498006FF06C516E276D516F232E0E6E258F6F56
:1034A800000E6F21906F20EE01F08F51D9269051B8
:1034B800DA22DF506A6F6A516C6F6B6B20EE02F094
:1034C8008F51D9269051DA22DF506D6F6DC06EF0A2
:1034D8006F6B706B716B6FC071F06EC070F06F6B5B
:1034E8006E6B20EE03F08F51D9269051DA22DF500F
:1034F800726F72C073F0746B756B766B73C076F015
:10350800756B746B736B6E517311776F6F517411A8
:10351800786F70517511796F715176117A6F6B519F
:1035280077117B6F6C5178117C6F000E79117D6F6C
:10353800000E7A117E6F8FC0D9FF90C0DAFFDF507E
:103548007F6F7F517B11806F7C51816F7D51826FBE
:103558007E51836F000E8015846F000E8115856F74
:10356800000E8215866FF00E8315876F84516613DF
:103578008551671386516813875169138FC0D9FF26
:1035880090C0DAFF66C0DFFF20EE01F08F51D92628
:103598009051DA226751DF6E20EE02F08F51D92662
:1035A8009051DA2268C0DFFF20EE03F08F51D92650
:1035B8009051DA2269C0DFFF20EE04F06051D9266D
:1035C8006151DA22010EDF6E16D060C0D9FF61C0EA
:1035D800DAFFDF506A6F6B6B6B51000AD8A4A1D574
:1035E8006A51010AD8B4A0D5030AD8B4A6D6010AEC
:1035F800D8B403D796D58E5112000001DD51DE11E3
:10360800D8A402D0090E1200DDC0D9FFDEC0DAFF4F
:10361800000EDE6E000EDD6E8AC1C7F18BC1C8F1E7
:103628001F0EE117C70E846F010E856FDF0E866FC0
:10363800000E876FE151FE0B886FB8EC00F00101B6
:10364800C46FC451D8A453D2B00EDB6F010EDC6F27
:10365800C70E0001BD6F010EBE6FDFC0BFF0E0C036
:10366800C0F04AEC42F00101C46FD9C1C5F1DAC11A
:10367800C6F1C451D8A406D0C551C611D8A402D0E9
:10368800060EC46FE1C0E2F01C0E0001E217D8B4C8
:103698001ED10101C451D8B414D0040EC419D8A441
:1036A80009D0C70E0001C16F010EC26F9BEC4DF02F
:1036B8000101C46F0001E187D9C1C5F1DAC1C6F1C2
:1036C80014D020EE0BF0C551D926C651DA22DF50AE
:1036D8000001E26F110EE217D8B402D0070E03D032
:1036E800E1A503D0080E0101C46F0101C451D8A49B
:1036F8000AD10001E1A707D1010120EE0EF0C55162
:10370800D926C651DA22000EDF6E20EE0FF0C55121
:10371800D926C651DA22000EDF6E20EE10F0C55110
:10372800D926C651DA22210EDF6E20EE11F0C551DE
:10373800D926C651DA22460EDF6E20EE16F0C551A4
:10374800D926C651DA22000EDF6E20EE17F0C551D9
:10375800D926C651DA22000EDF6E20EE18F0C551C8
:10376800D926C651DA22210EDF6E20EE19F0C55196
:10377800D926C651DA22460EDF6E20EE0BF0C5516F
:10378800D926C651DA22000EDF6E20EE1CF0C55194
:10379800D926C651DA22000EDF6E20EE1DF0C55183
:1037A800D926C651DA22000EDF6E20EE1EF0C55172
:1037B800D926C651DA22000EDF6E20EE1FF0C55161
:1037C800D926C651DA22000EDF6EC7C10CF0C8C177
:1037D8000DF0C5C10EF0C6C10FF06BEC4EF00CC079
:1037E800BCF10DC0BDF10EC0BEF10FC0BFF1C5C127
:1037F8000CF0C6C10DF0000E0E6E000E0F6E000E1E
:10380800106E000E116E5CEC58F0010120EE04F011
:10381800C751D926C851DA22010EDF6EBC51BD113D
:10382800BE11BF11D8B46FD020EE2AF0C751D926E7
:10383800C851DA22DECFC0F1DECFC1F1DECFC2F14E
:10384800DECFC3F1C7C191F0C8C192F0BCC193F0FB
:10385800BDC194F0BEC195F0BFC196F0F3EC45F040
:103868000101C46FC451D8A44ED0FF0EBC2500017D
:10387800E26FFF0E0101BD210001E36FFF0E0101A0
:10388800BE210001E46FFF0E0101BF210001E56FB9
:10389800010120EE0AF0C751D926C851DA22E2C048
:1038A800DEFFE3C0DEFFE4C0DEFFE5C0DEFFC7C128
:1038B8003AF0C8C13BF0C0C13CF0C1C13DF0C2C143
:1038C8003EF0C3C13FF084EC4FF001011BD0010171
:1038D800C451D8A418D020EE0BF0C551D926C65132
:1038E800DA22DFA802D0040E0DD00001E1A30BD02C
:1038F800010120EE0BF0C551D926C651DA22DFA00E
:1039080002D0070EC46F0101C451D8A423D000010E
:10391800E1B7E18B010120EE2AF0C751D926C85141
:10392800DA22000110EE1AF0DD51E126DE51E22222
:10393800DECFE6FFDECFE6FFDECFE6FFDECFE6FF37
:1039480020EE1EF0DD51D926DE51DA22C5C1DEFF98
:10395800C6C1DDFF0101C451D8A4C9D0000120EEC1
:1039680004F0DD51D926DE51DA22E1C0DFFF20EE76
:1039780005F0DD51D926DE51DA22000EDF6EC7C10F
:103988000CF0C8C10DF0C5C10EF0C6C10FF06BEC4C
:103998004EF0000120EE0EF0DD51D926DE51DA227C
:1039A8000CC0DEFF0DC0DEFF0EC0DEFF0FC0DEFF65
:1039B800010120EE1DF0C551D926C651DA22DF508B
:1039C8000001E26FE251E46FE36B010120EE1EF0AB
:1039D800C551D926C651DA22DF500001E56FE5C08E
:1039E800E6F0E76BE86BE96BE7C0E9F0E6C0E8F002
:1039F800E76BE66B010120EE1FF0C551D926C651D1
:103A0800DA22DF500001EA6FEAC0EBF0EC6BED6BF5
:103A1800EE6BEBC0EEF0ED6BEC6BEB6BE651EB1184
:103A2800EF6FE751EC11F06FE851ED11F16FE951CB
:103A3800EE11F26FE351EF11F36FE451F011F46FEF
:103A4800000EF111F56F000EF211F66F010120EE74
:103A58001CF0C551D926C651DA22DF500001F76F94
:103A6800F751F311F86FF451F96FF551FA6FF651F8
:103A7800FB6F20EE0AF0DD51D926DE51DA22F8C0BC
:103A8800DEFFF9C0DEFFFAC0DEFFFBC0DEFF20EE7E
:103A980006F0DD51D926DE51DA22DE6ADE6ADE6AF8
:103AA800DD6A20EE16F0DD51D926DE51DA22DE6A13
:103AB800DE6ADE6ADD6ADDC0D9FFDEC0DAFFC7C1B3
:103AC800DEFFC8C1DDFFDDC0D9FFDEC0DAFF10EEC2
:103AD80006F0DE50E126DD50E22220EE02F0DD5154
:103AE800D926DE51DA22E6CFDEFFE5CFDDFF010180
:103AF800C45112002B6E1CC042F01DC043F02B5065
:103B0800D8B402D0040E1200010E406E51A016D295
:103B1800030E120026EC5BF00009D8B430D2000E78
:103B28000BD2000E156E000E166E000E176E000EEC
:103B3800186E090E7DEC58F00009D8A420D22C0E7E
:103B48000C6E000E0D6E000E0F6E100E0E6E22EC37
:103B580055F00009D8B413D22C44E846030BE80604
:103B6800D8A44ED033C01EF03F0E1E161EC01FF044
:103B7800206A216A226A20C022F01FC021F0206A30
:103B88001F6A3450246E236A3550256E266A2350E6
:103B980025262450262225501F24276E2650202013
:103BA800286E000E2120296E000E22202A6E010E9A
:103BB80027243C6E000E28203D6E000E29203E6E04
:103BC800000E2A203F6E3CC01EF03DC01FF03EC0D4
:103BD80020F03FC021F00A0ED8901E361F3620363E
:103BE8002136E82EF9D71CC0D9FF1DC0DAFF1EC048
:103BF800DEFF1FC0DEFF20C0DEFF21C0DEFF8FD743
:103C08001E6A36AE01D01E2A010E1E1631C01FF0E4
:103C18000F0E1F163550030B020DF3501F241E24E0
:103C2800020F416E3250030B1E6E1F6A0A0ED890A7
:103C38001E361F36E82EFBD73350206E216AD890E7
:103C480020362136D890203621363444E846030BF6
:103C5800226E236A20502226215023221E5022261B
:103C68001F502322010E2226000E232222C03CF0E0
:103C780023C03DF03E6A3F6A41C01EF0F70E1E2683
:103C88003CC01FF03DC020F03EC021F03FC022F0F4
:103C98001E2A05D0D8901F362036213622361E2EF1
:103CA800F9D73BD04EA446D0000E156E000E166E06
:103CB800000E176E000E186E8D0E7DEC58F0000980
:103CC800D8A45DD195EC5BF02C0E0C6E000E0D6E39
:103CD800000E0F6E100E0E6E22EC55F00009D8B4CF
:103CE8004ED1300E416E03D095EC5BF04106415049
:103CF800D8A4FAD736C01EF01E3A0F0E1E16100EA4
:103D08001F6E206A216A226A1E2A05D0D8901F36A3
:103D18002036213622361E2EF9D71CC0D9FF1DC0E9
:103D2800DAFF1FC0DEFF20C0DEFF21C0DEFF22C099
:103D3800DEFFF5D6000E156E000E166E000E176E1D
:103D4800000E186E090E7DEC58F00009D8A417D1A2
:103D58002C0E0C6E000E0D6E000E0F6E100E0E6EF9
:103D680022EC55F00009D8B40AD14EA22AD039C0A5
:103D78001EF0060E1F6ED8901E321F2EFCD7FF0EA7
:103D88001E2636503F0B206E216AD89020362136E9
:103D9800226A37AE01D0222A010E2216225020268E
:103DA800000E2122010E2026000E21221E2A03D0F9
:103DB800D890203621361E2EFBD72050236E215056
:103DC80034D036C01EF0D8901E32D8901E321F0E46
:103DD8001E16010E1E240C6E0D6A000E0D223750A1
:103DE800030B1F6E206AD8901F362036D8901F36D6
:103DF8002036D8901F36203637C021F0050E226EA7
:103E0800D8902132222EFCD7070E211621501F26CA
:103E1800000E2022010E1F240E6E000E20200F6EB1
:103E2800E2EC5AF00C50236E0D50246E256A266A77
:103E38001CC0D9FF1DC0DAFF23C0DEFF24C0DEFF8F
:103E480025C0DEFF26C0DEFF6AD642C0D9FF43C0C8
:103E5800DAFF4EC0DFFF63D6000E156E000E166E39
:103E6800000E176E000E186E090E7DEC58F0000952
:103E7800D8A485D042C00CF043C00DF0000E0F6EE0
:103E8800100E0E6E22EC55F00009D8A448D677D053
:103E9800000E156E000E166E000E176E000E186ED0
:103EA8000A0E7DEC58F00009D8A469D042C00CF085
:103EB80043C00DF0000E0F6E100E0E6E22EC55F082
:103EC800E3D7000E156E000E166E000E176E000E6C
:103ED800186E3A0E7DEC58F00009D8A450D0040EA4
:103EE800416E0AD095EC5BF042C0D9FF43C0DAFFBF
:103EF800DF6E424A432A41064150D8B410D6F2D761
:103F0800000E156E000E166E000E176E000E186E5F
:103F18008D0E7DEC58F00009D8A431D095EC5BF0FB
:103F280042C00CF043C00DF0000E0F6E400E0E6E36
:103F380022EC55F0A9D7040E406E21D01B501E6EFE
:103F48001F6A1F50000AD8A4F6D71E50000AD8B41A
:103F5800E1D5010AD8B4E5D5020AD8B4A3D6090A2E
:103F6800D8B473D7010AD8B477D7070AD8B490D78A
:103F7800010AD8B4A6D7030AD8B4C2D7DCD7A1ECB3
:103F88005BF04050120019C0F6FF1AC0F7FF080096
:103F9800F5CF89F0194A1A2A00018951D8B41200BC
:103FA800250E8919D8B404D0895169EC5BF0EBD798
:103FB800000E856F000E846F19C0F6FF1AC0F7FF58
:103FC8000800F5CF89F0194A1A2A300E8919D8A4A1
:103FD8000ED0000E856F010E846F19C0F6FF1AC04F
:103FE800F7FF0800F5CF89F0194A1A2A08D02D0ED4
:103FF8008919D8A404D0000E856F020EEDD7000EE3
:104008007D6F000E7C6F1ED07CC00CF07DC00DF063
:10401800000E0F6E0A0E0E6EE2EC5AF00001895186
:104028000C26000E0D22D00E0C247C6FFF0E0D20E6
:104038007D6F19C0F6FF1AC0F7FF0800F5CF89F0A9
:10404800194A1A2A2F0E896503D0390E8965DCD7DB
:104058006C0E8919D8B404D04C0E8919D8A40AD08A
:10406800848519C0F6FF1AC0F7FF0800F5CF89F05C
:10407800194A1A2A8951D8B4120089C088F0600EEA
:1040880088658DD0200E885F8AD01BC0D9FF1CC0E0
:10409800DAFFDFCF1DF0020EDE26DFCF1EF0000EA6
:1040A800DD221DC0D9FF1EC0DAFFDECF78F0DDCFDC
:1040B80079F0000E7F6F000E7E6F03D000017E4BFB
:1040C8007F2B7E5178251D6E7F5179211E6E1DC074
:1040D800F6FF1EC0F7FF000EF86E0E0EF76403D051
:1040E8000800F55005D0F6CFE9FFF7CFEAFFEF500B
:1040F8000009D8B404D0E2D7200E69EC5BF00001C7
:1041080084B30CD07E511D6E7F511E6E7E4B7F2B6B
:104118007C511D5C7D511E58D8A0EED778C00DF09B
:1041280079C00EF032EC57F003D0200E69EC5BF04A
:1041380000017E511D6E7F511E6E7E4B7F2B7C5180
:104148001D5C7D511E58D8B01ED7EFD71BC0D9FFB4
:104158001CC0DAFFDFCF1DF0020EDE26DFCF1EF017
:10416800000EDD221DC0D9FF1EC0DAFFDF5069EC4A
:104178005BF009D7000E7B6F020E0BD0000E7B6F31
:10418800080E07D0000E7B6F0A0E03D0000E7B6F5F
:10419800100E7A6F22D0895169EC5BF0F4D6885101
:1041A8001D6E1E6A1E50000AD8A4F5D71D50420A7B
:1041B800D8B4E0D7010AD8B4C9D7070AD8B4E2D727
:1041C8000B0AD8B4DBD71C0AD8B45FD7060AD8B410
:1041D800D9D70D0AD8B4DAD7DED784B541D0440E82
:1041E8008819D8B41BD01BC0D9FF1CC0DAFFDFCF99
:1041F8001DF0020EDE26DFCF1EF0000EDD221DC0F0
:10420800D9FF1EC0DAFFDECF1FF0DDCF20F01FC0C0
:1042180070F020C071F0726B736B19D01BC0D9FF9E
:104228001CC0DAFFDFCF1DF0020EDE26DFCF1EF046
:10423800000EDD221DC0D9FF1EC0DAFFDECF70F0F0
:10424800DDCF71F0000E71BFFF0E726F736F70C01B
:1042580080F071C081F072C082F073C083F018D012
:104268001BC0D9FF1CC0DAFFDFCF1DF0040EDE260D
:10427800DFCF1EF0000EDD221DC0D9FF1EC0DAFF01
:10428800DECF80F0DECF81F0DECF82F0DECF83F0AC
:10429800440E8819D8B483AF0AD0806D811FD8B076
:1042A800812B821FD8B0822B000E83578487000E83
:1042B800876F000E866F80C00CF081C00DF082C041
:1042C8000EF083C00FF07AC010F07BC011F0126AB4
:1042D800136A8AEC55F00C500001886F80C00CF00E
:1042E80081C00DF082C00EF083C00FF07AC010F0CC
:1042F8007BC011F0126A136ACFEC52F00CC080F048
:104308000DC081F00EC082F00FC083F0090E0001CD
:1043180088650ED0780E8919D8B404D0000E756F50
:10432800070E03D0000E756F270E746F745188271F
:10433800600E8625D96E000E8721DA6E8851300FFF
:10434800DF6E864B872B8051811182118311D8B47F
:1043580006D0875104E1100E865DD8A0ACD784A79B
:104368000AD0600E8625D96E000E8721DA6E2D0ED2
:10437800DF6E864B872B86C07EF087C07FF084B1C6
:1043880004D0000E776F200E03D0000E776F300E2A
:10439800766F76C088F003D0885169EC5BF0000135
:1043A80084B30CD07E511D6E7F511E6E7E4B7F2BC9
:1043B8007C511D5C7D511E58D8A0EED78607D8A029
:1043C8008707600E8625D96E000E8721DA6EDF50CA
:1043D80069EC5BF0000186518711D8B404D0EED7A0
:1043E800200E69EC5BF000017E511D6E7F511E6E40
:1043F8007E4B7F2B7C511D5C7D511E58D8B0C3D598
:10440800EFD7116E0D50D8A4FEEC51F0000E106ECF
:104418000C50D8B4C3D111507F0B116E040E111873
:10442800D8B404D0140E1118D8A40AD0000E010173
:104438007F6F000E7E6F000E0D6E070E0C6E120061
:104448003F0E1118D8A40CD0000E4B6E000E0101BF
:104458007F6F000E7E6F000E0D6E000E0C6E120048
:104468005F0E1118D8A40CD0000E4C6E000E01017E
:104478007F6F000E7E6F000E0D6E000E0C6E120028
:104488003F0E116407D05F0E116004D0400E111862
:10449800D8A4EAD7400E1118D8A40ED0010E4C6E3D
:1044A800000E4B6E000E01017F6F000E7E6F000E36
:1044B8000D6E000E0C6E1200200E1118D8A46ED1CD
:1044C800010E4B6E000E01017F6F000E7E6F000E15
:1044D8000D6E000E0C6E1200600E1118D8A40DD0CF
:1044E8004C50D8B40AD001019451D8B402D0080E67
:1044F80001D0030E106E000E27D0600E1118D8A43C
:104508000BD04B50D8B408D001019451D8B402D084
:10451800090EF0D7050EEED7680E1118D8A40AD0E8
:104528004B50D8B407D01A0E01017F6F900E22D1DC
:1045380083809CD1680E1118D8A40AD04C50D8B4E6
:1045480007D0020E106E65D07F6F000E7E6F8ED181
:104558006A0E1118D8A408D04B50D8B405D01A0E3A
:1045680001017F6FF40E06D16C0E1118D8A408D083
:104578004B50D8B405D01A0E01017F6F2C0EFAD01B
:10458800700E1118D8A40AD04C50D8B407D0040E15
:10459800106E000E01017F6F000EECD0700E111826
:1045A800D8A464D14B50D8B461D11B0E01017F6FE0
:1045B800620EE0D08380020E1118D8A405D01A0E1E
:1045C80001017F6F920E7E6F050E1118D8A405D0D9
:1045D8001A0E01017F6FAE0E7E6F070E1118D8A458
:1045E80005D01A0E01017F6FB80E7E6F080E1118E4
:1045F800D8A405D01A0E01017F6FCC0E7E6F030E72
:104608001118D8B403D01128D8A406D0000E106E03
:104618008390000E010198D7160E1118D8A426D140
:104628001A0E01017F6FA40E91D7050E1118D8A498
:104638001DD11A0E01017F6FF50E88D711C0FFF04A
:104648001A0E01017F6F9B0E81D71A0E01017F6F31
:104658009C0E7CD70001FF51070D500EF324D96E34
:10466800010EF420DA6E11C0DFFF1A0E01017F6F10
:104678009D0E6CD70001FF51070D510EF324D96E22
:10468800010EF420DA6E11C0DFFF1A0E01017F6FF0
:104698009E0E5CD70001FF51070D520EF324D96E10
:1046A800010EF420DA6E11C0DFFF000E01017F6FEA
:1046B800000E7E6F010E64D01A0E01017F6FB90ED5
:1046C80059D01A0E01017F6FBA0E40D71A0E010198
:1046D8007F6FBB0E3BD7000E01017F6F000E7E6F10
:1046E80041D0000E01017F6F000E7E6F060E48D08C
:1046F80011C0FFF0000E01017F6F000E7E6F000EEB
:1047080030D0000E0101946F1A0E7F6FF70EE7D7B5
:104718001A0E01017F6FF70E19D78390270E01013A
:104728007F6F0F0E13D7180E1118D8A49FD01A0E2A
:1047380001017F6F2D0E0AD71A0E01017F6F2E0E11
:1047480005D71A0E01017F6F2F0E00D71A0E01012F
:104758007F6F300EFBD6000E01017F6F000E7E6F5B
:104768000A0E106E839082D0040E106E270E01017F
:104778007F6F0F0E7E6FDCD68380000E010109D09B
:10478800106E74D08390010E0101946F080E106EA4
:10479800000E7F6F000E7E6F000EF2D77EC10EF006
:1047A8007FC10FF00F50000AD8B40AD01A0AD8B443
:1047B8000CD0010AD8B450D03C0AD8B455D056D041
:1047C8000E50000AD8B488D651D00E502C0AD8B44E
:1047D800AAD7010AD8B4B0D7030AD8B4B2D7010A05
:1047E800D8B4B4D71F0AD8B4B6D7A00AD8B4E2D67A
:1047F800020AD8B423D7090AD8B427D7070AD8B4E5
:1048080029D7010AD8B436D7030AD8B443D73A0A05
:10481800D8B467D70A0AD8B4B5D7160AD8B44CD7CB
:10482800010AD8B44ED7030AD8B450D7010AD8B46D
:1048380052D7790AD8B485D60E0AD8B459D7380AC7
:10484800D8B4F3D6010AD8B45CD7030AD8B460D771
:10485800010AD8B462D70AD00E50580AD8B484D7FF
:104868003A0AD8B489D702D00E500F0A10C00CF0FB
:104878000D6A1200000165516411631104E1020E12
:10488800625DD8A010D020EE12F06051D926615197
:10489800DA22DE50625DDE506359DE506459DE5024
:1048A8006559D8A008D0010E846F000E856F000EE0
:1048B800866F000EF4D18469856986698769F1D1AC
:1048C80062C088F063C089F0D8908931676F8831F9
:1048D800666F665188276751892360C03AF061C0C6
:1048E8003BF020EE1EF06051D9266151DA22DECF6E
:1048F80066F0DECF67F0DECF68F0DECF69F088C003
:104908006AF089C06BF0090E6C6FD8906B336A330C
:104918006C2FFBD76A5166253C6E6B5167213D6E43
:10492800000E68213E6E000E69213F6E84EC4FF048
:104938000009D8A4CCD1FF0E0001666F010E676F85
:1049480088C068F089C069F06651681767516917AF
:1049580060C06AF061C06BF068516A2769516B23C7
:104968002E0E6A25D96E000E6B21DA6EDF506C6F41
:104978006C51826F836B884B892B60C03AF061C0A1
:104988003BF020EE1EF06051D9266151DA22DECFCD
:1049980066F0DECF67F0DECF68F0DECF69F088C062
:1049A8006AF089C06BF0090E6C6FD8906B336A336C
:1049B8006C2FFBD76A5166253C6E6B5167213D6EA3
:1049C800000E68213E6E000E69213F6E84EC4FF0A8
:1049D8000009D8A47CD1FF0E0001666F010E676F35
:1049E80088C068F089C069F066516817675169170F
:1049F80060C06AF061C06BF068516A2769516B2327
:104A08002E0E6A25D96E000E6B21DA6EDF506C6FA0
:104A18006C516E6F6D6B6D5182136E51831362B161
:104A280007D0FF0E8215806F0F0E8315816F0FD090
:104A380082C066F083C067F0040E686FD890673351
:104A48006633682FFBD766C080F067C081F080C0EE
:104A580084F081C085F069D060C03AF061C03BF055
:104A680020EE1EF06051D9266151DA22DECF66F0C1
:104A7800DECF67F0DECF68F0DECF69F062C06AF0A3
:104A880063C06BF064C06CF065C06DF06BC06AF019
:104A98006CC06BF06DC06CF06D6B66516A253C6E36
:104AA80067516B213D6E68516C213E6E69516D21D5
:104AB8003F6E84EC4FF00009D8A409D1FF0E000125
:104AC800666F010E676F62C068F063C069F0D890C6
:104AD80068376937665168176751691760C06AF0A7
:104AE80061C06BF068516A2769516B232E0E6A25E5
:104AF8008A6F000E6B218B6F20EE01F08A51D92648
:104B08008B51DA22DF50666F6651686F676B8AC017
:104B1800D9FF8BC0DAFFDF50696F69516713000E48
:104B2800681367C084F068C085F0866B876BCFD048
:104B380060C03AF061C03BF020EE1EF06051D9260B
:104B48006151DA22DECF66F0DECF67F0DECF68F0A3
:104B5800DECF69F062C06AF063C06BF064C06CF0CD
:104B680065C06DF0080E05D0D8906D336C336B338B
:104B78006A33E82EF9D766516A253C6E67516B2176
:104B88003D6E68516C213E6E69516D213F6E84EC1B
:104B98004FF00009D8A49BD0FF0E0001666F010EEC
:104BA800676F62C068F063C069F0D890683769378A
:104BB800D89068376937665168176751691760C0B8
:104BC8006AF061C06BF068516A2769516B232E0E39
:104BD8006A258A6F000E6B218B6F20EE01F08A51D7
:104BE800D9268B51DA22DF50666F6651686F676B82
:104BF80020EE02F08A51D9268B51DA22DF50696FF4
:104C080069C06AF06B6B6C6B6D6B6BC06DF06AC0E2
:104C18006CF06B6B6A6B20EE03F08A51D9268B51CE
:104C2800DA22DF506E6F6EC06FF0706B716B726B53
:104C38006FC072F0716B706B6F6B6A516F11736F2D
:104C48006B517011746F6C517111756F6D517211D8
:104C5800766F67517311776F68517411786F000E12
:104C68007511796F000E76117A6F8AC0D9FF8BC0E3
:104C7800DAFFDF507B6F7B5177117C6F78517D6F46
:104C880079517E6F7A517F6FFF0E7C15846FFF0E0E
:104C98007D15856FFF0E7E15866F0F0E7F15876F4A
:104CA80016D060C0D9FF61C0DAFFDF50666F676B4E
:104CB8006751000AD8A4F7D56651010AD8B400D6BE
:104CC800030AD8B4C9D6010AD8B432D7ECD584C0FF
:104CD80060F085C061F086C062F087C063F01200A2
:104CE800140E00018C6F020E8D6F340E8E6F0B0E3A
:104CF8008F6F020E916F000E906FE50E926F000E8F
:104D0800936F09EC13F04F6E140E00018A6FFE0EBC
:104D18008B6FE5C08CF0E6C08DF035EC5BF0000ED3
:104D28000001E86F000EE76F000EE26F000EE16F02
:104D3800000EEA6F000EE96FC30EE925D96E000E6A
:104D4800EA21DA6E000EDF6ED20EE925D96E000E6A
:104D5800EA21DA6E000EDF6EE94BEA2BEABFECD7E8
:104D6800EA5104E10F0EE95DD8A0E6D7000EEC6F1A
:104D7800000EEB6F59D1340EEB25D96E0B0EEC21DA
:104D8800DA6E0D0EDE18D8A409D18E0E0C6EFF0E49
:104D98000D6EC30E0E6E000E0F6ED7EC4FF00C505A
:104DA8000D10D8A409D0D20E136E000E146E34EC78
:104DB80047F013500101E76F880E0C6EFF0E0D6E61
:104DC800C30E0E6E000E0F6ED7EC4FF00C500D1088
:104DD800D8A409D0D20E136E000E146E34EC47F02E
:104DE80013500101A36F6D0E0C6EFF0E0D6EC30EF6
:104DF8000E6E000E0F6ED7EC4FF00C500D10D8A4AD
:104E080009D0D20E136E000E146E34EC47F0135016
:104E180001019F6FD30E0C6EFF0E0D6EC30E0E6E4A
:104E2800000E0F6ED7EC4FF00C500D10D8A409D01F
:104E3800D20E136E000E146E34EC47F013500101BD
:104E48009D6F000E0001EE6F000EED6FB40E826FC5
:104E5800000E836F740E846FFF0E856FEDC086F0B1
:104E6800EEC087F05DEC57F0B40E0C6E000E0D6EC0
:104E7800C30E0E6E000E0F6ED7EC4FF00C500D10D7
:104E8800D8A41AD0EDC00CF0EEC00DF0000E0F6ED5
:104E98000F0E0E6EE2EC5AF0340E0C24126E0D0E4C
:104EA8000D20136ED20E146E000E156E000E176EC6
:104EB8000F0E166E50EC56F00001ED4BEE2BEEBFC8
:104EC800C5D7EE5104E1100EED5DD8A0BFD7000E96
:104ED800EE6F010EED6FB40E826F000E836F7B0EC6
:104EE800846FFF0E856FEDC086F0EEC087F05DEC35
:104EF80057F0B40E0C6E000E0D6EC30E0E6E000E43
:104F08000F6ED7EC4FF00C500D10D8A41AD0EDC08E
:104F18000CF0EEC00DF0000E0F6E0F0E0E6EE2ECF0
:104F28005AF0240E0C24126E0E0E0D20136ED20EA3
:104F3800146E000E156E000E176E0F0E166E50ECE6
:104F480056F00001ED4BEE2BEEBFC5D7EE5104E154
:104F5800040EED5DD8A0BFD7000EEA6F000EE96F12
:104F6800C30EE925D96E000EEA21DA6E000EDF6E57
:104F7800D20EE925D96E000EEA21DA6E000EDF6E38
:104F8800E94BEA2BEABFECD7EA5104E10F0EE95DE1
:104F9800D8A0E6D7000EE26F000E17D0340EEB252E
:104FA800D96E0B0EEC21DA6E0A0EDE18D8B43AD0A0
:104FB800340EEB25D96E0B0EEC21DA6E200EDE18BE
:104FC800D8A409D0000EE26F010EE16F000EE86F61
:104FD800000EE76F27D0E151E211D8B40BD0340EA0
:104FE800EB25D96E0B0EEC21DA6ED20EE725E16EB9
:104FF800000E0AD0340EEB25D96E0B0EEC21DA6EBA
:10500800C30EE725E16E000EE821E26EDFCFE7FF71
:10501800E8BF06D0E85106E10F0EE75DD8B002D030
:10502800E74BE82BEB4BEC2BE551EB5DE651EC59EC
:10503800D8A0A1D6040E8A6FFE0E8B6F9FC18CF08C
:105048008D6B35EC5BF0600E00018A6FFE0E8B6F86
:10505800E7C18CF08D6B35EC5BF0510E00018A6F67
:10506800FE0E8B6FA3C18CF08D6B35EC5BF0000EE0
:105078000001EE6F000EED6FEDC00CF0EEC00DF00C
:10508800000E0F6E0F0E0E6EE2EC5AF0340E0C246A
:105098000001E36F0D0E0D20E46F920E8A6FFD0E76
:1050A8008B6FEDC08CF0EEC08DF0E3C08EF0E4C0E5
:1050B8008FF035EC5BF00001ED4BEE2BEEBFDCD74B
:1050C800EE5104E1100EED5DD8A0D6D7000EEC6FBE
:1050D800010EEB6FEBC00CF0ECC00DF0000E0F6E84
:1050E8000F0E0E6EE2EC5AF0240E0C240001E36F52
:1050F8000E0E0D20E46FA30E8A6FFD0E8B6FEBC0B2
:105108008CF0ECC08DF0E3C08EF0E4C08FF035EC8D
:105118005BF00001EB4BEC2BECBFDCD7EC5104E16E
:10512800040EEB5DD8A0D6D7B40E8A6FFB0E8B6F3A
:1051380035EC5BF01200000120EE04F0A451D926F2
:10514800A551DA22DECFA8F0DDCFA9F0010EA825FF
:10515800B16F000EA921B26FB151B211D8B40CD001
:1051680020EE0EF0A451D926A551DA22DE50DE1029
:10517800DE10DE10D8A402D0040E12000F0EB115F6
:10518800A86F000EB215A96FA851A911D8A4A4D16F
:1051980020EE0EF0A451D926A551DA22DE2A000EFF
:1051A800DE22DE22DE2220EE0AF0A451D926A55105
:1051B800DA22DE50DE10DE10DE10D8A411D0A4C032
:1051C800D9FFA5C0DAFF10EE08F0DE50E126DD5069
:1051D800E222E650B15DE650B259D8B0CDD77CD1C5
:1051E800B1C0A8F0B2C0A9F0040EAA6FD890A93334
:1051F800A833AA2FFBD7FF0EAB6FFF0EAC6FA4C06E
:10520800D9FFA5C0DAFF10EE02F0DE50E126DD502E
:10521800E222E750AD6FAE6BAB51AD27AC51AE2378
:10522800A851AD17A951AE17AD51AE11D8A454D19C
:10523800A4C0D9FFA5C0DAFFDECF60F0DDCF61F0F2
:1052480020EE0AF0A451D926A551DA22DECF62F069
:10525800DECF63F0DECF64F0DECF65F03EEC24F005
:1052680060C0B3F061C0B4F062C0B5F063C0B6F01E
:105278000001B651B511B41106E1020EB35DD8B004
:1052880002D0020E1200B32909E1B42907E1B529B9
:1052980005E1B629D8A402D0010E1200A4C0D9FF96
:1052A800A5C0DAFF10EE12F0DE50E126DD50E22252
:1052B800E650B35DE650B459E650B559E650B659D4
:1052C800D8A0DBD0A651A711D8B456D7A4C0D9FF0F
:1052D800A5C0DAFFDECF91F0DDCF92F020EE0AF024
:1052E800A451D926A551DA22DECF93F0DECF94F06F
:1052F800DECF95F0DECF96F0DFEC2DF091C0B3F065
:1053080092C0B4F093C0B5F094C0B6F00001B351A8
:10531800B411B511B611D8A402D0070E1200B30506
:10532800B411B511B611D8B4ACD7B32907E1B42973
:1053380005E1B52903E1B629D8B4AED7A4C0D9FF91
:10534800A5C0DAFFDECF25F0DDCF26F047EC45F02B
:105358000009D8A4A1D7A4C0D9FFA5C0DAFFDECF21
:10536800A8F0DDCFA9F02E0E0001A8250C6E000EC6
:10537800A9210D6E000E0F6E000E0E6E020E116E3C
:10538800000E106E92EC5AF0A4C0D9FFA5C0DAFF47
:10539800DECF18F0DDCF19F0B3C01AF0B4C01BF09F
:1053A800B5C01CF0B6C01DF0CDEC4EF0A4C0D9FFBE
:1053B800A5C0DAFF10EE2AF0DE50E126DD50E22229
:1053C80018C0E6FF19C0E6FF1AC0E6FF1BC0E6FFDB
:1053D800000E0001B06F000EAF6F2BD0A4C0D9FF34
:1053E800A5C0DAFF10EE04F0DE50E126DD50E2221F
:1053F800010EE76EA4C0D9FFA5C0DAFFDECF25F005
:10540800DDCF26F047EC45F00009D8A445D7A4C065
:10541800D9FFA5C0DAFF10EE2AF0DE50E126DD50F4
:10542800E222E62A000EE622E622E6220001AF4B3F
:10543800B02BA4C0D9FFA5C0DAFF10EE02F0DE50F1
:10544800E126DD50E222E750A86FA96BA851AF5DB5
:10545800A951B059D8A0C2D7A4C0D9FFA5C0DAFFB6
:1054680010EE2AF0DE50E126DD50E222AF51E65E72
:10547800B051E65A000EE65AE65A20EE0AF0A45158
:10548800D926A551DA22B3C0DEFFB4C0DEFFB5C00D
:10549800DEFFB6C0DEFFA4C0D9FFA5C0DAFFDECFAD
:1054A80018F0DDCF19F0B3C01AF0B4C01BF0B5C0C6
:1054B8001CF0B6C01DF0CDEC4EF0000120EE0EF051
:1054C800A451D926A551DA2218C0DEFF19C0DEFF83
:1054D8001AC0DEFF1BC0DEFF20EE04F0A451D9265F
:1054E800A551DA22B1C0DEFFB2C0DDFF0F0EB11543
:1054F800A86F000EB215A96F050ED890A837A93766
:10550800E82EFBD7A4C0D9FFA5C0DAFFDECFAAF0EA
:10551800DDCFABF0A851AA27A951AB232E0EAA279D
:10552800000EAB2320EE12F0A451D926A551DA22A1
:10553800AAC0DEFFABC0DDFF000E120044C025F09C
:1055480045C026F047EC45F0466E4650D8A499D1A0
:1055580044C0D9FF45C0DAFF030EDE18D8A47DD1B8
:1055680020EE05F04450D9264550DA22DE04D8A4AE
:1055780074D12E0E44240C6E000E45200D6E000EC4
:105588000F6E000E0E6E020E116E000E106E92EC73
:105598005AF022EE2CF04450D9264550DA22550E06
:1055A800DF6E22EE2DF04450D9264550DA22AA0E9D
:1055B800DF6E20EE2EF04450D9264550DA22520EE6
:1055C800DF6E20EE2FF04450D9264550DA22520ED5
:1055D800DF6E20EE30F04450D9264550DA22610EB5
:1055E800DF6E20EE31F04450D9264550DA22410EC4
:1055F800DF6E22EE12F04450D9264550DA22720EA0
:10560800DF6E22EE13F04450D9264550DA22720E8E
:10561800DF6E22EE14F04450D9264550DA22410EAE
:10562800DF6E22EE15F04450D9264550DA22610E7D
:10563800DF6E20EE0EF04450D9264550DA2212EEE5
:1056480016F04450E1264550E222DFCFE7FF22EE74
:1056580017F04450D9264550DA2210EE0EF0445087
:10566800E1264550E222E6CF60F0E5CF61F061C067
:1056780060F00001616B6051DF6E22EE18F044505B
:10568800D9264550DA2210EE0EF04450E126455056
:10569800E222E6CF60F0E6CF61F0E6CF62F0E6CF37
:1056A80063F0110E05D0D8906333623361336033F1
:1056B800E82EF9D76051DF6E22EE19F04450D92652
:1056C8004550DA2210EE0EF04450E1264550E22211
:1056D800E6CF60F0E6CF61F0E6CF62F0E6CF63F0A8
:1056E800190E05D0D8906333623361336033E82EE6
:1056F800F9D76051DF6E20EE0AF04450D9264550A4
:10570800DA2212EE1AF04450E1264550E222DFCFA9
:10571800E7FF22EE1BF04450D9264550DA2210EE5E
:105728000AF04450E1264550E222E6CF60F0E5CF8A
:1057380061F061C060F0616B6051DF6E22EE1CF0B9
:105748004450D9264550DA2210EE0AF04450E1269A
:105758004550E222E6CF60F0E6CF61F0E6CF62F096
:10576800E6CF63F0110E05D0D8906333623361330E
:105778006033E82EF9D76051DF6E22EE1DF04450F9
:10578800D9264550DA2210EE0AF04450E126455059
:10579800E222E6CF60F0E6CF61F0E6CF62F0E6CF36
:1057A80063F0190E05D0D8906333623361336033E8
:1057B800E82EF9D76051DF6E20EE1AF04450D92652
:1057C8004550DA22DECF60F0DECF61F0DECF62F046
:1057D800DECF63F0010E6025646F000E6121656FF6
:1057E800000E6221666F000E6321676F20EE2AF0BB
:1057F8004450D9264550DA2264C0DEFF65C0DEFF7A
:1058080066C0DEFF67C0DEFF2E0E44241B6E000E4E
:1058180045201C6E20EE2AF04450D9264550DA2245
:10582800DECF1DF0DECF1EF0DECF1FF0DECF20F082
:10583800000E226E010E216E20EE01F04450D92692
:105848004550DA22DF5024EC4AF020EE05F04450AF
:10585800D9264550DA22000EDF6E000E1B6E000EB0
:105868001C6E000E1D6E20EE01F04450D9264550E6
:10587800DA22DF507EEC1DF00009D8B402D0010E08
:10588800466E46501200838011EC43F0CBC0B7F14E
:10589800CCC0B8F10101B751B811D8B41BD0000180
:1058A800FF51140D130EF324D96E010EF420DA6E95
:1058B800FF51140D130EF324E16E010EF420E26E75
:1058C800E7500409DF6E3CEC59F0B7C1E2F0B8C10B
:1058D800E3F012000001FF51140D070EF324D96EF6
:1058E800010EF420DA6E6CC1E9F06DC1EAF06EC108
:1058F800EBF0E86B000EE825EC6F010EE921ED6F87
:10590800000EEA21EE6F000EEB21EF6FDE50EC196E
:1059180044E1DE50ED1941E1DE50EE193EE1DE5082
:10592800EF19D8A43AD010EC53F010C0BBF111C055
:10593800BCF112C0BDF113C0BEF1000EE8CF34FBBC
:105948002BEE35F0BEC1DFFF000EE8CF36FB2BEEA5
:1059580037F0BDC1DFFF000EE8CF38FB2BEE39F082
:10596800BCC1DFFF000EE8CF3AFB2BEE3BF0BBC11A
:10597800DFFF5350FD0B536E010E246E000E236E95
:105988008EEC3AF05350FD0B536E000E4D6E839023
:105998004DC0E2F00001E36B1200FF51140D0F0E31
:1059A800F324D96E010EF420DA6EDECFE4F0DECFF8
:1059B800E5F0DECFE6F0DECFE7F0E5C0E4F0E6C0E4
:1059C800E5F0E7C0E6F0E76BE4C0B0F1E5C0B1F19F
:1059D800FF51140D0F0EF324D96E010EF420DA6E68
:1059E800DECFE4F0DDCFE5F0E4510101B96FBA6B29
:1059F8005350FD0B536E000EB66F000EB56F000EC0
:105A0800B36F000EB26F70D0FF0EE46FFF0EE56F3C
:105A1800B0C1E6F0B1C1E7F0E451E627E551E7236C
:105A28000101B2510001E6190EE10101B351000173
:105A3800E719D8A408D00101B951BA11D8A403D0E4
:105A480053500209536E0001FF51200D140EF32428
:105A58008C6F020EF4208D6F340E8E6F0B0E8F6FCD
:105A6800010E916F000E906FBF0E926F010E936F33
:105A780009EC13F00101B46FB451D8A410D7BFC119
:105A880023F0C0C124F08EEC3AF00101BF51B525D6
:105A9800B56FC051B621B66F0001FF51140D070E46
:105AA800F324D96E010EF420DA6E000EDE24E46FC2
:105AB800010EDE20E56F000EDE20E66F000EDE2010
:105AC800E76FFF51140D070EF324D96E010EF42071
:105AD800DA6EE4C0DEFFE5C0DEFFE6C0DEFFE7C049
:105AE800DEFF0101B24BB32BB051B25DB351800A56
:105AF8000001E46F0101B151800A0001E459D8A006
:105B080083D70101BABF3ED7BA5103E1B905D8A07E
:105B180039D70001FF51200D140EF3248C6F020EAB
:105B2800F4208D6F340E8E6F0B0E8F6FB9C190F00D
:105B3800BAC191F0BF0E926F010E936F09EC13F08A
:105B48000101B46FB451D8A4AAD653500209536EB8
:105B5800B9C123F0BAC124F08EEC3AF00101BF516B
:105B6800B525B56FC051B621B66F0001FF51140DB0
:105B7800070EF324D96E010EF420DA6E000EDE242F
:105B8800E46F010EDE20E56F000EDE20E66F000EEA
:105B9800DE20E76FFF51140D070EF324D96E010EB6
:105BA800F420DA6EE4C0DEFFE5C0DEFFE6C0DEFF0B
:105BB800E7C0DEFFE7D600019351941195119611C5
:105BC800D8A42DD020EE0AF09151D9269251DA228C
:105BD800DECF98F0DECF99F0DECF9AF0DECF9BF0E3
:105BE800985199119A119B11D8B410D020EE12F047
:105BF8009151D9269251DA22DE50985DDE5099599A
:105C0800DE509A59DE509B59D8A05BD0010E986F90
:105C1800000E996F000E9A6F000E9B6F52D091C0C4
:105C280060F092C061F093C062F094C063F095C0D8
:105C380064F096C065F03EEC24F060C0A0F061C04E
:105C4800A1F062C0A2F063C0A3F00001A351A211A9
:105C5800A1110DE1020EA05DD8B009D0010E916F1F
:105C6800000E926F000E936F000E946F1200A02921
:105C780010E1A1290EE1A2290CE1A329D8A409D099
:105C8800A0C091F0A1C092F0A2C093F0A3C094F07C
:105C9800120020EE12F09151D9269251DA22DE50EC
:105CA800A05DDE50A159DE50A259DE50A359D8A0FC
:105CB800E7D793C098F094C099F095C09AF096C031
:105CC8009BF098C09CF099C09DF09AC09EF09BC034
:105CD8009FF0010E9C27000E9D239E239F2320EEFC
:105CE80012F09151D9269251DA22DE509C5DDE5095
:105CF8009D59DE509E59DE509F59D8A019D0020EEA
:105D08009C6F000E9D6F000E9E6F000E9F6F9B5143
:105D18009A1199110DE1020E985DD8B009D0000EC4
:105D2800916F000E926F000E936F000E946F120029
:105D380091C060F092C061F09CC062F09DC063F0B9
:105D48009EC064F09FC065F03EEC24F060C0A0F0F7
:105D580061C0A1F062C0A2F063C0A3F00001A0512D
:105D6800A111A211A311D8B41DD0A02907E1A1291E
:105D780005E1A22903E1A329D8B482D7A005A1117E
:105D8800A211A311D8B47CD798519C19A2E19951BA
:105D98009D199FE19A519E199CE19B519F19D8B476
:105DA800BED797D791C060F092C061F09CC062F0F6
:105DB8009DC063F09EC064F09FC065F0FF0E666FE3
:105DC800FF0E676FFF0E686F0F0E696F7CEC18F09F
:105DD8000001976F9751D8A41ED093519411951133
:105DE8009611D8B418D091C060F092C061F093C0F9
:105DF80062F094C063F095C064F096C065F09CC0F2
:105E080066F09DC067F09EC068F09FC069F07CECAA
:105E180018F00001976F9751D8A431D020EE0AF0FE
:105E28009151D9269251DA229CC0DEFF9DC0DEFF37
:105E38009EC0DEFF9FC0DEFF20EE0EF09151D926F6
:105E48009251DA22DE2807E1DE2805E1DE2803E1A7
:105E5800DE28D8B424D020EE0EF09151D9269251E4
:105E6800DA22DE06000EDE5ADE5ADE5A20EE05F091
:105E78009151D9269251DA22000EDB8010D0970575
:105E8800D8B409D0010E9C6F000E9D6F000E9E6F56
:105E9800000E9F6F04D09C699D699E699F699CC094
:105EA80091F09DC092F09EC093F09FC094F01200B4
:105EB80016C0D9FF17C0DAFFDECF24F0DDCF25F0FA
:105EC80002D0244A252A24C0F6FF25C0F7FF000E79
:105ED800F86E0E0EF76403D00800F55005D0F6CF23
:105EE800E9FFF7CFEAFFEF502F0AD8B4EAD724C06A
:105EF800F6FF25C0F7FF000EF86E0E0EF76403D00C
:105F08000800F55005D0F6CFE9FFF7CFEAFFEF50CC
:105F18005C0AD8B4D6D720EE14F01450D926155000
:105F2800DA22DECF26F0DDCF27F026C00CF027C01E
:105F38000DF0000E0F6E200E0E6E000E116E0B0E81
:105F4800106E92EC5AF0000E206E20C028F0296ADC
:105F580028C01EF029C01FF0000E226E080E216E08
:105F68001E502424186E1F502520196E18C0F6FFE5
:105F780019C0F7FF000EF86E0E0EF76403D0080084
:105F8800F55005D0F6CFE9FFF7CFEAFFEF502A6EBC
:105F98001E4A1F2A200E2A64AFD02F0E2A18D8B402
:105FA800ABD05C0E2A18D8B4A7D02E0E2A18D8B4B5
:105FB80006D02150285C22502958D8A018D0080EA5
:105FC80021182210D8A404D02E0E2A18D8B402D032
:105FD800060E1200000E296E080E286E000E226EA4
:105FE8000B0E216ED8902036D8902036B9D77F0E68
:105FF8002A6402D0030E2012800E2A6403D09F0E5A
:106008002A6406D0DF0E2A644ED0FD0E2A604BD0DB
:106018001E502424186E1F502520196E18C0F6FF34
:1060280019C0F7FF000EF86E0E0EF76403D00800D3
:10603800F55005D0F6CFE9FFF7CFEAFFEF50236E12
:106048001E4A1F2A3F0E236403D07E0E236406D007
:106058007F0E2364BDD7FD0E2360BAD7FF0E186EDE
:10606800FF0E196E21C01AF022C01BF018501A2614
:1060780019501B221A50285C1B502958D8B0A8D791
:1060880028502624D96E29502720DA6E2AC0DFFF2F
:10609800284A292A28502624D96E29502720DA6E22
:1060A80023C0DFFF26D0330E0C6EFE0E0D6E2AC005
:1060B8000EF00F6AD1EC57F00C500D10D8A488D709
:1060C800400E2A6405D05B0E2A6002D0208209D0D7
:1060D800600E2A6406D07B0E2A6003D02080200E32
:1060E8002A5E28502624D96E29502720DA6E2AC025
:1060F800DFFF284A292A34D71E502424186E1F503F
:106108002520196E16C0D9FF17C0DAFF18C0DEFFA8
:1061180019C0DDFF200E2A6404D0000E1D6E000E8B
:1061280003D0000E1D6E040E1C6E1CC02AF02850F1
:106138002910D8B44DD726C0D9FF27C0DAFFE50EFD
:10614800DE18D8A406D026C0D9FF27C0DAFF050E6E
:10615800DF6E080E21182210D8A404D0D89020365B
:10616800D89020362050030BE806D8B42A8820504F
:106178000C0B040AD8B42A8620EE0BF02650D92638
:106188002750DA222AC0DFFF000E120020EE04F0AA
:106198004550D9264650DA2247C0DEFF48C0DDFF09
:1061A80020EE06F04550D9264650DA22DECF99F087
:1061B800DECF9AF0DECF9BF0DECF9CF00001990590
:1061C8009A119B119C11D8B414D045C0D9FF46C070
:1061D800DAFF10EE12F0DE50E126DD50E222E65042
:1061E800995DE6509A59E6509B59E6509C59D8A0BB
:1061F80002D0020E120099519A119B119C11D8A439
:1062080022D045C0D9FF46C0DAFFDECF8CF0DDCF03
:106218008DF08CC0D9FF8DC0DAFF030EDE18D8A42C
:1062280012D045C0D9FF46C0DAFF10EE22F0DE508A
:10623800E126DD50E222E6CF99F0E6CF9AF0E6CFEC
:106248009BF0E6CF9CF099519A119B119C11D8A410
:1062580023D045C0D9FF46C0DAFF10EE08F0DE5063
:10626800E126DD50E222E650475CE6504858D8B0B7
:10627800C0D745C0D9FF46C0DAFF10EE22F0DE5085
:10628800E126DD50E222E6CF95F0E6CF96F0E6CFA4
:1062980097F0E6CF98F079D045C0D9FF46C0DAFF2D
:1062A80010EE02F0DE50E126DD50E222E7508C6F5E
:1062B8008C51100DF3CF93F0F4CF94F046D045C035
:1062C800D9FF46C0DAFFDECF60F0DDCF61F099C0BC
:1062D80062F09AC063F09BC064F09CC065F03EEC2D
:1062E80024F060C099F061C09AF062C09BF063C06E
:1062F8009CF00001992909E19A2907E19B2905E108
:106308009C29D8A402D0010E12009C519B119A110D
:1063180004E1020E995DD8A06CD745C0D9FF46C0EC
:10632800DAFF10EE12F0DE50E126DD50E222E650F0
:10633800995DE6509A59E6509B59E6509C59D8B059
:1063480058D79351475E9451485A9351475C94519A
:106358004858D8B0B4D745C0D9FF46C0DAFFDECF19
:1063680018F0DDCF19F099C01AF09AC01BF09BC045
:106378001CF09CC01DF0CDEC4EF018C095F019C073
:1063880096F01AC097F01BC098F020EE0AF045501E
:10639800D9264650DA2299C0DEFF9AC0DEFF9BC09C
:1063A800DEFF9CC0DEFF00019551961197119811F0
:1063B800D8B41FD747C08CF048C08DF0040E8E6F3C
:1063C800D8908D338C338E2FFBD78C5195258F6FBA
:1063D8008D519621906F000E9721916F000E982194
:1063E800926F20EE0EF04550D9264650DA228FC023
:1063F800DEFF90C0DEFF91C0DEFF92C0DEFF0F0E11
:1064080047148C6F000E48148D6F050ED8908C378A
:106418008D37E82EFBD745C0D9FF46C0DAFFDECF5F
:106428008EF0DDCF8FF08C518E278D518F232E0E5D
:106438008E27000E8F2320EE12F04550D9264650A5
:10644800DA228EC0DEFF8FC0DDFF000E1200000EC4
:106458000101E26F0A0EE16F000EE06F050EDF6FBB
:106468003ED1000EE26F140EE16F30D1130E0D6EA7
:10647800FD0E0E6E32EC57F08FB205D0000E010102
:10648800E26F1E0EE16F290E0101DE6F960EDD6FC1
:106498007F0EE82EFED7DD2FFCD7DE2FFAD716D1D8
:1064A800EB0E0D6EFE0E0E6E32EC57F0060E00016E
:1064B800DD6F090EDE6FB60EDF6FFB0EE06F000EAC
:1064C800E16F2AEC4FF04F6E4F50F0EC55F04F5003
:1064D800D8A4D9D7000E0101E26F230ED3D76F0ECF
:1064E8000D6EFE0E0E6E32EC57F0140E0001DD6FCD
:1064F800020EDE6F0E0EDF6FFF0EE06F010EE16F12
:1065080001EC1BF04F6E4F50F0EC55F04F50D8A4F3
:106518000AD074EC26F0140E0001736F020E746F2B
:106528009EEC58F04F6E4F50F0EC55F0000E010104
:10653800E26F280EE16F9F51D8A40ED0000EE86FCD
:10654800340E0001826F0D0E836FC50E846FFE0E30
:10655800856F5DEC57F00DD01C0E00018A6FFC0EA4
:106568008B6F9FC18CF08D6BE8C18EF08F6B35EC13
:106578005BF07E0E00018A6FFE0E8B6F0101E85101
:106588000F0D340EF32400018C6F0D0EF4208D6F67
:1065980035EC5BF078D7E50E00018A6FFC0E8B6F47
:1065A8000101E8510F0D340EF32400018C6F0D0E1C
:1065B800F4208D6F35EC5BF0140E0001DD6F020ED8
:1065C800DE6F0101E8510F0D340EF3240001DF6F77
:1065D8000D0EF420E06F030EE16F01EC1BF04F6E1F
:1065E8004F50D8A405D0000E0101E26F3C0EE16FB8
:1065F800040E4F18D8A447D7000E0101E26F320EDF
:1066080041D74D0E00018A6FFD0E8B6F0101E851D5
:106618000F0D340EF32400018C6F0D0EF4208D6FD6
:1066280035EC5BF0140E0001DD6F020EDE6F010128
:10663800E8510F0D340EF3240001DF6F0D0EF42026
:10664800E06F070EE16F01EC1BF04F6E4F50D8A4BE
:106658001AD7000E0101E26F3C0E14D7270E000175
:106668008A6FFD0E8B6F0101E8510F0D340EF32474
:1066780000018C6F0D0EF4208D6F35EC5BF0000E71
:106688000001FD6F010EFC6F1200E1C1DDF1E2C1F6
:10669800DEF1DE51000AD8A419D0DD510A0AD8B4B7
:1066A800E0D61E0AD8B4E2D60A0AD8B4F9D63D0A0A
:1066B800D8B415D70B0AD8B46ED7050AD8B406D003
:1066C8001F0AD8B49ED70E0AD8B4C8D7140E010131
:1066D800E119E211D8B403D0DF07D8A0E007E0BF82
:1066E80005D0E051D2E1DF05D8B0CFD7000E0001C8
:1066F800FD6F000EFC6F1200340E0101BC6F0B0E13
:10670800BD6FEBC012F0ECC013F03AEC58F0125029
:106718000101B06FCB0E0001A46F000EA56F000E33
:10672800A66F000EA76F000EA86F000EA96F02ECEF
:1067380010F00101B96FB951D8B411D06E0E000133
:106748008A6FFC0E8B6F35EC5BF0000E0001CB6F8F
:10675800000ECC6F000ECD6F000ECE6F1200CB0E68
:1067680000018C6F000E8D6FBCC18EF0BDC18FF023
:10677800010E916F000E906FB70E926F010E936F1E
:1067880009EC13F00101B96FB951D8B408D0CE0E95
:1067980000018A6FFC0E8B6F35EC5BF0D6D7BCC15D
:1067A800D9FFBDC1DAFF800EDE18D8B408D0700E4C
:1067B80000018A6FFD0E8B6F35EC5BF0C6D720EEBB
:1067C8000AF0BC51D926BD51DA22DF500001ED6F25
:1067D800ED51EF6FEE6B010120EE0BF0BC51D926A5
:1067E800BD51DA22DF500001F06FF051EE250101B2
:1067F800B56F000E0001EF210101B66FB70E000161
:106808008A6FFC0E8B6FB5C18CF0B6C18DF035EC7C
:106818005BF0CB0E0001A46F000EA56F0101B5510E
:106828000001EE6FED6BEDC0A6F0EEC0A7F0A86B0F
:10683800A96B02EC10F00101B96FB951D8A485D742
:10684800CB0E00018C6F000E8D6FBCC18EF0BDC1E8
:106858008FF0010E916F000E906FB70E926F010EC0
:10686800936F09EC13F00101B96FB951D8A46DD732
:10687800000EBB6F000EBA6FEBC00CF0ECC00DF051
:10688800BAC1EDF0BBC1EEF0050ED8900001ED37AE
:10689800EE37E82EFAD7ED510101BC250E6E000146
:1068A800EE510101BD210F6EB0C110F0116A7AECF2
:1068B80050F00C500D10D8A45FD0BAC1EDF0BBC198
:1068C800EEF0050ED8900001ED37EE37E82EFAD736
:1068D800BCC1EFF0BDC1F0F0ED51EF27EE51F02350
:1068E8000E0EEF25D96E000EF021DA6EDF50F16F33
:1068F800F151F36FF26BBAC1F4F0BBC1F5F0050EBC
:10690800D890F437F537E82EFBD7BCC1F6F0BDC1F7
:10691800F7F0F451F627F551F7230F0EF625D96E47
:10692800000EF721DA6EDF50F86FF96BF251F82795
:10693800F351F923F8C0B1F1F9C0B2F10101000E29
:10694800B2BFFF0EB36FB46F240E00018A6FFE0E44
:106958008B6FB1C18CF0B2C18DF0B3C18EF0B4C1F0
:106968008FF035EC5BF0B1C1CBF0B2C1CCF0B3C164
:10697800CDF0B4C1CEF012000101BA4BBB2BBBBFA6
:106988007BD7BB5105E10F0EBA5DD8B0DED674D700
:10699800DCD63E6E0001B151D8A4D6EC43F0000E0F
:1069A8003D6E0001B051D8B412D1040E3E18D8B4CF
:1069B80004D0140E3E18D8A40DD0000E0101966F15
:1069C800000E816F000E806F000E0001B16F070E80
:1069D800B06F12003F0E3E18D8A40BD0000EFE6F09
:1069E800000E0101966F000E0001B16F000EB06F2E
:1069F80012005F0E3E18D8A40BD0000E0101976F4D
:106A0800000E966F000E0001B16F000EB06F1200FD
:106A18003F0E3E6407D05F0E3E6004D0400E3E1825
:106A2800D8A4EBD7400E3E18D8A40BD0010E010114
:106A3800976F000E966F000E0001B16F000EB06FD9
:106A48001200200E3E18D8A412D0010EFE6F000EC0
:106A58000101966F820E00018A6FFF0E8B6F35EC75
:106A68005BF0000E0001B16F000EB06F1200650EF2
:106A78003E18D8A410D0FE51D8B40DD0000E010194
:106A8800816F000E806F010E966F000E0001B16FCE
:106A9800000EB06F12006E0E3E18D8A403D0020E7E
:106AA8000101966F700E3E18D8A40AD001019751C3
:106AB800D8B406D0000E816F000E806F030E966F5B
:106AC800700E3E18D8A412D00001FE51D8B40ED0D2
:106AD8008380000E0101816F000E806F040E966F97
:106AE800000E0001B16F000EB06F1200720E3E185A
:106AF800D8A46DD00001FE51D8B469D083801C0E93
:106B08000101816F2A0E806F050E966F000E00013D
:106B1800B16F000EB06F12003E50D5EC15F045D0A5
:106B280083803E5007EC54F03D6E000E0101966FD5
:106B380069D08380340E0C6E0B0E0D6E000E0F6E36
:106B4800000E0E6E010E116E000E106ED1EC47F0A5
:106B580053500209536E2BEE34F04DC0DFFF810E07
:106B680000018A6FFD0E8B6F000E8D6F010E8C6F0A
:106B780035EC5BF0340E236E0B0E246E000E266E81
:106B8800010E256E660E276EFF0E286E77EC39F023
:106B9800000E246E010E236E8EEC3AF05350FD0B5E
:106BA800536E080EC1D78390000E3D6E2BD0080E91
:106BB8003E18D8A427D08390000E3D6E000E4D6E6F
:106BC800000E966F000E816F000E806F1BD00101C2
:106BD80096513B6E3C6A3C50000AD8A413D03B50F7
:106BE800000AD8B40FD0010AD8B496D7030AD8B48B
:106BF80097D7010AD8B49DD7070AD8B4D4D7010AC1
:106C0800D8B4D5D73DC0B0F00001B16B1200000177
:106C180020EE04F06051D9266151DA22000EDF6EB1
:106C280020EE2AF06051D9266151DA22FF0EDE6E7D
:106C3800FF0EDE6EFF0EDE6EFF0EDD6E60C03AF0F8
:106C480061C03BF062C03CF063C03DF064C03EF000
:106C580065C03FF084EC4FF00009D8B402D0030EB1
:106C68001200000122EE2DF06051D9266151DA227E
:106C7800DF50666F6651686F676B22EE2CF06051CB
:106C8800D9266151DA22DF50696F69516713000E06
:106C98006813550E671904E1AA0E6819D8B402D012
:106CA800020E120020EE65F06051D9266151DA22F9
:106CB800DF50666F6651686F676B20EE66F0605153
:106CC800D9266151DA22DF50696F69C06AF06B6BAF
:106CD8006C6B6D6B6BC06DF06AC06CF06B6B6A6B44
:106CE80020EE67F06051D9266151DA22DF506E6FCD
:106CF8006EC06FF0706B716B726B6FC072F0716BFE
:106D0800706B6F6B6A516F11736F6B517011746F89
:106D18006C517111756F6D517211766F67517311E6
:106D2800776F68517411786F000E7511796F000EC6
:106D380076117A6F20EE64F06051D9266151DA221B
:106D4800DF507B6F7B5177117C6F78517D6F795164
:106D58007E6F7A517F6FFF0E7C15806FFF0E7D1559
:106D6800816FFF0E7E15826F000E7F15836F460EB2
:106D780080190AE1410E811907E1540E8219831125
:106D8800D8A402D0000E120020EE81F06051D9265E
:106D98006151DA22DF50666F6651686F676B20EECB
:106DA80082F06051D9266151DA22DF50696F69C0DB
:106DB8006AF06B6B6C6B6D6B6BC06DF06AC06CF0DE
:106DC8006B6B6A6B20EE83F06051D9266151DA2231
:106DD800DF506E6F6EC06FF0706B716B726B6FC04F
:106DE80072F0716B706B6F6B6A516F11736F6B51CF
:106DF8007011746F6C517111756F6D517211766FDE
:106E080067517311776F68517411786F000E75119F
:106E1800796F000E76117A6F20EE80F06051D926D6
:106E28006151DA22DF507B6F7B5177117C6F78518B
:106E38007D6F79517E6F7A517F6FFF0E7C15806F61
:106E4800FF0E7D15816FFF0E7E15826F000E7F1578
:106E5800836F460E801908E1410E811905E1540E31
:106E680082198311D8B48ED7010E1200010179AFAF
:106E78007A9379BF05D0795109E17805D8B006D061
:106E8800000E0001656F010E646F04D078C164F0D4
:106E980079C165F076C166F077C167F001017AA91A
:106EA80005D00001FE0E6627FF0E67232AC068F092
:106EB8002BC069F02CC06AF02DC06BF02EC06CF0AE
:106EC8002FC06DF030C06EF031C06FF0000E0001C1
:106ED800716F1F0E706F000E0201B36F95D0000125
:106EE8007007D8A071070F0E6815726F736B73BFA8
:106EF80008D0735104E10A0E725DD8A002D0570E73
:106F080001D0300E7225726F000E7321736FBF0EA1
:106F1800336EFF0E346E3250356E366A3350352676
:106F280034503622365006E11A0E355CD8B002D0FD
:106F3800010E01D0000E606F616B60516111D8B411
:106F480027D09F0E336EFF0E346E200E7211356EF1
:106F5800000E7311366E33503526345036223650B3
:106F680006E11A0E355CD8B002D0010E01D0000E31
:106F7800626F636B62516311D8B40AD072C012F0A9
:106F880073C013F0ACEC57F012C072F013C073F07A
:106F9800940E00017025D96E020E7121DA6E72C04E
:106FA800DFFF6407D8A065076607D8A0670768C031
:106FB80033F069C034F06AC035F06BC036F06CC08D
:106FC80037F06DC038F06EC039F06FC03AF0050E7A
:106FD80009D0D8903A3239323832373236323532EF
:106FE80034323332E82EF5D733C068F034C069F054
:106FF80035C06AF036C06BF037C06CF038C06DF041
:1070080039C06EF03AC06FF0000171BF21D07151E4
:1070180004E1020E705DD8A01BD0685169116A1195
:107028006B116C116D116E116F11D8A458D765BF13
:1070380005D0655102E16405D8B051D767BF08D0C3
:10704800675103E16605D8A003D001017AB347D799
:1070580001017AA917D000017007D8A07107940E12
:107068007025D96E020E7121DA6E32C0DFFF70070B
:10707800D8A07107940E7025D96E020E7121DA6EB0
:10708800300EDF6E28C01DF029C01EF0940E0001DE
:1070980070251F6E020E7121206E66C021F067C038
:1070A80022F01BEC51F01DC028F01EC029F0120080
:1070B8008380000E4D6E11EC43F0CBC0B4F1CCC010
:1070C800B5F10101B451B511D8B405D0B4C1EDF092
:1070D800B5C1EEF01200000EB66F000EB76F000ECD
:1070E800B86F000EB96F000EB36F010EB26F000ECD
:1070F800BC6FEAD0000EBB6F000EBA6F1DD016EC45
:107108005BF00C500D10D8B413D0BC0E0C6E010EF1
:107118000D6E44EC52F00101B16F000EA925D96E35
:10712800DA6A040EDA22B1C1DFFFA92BBA4BBB2BF6
:107138000101BCAB8EAC05D0BBBFE1D7BB05D8A065
:10714800DED7BAC1EFF0BBC1F0F0000E0001F0BF0E
:10715800FF0EF16FF26F0101B6510001EF25010139
:10716800B66FB7510001F0210101B76FB8510001A6
:10717800F1210101B86FB9510001F2210101B96F84
:107188000001FF51140D0F0EF324D96E010EF420E7
:10719800DA6EDE500101B65DDE50B759DE50B859DF
:1071A800DE50B959D8A004D0000EB36F000EB26FEC
:1071B800BCAB04D0000EB36F000EB26F8EBC04D00F
:1071C800000EB36F000EB26FBBBF03D0BB05D8B0C3
:1071D8001DD0000EA9250C6E0D6A040E0D22FF0E9F
:1071E800A925D96EDA6A030EDA22DF500001EF6FA3
:1071F800EF510E6E0F6A0101A9510008106E000EC2
:10720800D8A0E82A0108116ED1EC47F00001FF511F
:10721800140D070EF324D96E010EF420DA6E6CC13A
:10722800F4F06DC1F5F06EC1F6F0F36B000EF325C6
:10723800F76F010EF421F86F000EF521F96F000EBB
:10724800F621FA6FDE50F7191CE1DE50F81919E142
:10725800DE50F91916E1DE50FA19D8A412D001C48B
:10726800C0F103C4BFF105C4BEF107C4BDF1BDC17F
:107278000FF0BEC110F0BFC111F0C0C112F0AEECEA
:1072880056F0CBEC53F00001E2510101B06FB05160
:10729800D8B41AD0010E4D6E0001FF51140D130E13
:1072A800F324D96E010EF420DA6EFF51140D130E7B
:1072B800F324E16E010EF420E26EE7500409DF6E5C
:1072C8004DC0EDF0EE6B1200B251B311D8A412D735
:1072D8008FA402D0010E4D6E8390000E0001EE6F58
:1072E800000EED6F1200D20E00018A6FFE0E8B6F3A
:1072F80027C08CF028C08DF023C08EF024C08FF0FA
:1073080025C090F026C091F035EC5BF0000E306E91
:10731800000E2F6ED8D0B40E00018A6FFB0E8B6F53
:1073280035EC5BF0000E326E000E316E29D02FC0A6
:1073380029F030C02AF0293A2A3AF00E2A162950A4
:107348000F0B2A12F00E291623C02BF024C02CF0A4
:1073580029502B262A502C2231502B24D96E3250FA
:107368002C20DA6EDF502E6E9A0E00018A6FFF0E07
:107378008B6F2EC08CF08D6B35EC5BF0314A322A66
:1073880032BE06D032501FE1100E315CD8B01BD08F
:107398002FC029F030C02AF0293A2A3AF00E2A16CE
:1073A80029500F0B2A12F00E291631502926325077
:1073B8002A222950255C2650800A2B6E2A50800AE2
:1073C8002B58D8B0B4D7DF0E00018A6FFF0E8B6F31
:1073D80035EC5BF0000E326E000E316E4FD02FC0D0
:1073E80029F030C02AF0293A2A3AF00E2A162950F4
:1073F8000F0B2A12F00E291623C02BF024C02CF0F4
:1074080029502B262A502C2231502B24D96E325049
:107418002C20DA6E200EDF6428D0FB0E00018A6F64
:10742800FF0E8B6F2FC029F030C02AF0293A2A3A74
:10743800F00E2A1629500F0B2A12F00E291623C017
:107448002BF024C02CF029502B262A502C22315006
:107458002B24D96E32502C20DA6EDF502D6E2D5031
:107468008C6F8D6B35EC5BF007D00C0E00018A6FCA
:10747800FF0E8B6F35EC5BF0314A322A32BE06D0F4
:1074880032501FE1100E315CD8B01BD02FC029F04C
:1074980030C02AF0293A2A3AF00E2A1629500F0B42
:1074A8002A12F00E29163150292632502A22295044
:1074B800255C2650800A2B6E2A50800A2B58D8B09B
:1074C8008ED72F4A302A30BE06D030501BE1500EDE
:1074D8002F5CD8B017D02FC029F030C02AF0293A35
:1074E8002A3AF00E2A1629500F0B2A12F00E2916E6
:1074F8002550295C2A50800A2B6E2650800A2B586A
:10750800D8A009D7B40E00018A6FFB0E8B6F35EC3B
:107518005BF01200000E0101A76F000E4A6E000E0C
:10752800496E898689808982898489888B68849054
:10753800849284948498838E83B40ED052A607D004
:10754800B70E00018A6FFB0E8B6F35EC5BF0000EF7
:10755800246E000E236E12000F011391350EE82ED3
:10756800FED700F0D0D08EB808D08B680F011381F9
:1075780049C023F04AC024F012008EB80BD08D0EFB
:1075880000018A6FFE0E8B6F35EC5BF0630E010114
:10759800A76FC0D0100E706F270E716F000E726F3C
:1075A800000E736F90D08EB28EA410D07007000EAC
:1075B800715B725B735B702906E1712904E17229C2
:1075C80002E17329D8A49FD0620E73D0010E71D046
:1075D8008EA899D0020E6DD0FF0E256EFF0E266E76
:1075E80023C027F024C028F025502726265028221B
:1075F8004950271806E14A502818D8B453A201D098
:10760800899A340E4924D96E0B0E4A20DA6EDF505F
:10761800FF0A866E494A4A2A000E8B6E030E21D055
:10762800100E706F270E716F000E726F000E736F61
:107638006AD08EB20ED07007000E715B725B735BFE
:10764800702909E1712907E1722905E17329D8A494
:1076580002D0040EA76F8EA256D0040E2AD08990AD
:10766800050EA76FDDD789848EB40ED07007000E83
:10767800715B725B735B702909E1712907E17229FB
:1076880005E17329D8A402D0060EA76F8EA43BD0BB
:10769800060E0FD0898A89808B682350495C4A502E
:1076A800800A256E2450800A2558D8A08FD7630EEB
:1076B8000101A76F28D0A00E00018A6FFF0E8B6F03
:1076C80035EC5BF0F4D7A751256E266A2650000AE0
:1076D800D8A419D02550000AD8B465D7010AD8B45F
:1076E80077D7030AD8B478D7010AD8B4A2D7070A3B
:1076F800D8B4B5D7010AD8B4B6D7030AD8B4CAD70C
:10770800640AD8B4D8D7630E0101A719D8B402D037
:107718008EBC29D78980898289848988898A8B68DF
:10772800839E0F01138149C023F04AC024F0120040
:1077380047C00DF048C00EF0B4EC51F000016C6F7A
:107748006C51D8A4FDD020EE04F04750D9264850FB
:10775800DA22DFAAF5D047C0D9FF48C0DAFFDECF6A
:107768003AF0DDCF3BF020EE1AF04750D9264850CA
:10777800DA22DECF3CF0DECF3DF0DECF3EF0DECFCA
:107788003FF084EC4FF000016C6F6C51D8A4D8D056
:1077980020EE1EF04750D9264850DA22DECF71F08D
:1077A800DDCF72F020EE0BF07151D9267251DA223A
:1077B800000EDB8A20EE0AF04750D9264850DA221C
:1077C80010EE1CF07151E1267251E222DFCFE7FF83
:1077D80020EE1DF07151D9267251DA2210EE0AF00E
:1077E8004750E1264850E222E6CF68F0E5CF69F03D
:1077F80069C068F0696B6851DF6E20EE1EF0715148
:10780800D9267251DA2210EE0AF04750E126485084
:10781800E222E6CF68F0E6CF69F0E6CF6AF0E6CF7D
:107828006BF0110E05D0D8906B336A336933683327
:10783800E82EF9D76851DF6E20EE1FF07151D92676
:107848007251DA2210EE0AF04750E1264850E2223F
:10785800E6CF68F0E6CF69F0E6CF6AF0E6CF6BF0E6
:10786800190E05D0D8906B336A3369336833E82E24
:10787800F9D76851DF6E71C00CF072C00DF020EEC0
:107888000EF04750D9264850DA22DECF0EF0DECF70
:107898000FF0DECF10F0DECF11F05CEC58F00001F5
:1078A80020EE16F07151D9267251DA22000EDF6EE1
:1078B80020EE17F07151D9267251DA22000EDF6ED0
:1078C80020EE18F07151D9267251DA22210EDF6E9E
:1078D80020EE19F07151D9267251DA22460EDF6E68
:1078E80020EE12F07151D9267251DA22000EDF6EA5
:1078F80020EE13F07151D9267251DA22000EDF6E94
:1079080020EE04F04750D9264850DA22DF0EDF1661
:1079180047C0D9FF48C0DAFF10EE04F0DE50E12678
:10792800DD50E222010EE76E47C0D9FF48C0DAFFFA
:10793800DECF44F0DDCF45F0A2EC2AF000016C6FF9
:107948006C5112000001FF51070D520EF324D96E3D
:10795800010EF420DA6EDF2AFF51070D520EF324D0
:10796800D96E010EF420DA6E0F0EDF6431D0FF51AC
:10797800070D520EF324D96E010EF420DA6E000EB4
:10798800DF6EFF51070D510EF324D96E010EF4205E
:10799800DA6EDF2AFF51070D510EF324D96E010E5E
:1079A800F420DA6E010EDF6413D0FF51070D510E7B
:1079B800F324D96E010EF420DA6E000EDF6EFF514B
:1079C800070D500EF324D96E010EF420DA6EDF2A6B
:1079D800FF51070D520EF324D96E010EF420DA6E12
:1079E800DF50CB6FCBC0CCF0CD6BCE6BCF6BCEC0A6
:1079F800CFF0CDC0CEF0CCC0CDF0CC6BFF51070D91
:107A0800510EF324D96E010EF420DA6EDF50D06FD8
:107A1800D0C0D1F0D26BD36BD46BD3C0D4F0D2C06A
:107A2800D3F0D1C0D2F0D16B040ED890D137D23771
:107A3800D337D437E82EF9D7FF51070D500EF3246A
:107A4800D96E010EF420DA6EDF50D56FD5C0D6F0AE
:107A5800D76BD86BD96B040ED890D637D737D837B1
:107A6800D937E82EF9D7D8C0D9F0D7C0D8F0D6C0C2
:107A7800D7F0D66BD890D635DA6FD735DB6FD835D7
:107A8800DC6FD935DD6FD151DA25DE6FD251DB21BC
:107A9800DF6FD351DC21E06FD451DD21E16FCC5190
:107AA800DE25E26FCD51DF21E36FCE51E021E46F97
:107AB800CF51E121E56FFF51070D530EF324D96E25
:107AC800010EF420DA6EE2C0DEFFE3C0DEFFE4C0A0
:107AD800DEFFE5C0DEFFFF51200D140EF324A46F76
:107AE800020EF420A56FFF51070D530EF324D96E33
:107AF800010EF420DA6EDECFA6F0DECFA7F0DECFDF
:107B0800A8F0DECFA9F002EC10F00001E66FE65114
:107B1800D8B419D0870E8A6FFC0E8B6FFF51070DF2
:107B2800530EF324D96E010EF420DA6EDECF8CF0FA
:107B3800DECF8DF0DECF8EF0DECF8FF0E6C090F096
:107B4800916B35EC5BF0000E0101956F12005350FC
:107B58000209536E340E0C6E0B0E0D6E000E0F6E76
:107B6800000E0E6E010E116E000E106ED1EC47F075
:107B78002BEE34F0FFC0DFFFFF0EE8CF35FB00012E
:107B8800FF51140D130EF324D96E010EF420DA6E92
:107B98000101DFA403D0010EE8CF38FB0001FF513B
:107BA800140D130EF324D96E010EF420DA6E0101C0
:107BB800DFA003D0020EE8CF3AFB0001FF51140DFD
:107BC800130EF324D96E010EF420DA6E0101DFA240
:107BD80003D0020EE8CF3AFB8FA403D0080EE8CFFB
:107BE8003AFB000E2C6E000E2B6EFC0E00018A6F05
:107BF800FB0E8B6FCECF8CF08D6BCDCF8EF08F6B55
:107C08002BC090F02CC091F0360E2B24D96E0B0EA1
:107C18002C20DA6EDF50296E2950926F936B35EC69
:107C28005BF0000E2B24D96E020E2C20DA6EDF508A
:107C3800FF0A2A6E360E2B24D96E0B0E2C20DA6E14
:107C4800360E2B24E16E0B0E2C20E26EE7502A1420
:107C5800DF6E5F0E00018A6FFF0E8B6F360E2B24CE
:107C6800D96E0B0E2C20DA6EDF50296E29508C6FDE
:107C78008D6B35EC5BF02B4A2C2A2CBEB6D72C50DA
:107C880004E1070E2B5CD8A0B0D70001FF51140DFA
:107C9800130EF324D96E010EF420DA6EDF504D6E08
:107CA800FF51140D010EF324D96E010EF420DA6E83
:107CB800DF50296E29C03FFBFF51140D020EF3243B
:107CC800D96E010EF420DA6EDF50296E29C040FB10
:107CD800FF51140D030EF324D96E010EF420DA6E51
:107CE800DF50296E29C041FBFF51140D040EF32407
:107CF800D96E010EF420DA6EDF50296E29C042FBDE
:107D0800FF51140D050EF324D96E010EF420DA6E1E
:107D1800DF50296E29C043FBFF51140D060EF324D2
:107D2800D96E010EF420DA6EDF50296E29C044FBAB
:107D3800000E246E140E236E8EEC3AF05350FD0B99
:107D4800536E839012008EA604D04E0E246EFE0E43
:107D580003D0B50E246EFF0E256E8EAA04D04E0EEB
:107D6800266EFE0E03D0B00E266EFF0E276E8EA86E
:107D780004D04E0E286EFE0E03D0BA0E286EFF0EEB
:107D8800296E8EAE04D04E0E2A6EFE0E03D0BF0EA4
:107D98002A6EFF0E2B6E8EAC04D04E0E2C6EFE0E8D
:107DA80003D0AB0E2C6EFF0E2D6E8EA404D04E0E9B
:107DB8002E6EFE0E03D0C90E2E6EFF0E2F6E8EA2F3
:107DC80004D04E0E306EFE0E03D0CE0E306EFF0E77
:107DD800316E8EA004D04E0E326EFE0E03D0C40E4D
:107DE800326EFF0E336E90AE04D04E0E346EFE0E21
:107DF80003D0F80E346EFF0E356E90AC04D04E0EE4
:107E0800366EFE0E03D0F50E366EFF0E376E90AA54
:107E180004D04E0E386EFE0E03D0F20E386EFF0EF2
:107E2800396E90A804D04E0E3A6EFE0E03D0EF0EB7
:107E38003A6EFF0E3B6E90A604D04E0E3C6EFE0EC0
:107E480003D0EC0E3C6EFF0E3D6E90A404D04E0E97
:107E58003E6EFE0E03D0E90E3E6EFF0E3F6E90A200
:107E680004D04E0E406EFE0E03D0E60E406EFF0E9E
:107E7800416E90A004D04E0E426EFE0E03D0E30E6B
:107E8800426EFF0E436E3A0E00018A6FFB0E8B6F37
:107E98009050FF0A236E23508C6F8D6B8ECF8EF01F
:107EA8008F6B42C090F043C091F040C092F041C047
:107EB80093F03EC094F03FC095F03CC096F03DC0B2
:107EC80097F03AC098F03BC099F038C09AF039C0A2
:107ED8009BF036C09CF037C09DF034C09EF035C092
:107EE8009FF032C0A0F033C0A1F030C0A2F031C082
:107EF800A3F02EC0A4F02FC0A5F02CC0A6F02DC072
:107F0800A7F02AC0A8F02BC0A9F028C0AAF029C061
:107F1800ABF026C0ACF027C0ADF024C0AEF025C051
:107F2800AFF035EC5BF01200000E0001C86F010ED7
:107F3800C76F8380000EC16F000EC26F000EC36F43
:107F4800000EC46FD8D0FF51200D140EF3248C6F8F
:107F5800020EF4208D6F340E8E6F0B0E8F6F010E94
:107F6800916F000E906FCB0E926F000E936F09EC1D
:107F780013F00001FF51070D530EF324D96E010EC3
:107F8800F420DA6E6CC1B9F06DC1BAF06EC1BBF005
:107F9800B86B000EB825BC6F010EB921BD6F000E7D
:107FA800BA21BE6F000EBB21BF6FDE50BC1930E195
:107FB800DE50BD192DE1DE50BE192AE1DE50BF1991
:107FC800D8A426D010EC53F010C0CDF011C0CEF0DC
:107FD80012C0CFF013C0D0F0000EE8CF34FB2BEE68
:107FE80035F0D0C0DFFF000EE8CF36FB2BEE37F0C0
:107FF800CFC0DFFF000EE8CF38FB2BEE39F0CEC044
:10800800DFFF000EE8CF3AFB2BEE3BF0CDC0DFFFE1
:108018005350FD0B536ECBC023F0CCC024F08EEC34
:108028003AF023C0C9F024C0CAF00001C951C125E3
:10803800C16FCA51C221C26F000EC321C36F000EA7
:10804800C421C46F8EAC5CD0CB51C91904E1CC51AA
:10805800CA19D8B40BD0DF0E8A6FFE0E8B6FC9C059
:108068008CF0CAC08DF035EC5BF04AD0BCEC5AF00D
:1080780016EC5BF00C500D10D8B404D0010E0101C1
:10808800956F3ED0000E0001C66F050EC56F1FD05C
:10809800D00E0001B46FC90EE82EFED7B42FFCD75E
:1080A80000D016EC5BF00C500D10D8B410D0000EB8
:1080B8000001C86F000EC76FB40E8A6FFD0E8B6F7C
:1080C800C5C08CF0C6C08DF035EC5BF009D000015E
:1080D800C507D8A0C607C529DBE1C629D8A4D8D7C3
:1080E80016EC5BF00C500D10D8B405D0000E000152
:1080F800C86F000EC76F0001C751C811D8A423D795
:10810800000E0101956F839012001C6E1C50D8B4AC
:1081180002D0010E120051A202D051501200000EDE
:1081280064EC5AF00A0E276E03D095EC5BF0270634
:108138002750D8A4FAD7000E246E000E156E000E34
:10814800166E000E176E000E186E000E7DEC58F0BD
:10815800E806D8A4C1D0AA0E156E010E166E000E40
:10816800176E000E186E080E7DEC58F0E806D8A4BD
:1081780066D0000E276E1D0E2724D96EDA6A000E0F
:10818800DA2295EC5BF0DF6E272A030E2764F3D71B
:108198001F04D8A4A1D0AA0E2018D8A49DD0030EDD
:1081A800266EE80E256E19D0000E156E000E166E9E
:1081B800000E176E400E186EA90E7DEC58F00009DF
:1081C800D8B40FD0150E1B6EC60EE82EFED71B2E88
:1081D800FCD700D02506D8A0260625502610D8A4FE
:1081E800E3D725502610D8B477D0000E156E000EB0
:1081F800166E000E176E000E186E3A0E7DEC58F0D3
:108208000009D8A469D0000E276E1D0E2724D96E48
:10821800DA6A000EDA2295EC5BF0DF6E272A030E8D
:108228002764F3D71DBC04D0000E226E040E03D0C1
:10823800000E226E0C0E216E21C024F04DD0000ECF
:10824800156E000E166E000E176E000E186EA90E33
:108258007DEC58F01B6E020E1B6004D0020E246EDB
:10826800A90E03D0010E246E010E236E030E266E96
:10827800E80E256E19D0000E156E000E166E000E53
:10828800176E000E186E23507DEC58F00009D8B414
:108298000FD0150E1B6EC60EE82EFED71B2EFCD770
:1082A80000D02506D8A0260625502610D8A4E3D746
:1082B80025502610D8B40ED0000E156E020E166E7C
:1082C800000E176E000E186E100E7DEC58F00009A7
:1082D800D8B402D0000E246E24C04EF0A1EC5BF09E
:1082E8002450D8B41AD7519018D776C0D9FF77C080
:1082F800DAFFDECFF6FFDDCFF7FF0800F550250ADD
:10830800D8A4AAD076C0D9FF77C0DAFFDE2A000E3B
:10831800DD22000E0101776F000E766F76C17AF1CB
:1083280077C17BF17869796976C0D9FF77C0DAFFC0
:10833800DECFF6FFDDCFF7FF0800F550780AD8B496
:108348000DD076C0D9FF77C0DAFFDECFF6FFDDCFDC
:10835800F7FF0800F550580AD8A44DD076C0D9FFC9
:1083680077C0DAFFDECFF6FFDDCFF7FF0800F5CFE5
:1083780047F076C0D9FF77C0DAFFDE2A000EDD228B
:1083880078C0D9FF79C0DAFFDFCF3BF0020EDE26D6
:10839800DFCF3CF0000EDD223BC0D9FF3CC0DAFF46
:1083A800DECF3DF0DDCF3EF03DC03FF03EC040F0B7
:1083B800416A426A436A446A456A466A74C028F058
:1083C80075C029F03FC02AF040C02BF041C02CF006
:1083D80042C02DF043C02EF044C02FF045C030F00D
:1083E80046C031F047C032F03AEC37F028C074F09C
:1083F80029C075F0120076C0D9FF77C0DAFFDECF4A
:10840800F6FFDDCFF7FF0800F550250AD8A417D0EE
:1084180076C0D9FF77C0DAFFDE2A000EDD22000E13
:108428000E6E250E0D6E74C00FF075C010F0CBECFB
:1084380050F0000E0001756F010E746F120076C0C7
:10844800D9FF77C0DAFFDE2A000EDD22000E000118
:10845800756F000E746F120076C0D9FF77C0DAFF0F
:10846800DECFF6FFDDCFF7FF0800F5500D6E0E6A80
:1084780074C00FF075C010F0CBEC50F076C0D9FF87
:1084880077C0DAFFDE2A000EDD22D3D7BFC0F6FFA1
:10849800C0C0F7FF000EF86E0E0EF76403D0080098
:1084A800F55005D0F6CFE9FFF7CFEAFFEF502F0AD6
:1084B800D8B414D0BFC0F6FFC0C0F7FF000EF86EE6
:1084C8000E0EF76403D00800F55005D0F6CFE9FF8B
:1084D800F7CFEAFFEF505C0AD8A403D00001BF4BE6
:1084E800C02B000120EE06F0BD51D926BE51DA227C
:1084F800DE6ADE6ADE6ADD6ABFC0F6FFC0C0F7FF6B
:10850800000EF86E0E0EF76403D00800F55005D083
:10851800F6CFE9FFF7CFEAFFEF500001C16F200E59
:10852800C16117D0BDC045F0BEC046F0000E486E10
:10853800000E476ECAEC30F00001C56F20EE12F055
:10854800BD51D926BE51DA22000EDE6E000EDD6E58
:1085580062D0BDC014F0BEC015F0BF0E166E000E7E
:10856800176E5CEC2FF00001C56FC551D8A453D02D
:10857800BDC0B7F0BEC0B8F025EC4DF00001C56F26
:1085880020EE14F0BD51D926BE51DA2210EE0BF0C0
:10859800DE50E126DD50E222E750C46FC551D8B461
:1085A80008D0040EC519D8B4C4B535D0050EC56FAA
:1085B80032D0C4B530D020EE12F0BD51D926BE510C
:1085C800DA22DECFC2F0DDCFC3F020EE0BF0C251CD
:1085D800D926C351DA22DFA8E9D7BDC0D9FFBEC06A
:1085E800DAFFDECF0CF0DDCF0DF0C2C00EF0C3C055
:1085F8000FF06BEC4EF0000120EE06F0BD51D926CD
:10860800BE51DA220CC0DEFF0DC0DEFF0EC0DEFF59
:108618000FC0DEFF9ED7C55112000001FF51140D97
:10862800070EF324D96E010EF420DA6EDECFDDF0EA
:10863800DECFDEF0DECFDFF0DECFE0F0FF51140D4D
:10864800070EF324D96E010EF420DA6EFF51140DD3
:108658000B0EF324E16E010EF420E26EDE50E65CB0
:10866800DE50E658DE50E658DE50E658D8B015D051
:10867800010E4D6EFF51140D130EF324D96E010E29
:10868800F420DA6EFF51140D130EF324E16E010E7F
:10869800F420E26EE7500409DF6EFF51140D0F0E4F
:1086A800F324D96E010EF420DA6EDECFCDF0DECFE2
:1086B800CEF0DECFCFF0DECFD0F0FF51140D070E95
:1086C800F324D96E010EF420DA6EDECFD1F0DECFBE
:1086D800D2F0DECFD3F0DECFD4F0CD51D125D56F97
:1086E800CE51D221D66FCF51D321D76FD051D421BB
:1086F800D86FFF51140D0B0EF324D96E010EF42020
:10870800DA6ED551DE5CD651DE58D751DE58D851D5
:10871800DE58D8B015D0010E4D6EFF51140D130E52
:10872800F324D96E010EF420DA6EFF51140D130EE6
:10873800F324E16E010EF420E26EE7500409DF6EC7
:10874800000E4D6EFF51200D140EF324A46F020E7F
:10875800F420A56FDDC0A6F0DEC0A7F0DFC0A8F04A
:10876800E0C0A9F002EC10F00001E16FE151D8B4CB
:1087780015D0010E4D6EFF51140D130EF324D96E52
:10878800010EF420DA6EFF51140D130EF324E16E7E
:10879800010EF420E26EE7500409DF6E4DC0CBF005
:1087A800CC6B1200000E0001FF6F000EFF6F030E6E
:1087B800FF6501D0A3D0FF51140D130EF324D96E19
:1087C800010EF420DA6E000EDF6EFF51140D000E5C
:1087D800F324D96E010EF420DA6E000EDF6EFF511D
:1087E800140D070EF324D96E010EF420DA6EDE6A3A
:1087F800DE6ADE6ADD6AF3C223F0246A256A266A25
:1088080025C026F024C025F023C024F0236AF2C234
:1088180027F0286A296A2A6A28C02AF027C029F07E
:10882800286A276AF1C22BF02C6A2D6A2E6A2BC09F
:108838002EF02D6A2C6A2B6A0201F0512B242F6E20
:10884800000E2C20306E000E2D20316E000E2E20D2
:10885800326E27502F24336E28503020346E295022
:108868003120356E2A503220366E23503324376E2D
:1088780024503420386E25503520396E2650362045
:108888003A6E0001FF51140D0B0EF324D96E010E40
:10889800F420DA6E37C0DEFF38C0DEFF39C0DEFFF5
:1088A8003AC0DEFFDC0E8A6FFB0E8B6FFFC08CF0C8
:1088B8008D6BFF51140D0B0EF324D96E010EF420AD
:1088C800DA6EDECF8EF0DECF8FF0DECF90F0DECF27
:1088D80091F0FF51140D0B0EF324D96E010EF42004
:1088E800DA6EDECF92F0DECF93F0DECF94F0DECFFB
:1088F80095F035EC5BF00001FF2B59D7000E010114
:10890800976F000E0001FE6F000E0101AB6F000EA5
:10891800966F000E816F000E806F020E4D6E839071
:1089280012000001FF51070D520EF324D96E010EFB
:10893800F420DA6EDF50CB6FCBC0CCF0CD6BCE6BB2
:10894800CF6BCEC0CFF0CDC0CEF0CCC0CDF0CC6BCD
:10895800FF51070D510EF324D96E010EF420DA6E83
:10896800DF50D06FD0C0D1F0D26BD36BD46BD3C0F3
:10897800D4F0D2C0D3F0D1C0D2F0D16B040ED890CD
:10898800D137D237D337D437E82EF9D7FF51070D6F
:10899800500EF324D96E010EF420DA6EDF50D56F35
:1089A800D5C0D6F0D76BD86BD96B040ED890D63714
:1089B800D737D837D937E82EF9D7D8C0D9F0D7C0A4
:1089C800D8F0D6C0D7F0D66BD890D635DA6FD73571
:1089D800DB6FD835DC6FD935DD6FD151DA25DE6F25
:1089E800D251DB21DF6FD351DC21E06FD451DD217F
:1089F800E16FCC51DE25E36FCD51DF21E46FCE511D
:108A0800E021E56FCF51E121E66FFF51200D140EF3
:108A1800F324A46F020EF420A56FE3C0A6F0E4C00F
:108A2800A7F0E5C0A8F0E6C0A9F002EC10F000013C
:108A3800E26FE251D8B411D0870E8A6FFC0E8B6FAB
:108A4800E3C08CF0E4C08DF0E5C08EF0E6C08FF096
:108A5800E2C090F0916B35EC5BF00001FF51070D1F
:108A6800530EF324D96E010EF420DA6EE3C0DEFF54
:108A7800E4C0DEFFE5C0DEFFE6C0DEFF000E010158
:108A8800956F83901200000E336E20EE04F025508F
:108A9800D9262650DA22DF50D8B49FD020EE2AF00B
:108AA8002550D9262650DA22DECF36F0DECF37F031
:108AB800DECF38F0DECF39F02E0E25241B6E000EE7
:108AC80026201C6E36C01DF037C01EF038C01FF0BF
:108AD80039C020F0000E226E010E216E20EE01F04A
:108AE8002550D9262650DA22DF5024EC4AF0000916
:108AF800D8B403D0010E336E70D020EE04F02550A8
:108B0800D9262650DA22000EDF6E20EE16F0255008
:108B1800D9262650DA2210EE1EF02550E1262650DE
:108B2800E222E6CF2BF0E6CF2CF0E6CF2DF0E6CF11
:108B38002EF02B50365C2F6E2C503758306E2D503F
:108B48003858316E2E503958326EDE502F5CDE5058
:108B58003058DE503158DE503258D8B03ED020EE72
:108B680003F02550D9262650DA22DF50276E2750E9
:108B7800346E356A355004E1020E345CD8A02DD02D
:108B880020EE16F02550D9262650DA22DE50362659
:108B9800DE503722DE503822DD5039222E0E2524B1
:108BA8001B6E000E26201C6E36C01DF037C01EF04E
:108BB80038C01FF039C020F0000E226E010E216E61
:108BC80020EE01F02550D9262650DA22DF5024EC79
:108BD8004AF03406D8A03506CDD73350120000012C
:108BE80096519511941104E1020E935DD8A010D00E
:108BF80020EE12F09151D9269251DA22DE50935D7F
:108C0800DE509459DE509559DE509659D8A002D0BE
:108C1800020E30D0000E976F74D091C060F092C0F1
:108C280061F093C062F094C063F095C064F096C0A0
:108C380065F03EEC24F060C098F061C099F062C025
:108C48009AF063C09BF00001985199119A119B11F9
:108C5800D8B467D0980599119A119B11D8B4D8D770
:108C680098290AE1992908E19A2906E19B29D8A4BB
:108C780003D0010E976F55D091C060F092C061F09B
:108C880093C062F094C063F095C064F096C065F03C
:108C9800000E666F000E676F000E686F000E696F3A
:108CA8007CEC18F00001976F9751D8A43AD020EEC9
:108CB8000EF09151D9269251DA22DE2807E1DE28FA
:108CC80005E1DE2803E1DE28D8B413D020EE0EF04B
:108CD8009151D9269251DA22DE2A000EDE22DE22B6
:108CE800DE2220EE05F09151D9269251DA22000EAB
:108CF800DB8098C093F099C094F09AC095F09BC01F
:108D080096F020EE12F09151D9269251DA22DE50D7
:108D1800935DDE509459DE509559DE509659D8A08F
:108D28007CD797511200146815680CC0D9FF0DC084
:108D3800DAFFDE50DE10D8B489D00CC0D9FF0DC0E0
:108D4800DAFFDECF18F0DDCF19F002D0184A192A61
:108D580018C0F6FF19C0F7FF000EF86E0E0EF76484
:108D680003D00800F55005D0F6CFE9FFF7CFEAFFAA
:108D7800EF500E6E200E0E6414D018C0F6FF19C006
:108D8800F7FF000EF86E0E0EF76403D00800F550DA
:108D980005D0F6CFE9FFF7CFEAFFEF503A0AD8A49B
:108DA800D5D718C0F6FF19C0F7FF000EF86E0E0EE3
:108DB800F76403D00800F55005D0F6CFE9FFF7CFE8
:108DC800EAFFEF503A0AD8A446D00CC0D9FF0DC02C
:108DD800DAFFDECF12F0DDCF13F012C0F6FF13C0BA
:108DE800F7FF000EF86E0E0EF76403D00800F5507A
:108DF80005D0F6CFE9FFF7CFEAFFEF500E6ED00EA1
:108E08000E24166E176AFF0E1722124A132A1750DD
:108E18001DE10A0E165CD8B019D01850121816E1C8
:108E280019501318D8A412D016501710D8A40ED061
:108E380016C014F017C015F0184A192A0CC0D9FF2B
:108E48000DC0DAFF18C0DEFF19C0DDFF14C00CF03A
:108E580015C00DF01200000E156E000E146EF6D738
:108E6800000E216E000E206E000E1A6E000E196E96
:108E780002D0134A142A010E1F6E13C0D9FF14C062
:108E8800DAFF200EDE18D8B417D0F70E156EFF0ED5
:108E9800166E13C0D9FF14C0DAFFDF50176E186AB8
:108EA8001550172616501822185004E1050E175CA5
:108EB800D8A002D0000E1F6E1FC01BF01C6A1B50EA
:108EC8001C10D8B408D0D5D7000E1A6E010E196E32
:108ED800134A142A2ED013C0D9FF14C0DAFFDF506A
:108EE800156E166A1650000AD8A423D015502B0AFE
:108EF800D8B4EED7060AD8B4E7D71BD020C00CF0F8
:108F080021C00DF0000E0F6E0A0E0E6EE2EC5AF044
:108F180013C0D9FF14C0DAFFDF50156E15500C5E70
:108F2800000E0D5A300E0C24206E000E0D20216EFE
:108F3800CFD7D00E156EFF0E166E13C0D9FF14C012
:108F4800DAFFDF50176E186A1550172616501822C8
:108F5800185006E10A0E175CD8B002D0010E01D0F5
:108F6800000E1D6E1E6A1D501E10D8A4C7D71950BA
:108F78001A10D8A40DD020C015F021C016F0151E67
:108F8800161E154A162A15C013F016C014F0120042
:108F980020C013F021C014F012000CC016F00DC050
:108FA80017F010501110D8B4120016C0D9FF17C00E
:108FB800DAFF0EC0DFFF10501624126E1150172072
:108FC800136EFF0E1224D96EFF0E1320DA6E0EC038
:108FD800DFFF115004E1030E105CD8A0120020EE50
:108FE80001F01650D9261750DA220EC0DFFF20EE06
:108FF80002F01650D9261750DA220EC0DFFF1050A3
:109008001624126E11501720136EFE0E1224D96EFC
:10901800FF0E1320DA6E0EC0DFFF10501624126EFA
:1090280011501720136EFD0E1224D96EFF0E132057
:10903800DA6E0EC0DFFF115004E1070E105CD8A0F5
:10904800120020EE03F01650D9261750DA220EC06F
:10905800DFFF10501624126E11501720136EFC0EED
:109068001224D96EFF0E1320DA6E0EC0DFFF1150E6
:1090780004E1090E105CD8A0120016C012F017C047
:1090880013F0121E131E124A132A030E1214146E22
:10909800156A14501626155017221450105E1550D4
:1090A800115AFC0E1016FF0E11160BD016C0D9FF60
:1090B80017C0DAFF0EC0DFFF1006D8A01106164A47
:1090C800172A10501110D8B41200F0D72F6C696607
:1090D80064617461302E62696E20002F6C69666469
:1090E800617461312E62696E20002F6C696664615B
:1090F8007461322E62696E20002F6C696664617437
:1091080061332E62696E20002F6C69666461746138
:10911800342E62696E20002F6C6966646174613553
:109128002E62696E20002F6C696664617461362E48
:1091380062696E20002F6C696664617461372E6203
:10914800696E20002F6C696664617461382E6269EB
:109158006E20002F6C696664617461392E62696ED5
:1091680020002F6C696664617461612E62696E20EB
:10917800002F6C696664617461622E62696E2000FA
:109188002F6C696664617461632E62696E20002FBA
:109198006C696664617461642E62696E20002F6C6C
:1091A800696664617461652E62696E20002F6C695E
:1091B8006664617461662E62696E200000000000BA
:1091C8000000000000000000000000000000000097
:1091D8000000000000000000000000000000000087
:1091E8000000000000000000000000000000000077
:1091F80000000000000000008380000E0001F66FF0
:10920800000EF56F000EF36FB8EC54F016C0F7F0CF
:1092180017C0F8F00001F8BF0BD0040EF85DD8A015
:1092280007D0000EF725F56FFC0EF821F66F04D075
:10923800F7C0F5F0F8C0F6F0FF51070D530EF32410
:10924800D96E010EF420DA6E6CC1ECF06DC1EDF050
:109258006EC1EEF0EB6B000EEB25EF6F010EEC210B
:10926800F06F000EED21F16F000EEE21F26FDE506F
:10927800EF191CE1DE50F01919E1DE50F11916E181
:10928800DE50F219D8A412D001C4FCF003C4FBF0DC
:1092980005C4FAF007C4F9F0F9C00FF0FAC010F0ED
:1092A800FBC011F0FCC012F0AEEC56F08FB419D030
:1092B8000001FF51200D140EF324A46F020EF420B8
:1092C800A56F000EA66F040EA76F010EA96F000E02
:1092D800A86FF50EAA6F000EAB6F70EC0CF00001D2
:1092E800F46F0001F451D8B409D0C40E8A6FFD0E92
:1092F8008B6FF4C08CF08D6B35EC5BF0A6EC3CF01A
:10930800000E0101956F83905F0E00018A6FFD0EBC
:109318008B6FCECF8CF08D6BCDCF8EF08F6B35EC05
:109328005BF01200E8C125F077D0A8EC5AF0256E62
:109338000101E8512518D8B481D0290E246E960E63
:10934800236E7F0EE82EFED7232EFCD7242EFAD7C5
:1093580000F074D0BDEC55F0266E2650D8B46ED00F
:1093680026B0502A26B2500650500F0B506E000EF1
:109378000C6EC00E86EC57F07BEC5AF0000E0C6EAB
:10938800C00E86EC57F050500F0D340EF324106EBB
:109398000D0EF420116E8DEC53F0190E246E5A0E3A
:1093A800236EB20EE82EFED7232EFCD7242EFAD732
:1093B80026A444D0000E0D6E000E0C6E50C00EF0A8
:1093C80078EC59F03A0E00018A6FFD0E8B6F50C091
:1093D8008CF08D6B35EC5BF050C025F0000E0C6EF8
:1093E800800E86EC57F07BEC5AF0000E0C6E800E67
:1093F80086EC57F050500F0D340EF324106E0D0EFE
:10940800F420116E8DEC53F0000E0C6EC00E86EC3D
:1094180057F07BEC5AF012D001019F51236E246A59
:109428002450000AD8A40AD02350010AD8B47DD702
:10943800030AD8B47AD7010AD8B48CD725501200B9
:10944800246E2450D8A404D021502210D8A402D0CD
:10945800040E120051A002D0030E120051A402D033
:10946800020E12004EB608D0090ED8901D361E36D0
:109478001F362036E82EF9D721042210D8A41DD093
:109488001DC015F01EC016F01FC017F020C018F040
:10949800180E7DEC58F00009D8A44FD01BC00EF070
:1094A8001CC00FF0FE0E106E20EC56F00009D8B468
:1094B80044D0000E226E000E3FD04EC023F0060EA0
:1094C8002316D8B409D021C015F022C016F0176AA7
:1094D800186A970E7DEC58F01DC015F01EC016F0E6
:1094E8001FC017F020C018F0190E7DEC58F00009C5
:1094F800D8A423D01BC00EF01CC00FF0FC0E106EB9
:1095080020EC56F00009D8B409D0020E1C2621061A
:10951800D8A0220621502210D8A4ECD7000E0E6E37
:10952800000E0F6EFD0E106E20EC56F00009D8A448
:1095380004D0000E226E010E216EA1EC5BF02150CA
:109548002210D8B402D0010E1200000E120083803F
:10955800000E0C6E040E0D6E000E0F6EF60E0E6EE3
:10956800010E116E000E106ED1EC47F09C0E00013A
:109578008A6FFE0E8B6F35EC5BF0000E0001EC6F0E
:10958800000EEB6F2E0E69EC5BF08FB419D0000162
:10959800FF51200D140EF324A46F020EF420A56FC2
:1095A800000EA66F040EA76F010EA96F000EA86F1C
:1095B800E80EAA6F000EAB6F70EC0CF00001EA6FBA
:1095C8000001EA51D8B40AD0580E8A6FFF0E8B6F8B
:1095D800EAC08CF08D6B35EC5BF0120016EC5BF09A
:1095E8000C500D10D8B428D0ED0E0C6E000E0D6E78
:1095F80044EC52F00001E76FED51100B0C6E000EB9
:109608000D6EE75105EC22F00CC0EEF00DC0EFF046
:10961800040E0001EE19EF11D8B495EC59F0020EC2
:109628000001EE19EF11D8B4DBEC56F00001EE059D
:10963800EF11D8B495EC44F00001EB4BEC2BEC5156
:1096480004E1C80EEB5DD8A09DD7190E8A6FFF0EF6
:109658008B6F35EC5BF083901200000E0001F56F04
:10966800838079D0B8EC54F016C0F3F017C0F4F04A
:109678000001F4BF07D0040EF45DD8A003D0010E9A
:10968800F56F03D0F8C0F6F0F76B8FB418D0FF5120
:10969800200D140EF324A46F020EF420A56F000E03
:1096A800A66F040EA76F010EA96F000EA86FF60E25
:1096B800AA6F000EAB6F70EC0CF00001F86FF85158
:1096C800D8B409D0C40E8A6FFD0E8B6FF8C08CF029
:1096D8008D6B35EC5BF00001FF51070D530EF32441
:1096E800D96E010EF420DA6E6CC1ECF06DC1EDF0AC
:1096F8006EC1EEF0EB6B000EEB25EF6F010EEC2167
:10970800F06F000EED21F16F000EEE21F26FDE50CA
:10971800EF191CE1DE50F01919E1DE50F11916E1DC
:10972800DE50F219D8A412D001C4FCF003C4FBF037
:1097380005C4FAF007C4F9F0F9C00FF0FAC010F048
:10974800FBC011F0FCC012F0AEEC56F0A6EC3CF0F9
:10975800000E0101956F0001F551D8B483D78390AD
:109768001200818E819CD40EF66E900EF76E000E5C
:10977800F86E0DEE34F011EE2CF00900F5CFEEFF87
:10978800E550E150FAE1E250F8E10C0EF66EB60E43
:10979800F76E000EF86E03EE80F010EE20F0090070
:1097A800F5CFEEFFE550E150FAE1EA0EF66EAF0EA6
:1097B800F76E000EF86E02EEB4F010EE46F00900F7
:1097C800F5CFEEFFE550E150FAE1620EF66EB70E06
:1097D800F76E000EF86E0900F5CFE9F10900F5CF34
:1097E800EAF1600EF66EB70EF76E000EF86E09001D
:1097F800F5CF51F00900F5CF52F005EE00F018EE64
:1098080034F0EE6AE550E150FCE1E250FAE104EE92
:1098180000F011EE00F0EE6AE550E150FCE1E25094
:10982800FAE103EE00F0800EEE6AE806FDE102EED2
:1098380000F0B40EEE6AE806FDE101EE00F0B00EAD
:10984800EE6AE806FDE10001FF6BFE6B00EE49F0F1
:10985800080EEE6AE806FDE154905492000EF86E88
:10986800000179EF08F0B7C045F0B8C046F0000E27
:10987800486E000E476ECAEC30F00001C06FC05150
:10988800D8A461D0000EBF6F000EBE6FB7C0D9FF5D
:10989800B8C0DAFFDECF3AF0DDCF3BF020EE0EF0B5
:1098A800B751D926B851DA22DECF3CF0DECF3DF0F1
:1098B800DECF3EF0DECF3FF084EC4FF00001C06F0A
:1098C800C051D8A440D020EE12F0B751D926B851D3
:1098D800DA22DECFBBF0DDCFBCF0BBC0D9FFBCC005
:1098E800DAFFE50EDE18D8B411D020EE12F0B75129
:1098F800D926B851DA22DECFBBF0DDCFBCF0BBC031
:10990800D9FFBCC0DAFFDF50D8A40AD0BE4BBF2BAA
:10991800B951BE1909E1BA51BF19D8B414D004D04D
:10992800000EBF6F000EBE6FB7C0A4F0B8C0A5F0A0
:10993800000EA76F010EA66F9FEC28F00001C06F04
:10994800C051D8B4A3D7040EC019D8A402D0070EAA
:10995800C06FC05112000F015969000E116F000E3F
:10996800196F000E216F8C948C928C90889A110E2E
:10997800116E3C0E106ECB0EE82EFED7102EFCD7C3
:10998800112EFAD700F0110E116E3C0E106ECB0E90
:10999800E82EFED7102EFCD7112EFAD700F0020EB3
:1099A800116EA00E106E920EE82EFED7102EFCD768
:1099B800112EFAD700D0000E0C6E300E86EC57F040
:1099C8002A0E106E8E0EE82EFED7102EFCD7000E33
:1099D8000C6E300E86EC57F0000E0C6E300E86ECD6
:1099E80057F0000E0C6E390E86EC57F0000E0C6E18
:1099F800140E86EC57F0000E0C6E560E86EC57F0DF
:109A0800000E0C6E6D0E86EC57F0000E0C6E700E8C
:109A180086EC57F0000E0C6E0C0E86EC57F0000E1C
:109A28000C6E060E86EC57F0000E0C6E010E86ECDE
:109A380057F0D00E106ECA0EE82EFED7102EFCD7A7
:109A48001200B7C045F0B8C046F0000E486E000ED0
:109A5800476ECAEC30F00001BC6FBC51D8B403D0DB
:109A68000001BC511200B7C0D9FFB8C0DAFFDECF81
:109A78003AF0DDCF3BF020EE0EF0B751D926B851C1
:109A8800DA22DECF3CF0DECF3DF0DECF3EF0DECF97
:109A98003FF084EC4FF00001BC6FBC51D8A4E0D774
:109AA80020EE12F0B751D926B851DA22DECFBAF03B
:109AB800DDCFBBF0BAC0D9FFBBC0DAFFDF50B96F4A
:109AC800B951D8A403D0040EBC6FCAD720EE0BF04E
:109AD800BA51D926BB51DA22DFB618D0BAC00CF079
:109AE800BBC00DF020EE14F0B751D926B851DA22D8
:109AF800DECF0EF0DDCF0FF0000E116E0B0E106EE4
:109B080057EC55F00C500D10D8B4AAD7B7C0A4F034
:109B1800B8C0A5F0000E0001A76F000EA66F9FEC5D
:109B280028F00001BC6FBC51D8A49AD79CD7C1C0FB
:109B3800B7F0C2C0B8F0000E0001BA6F010EB96FDD
:109B480037EC4CF00001C36FC351D8A458D0C1C042
:109B5800D9FFC2C0DAFFDECF3AF0DDCF3BF020EE0E
:109B68000EF0C151D926C251DA22DECF3CF0DECF49
:109B78003DF0DECF3EF0DECF3FF084EC4FF0000149
:109B8800C36FC351D8A43BD020EE12F0C151D926DF
:109B9800C251DA22DECF0CF0DDCF0DF0000E0F6ED1
:109BA800000E0E6E000E116E200E106E92EC5AF022
:109BB800000120EE12F0C151D926C251DA22DECFBF
:109BC8000CF0DDCF0DF020EE14F0C151D926C251B2
:109BD800DA22DECF0EF0DDCF0FF0000E116E0B0E85
:109BE800106EBEEC58F0C1C0D9FFC2C0DAFF10EE4B
:109BF80004F0DE50E126DD50E222010EE76E00019E
:109C0800C3511200236E2350D8A404D0215022102F
:109C1800D8A402D0040E120051A002D0030E1200E4
:109C28004EB608D0090ED8901D361E361F3620367F
:109C3800E82EF9D7225008E1020E215CD8B004D0F2
:109C4800000E256E110E03D0000E256E120E246E26
:109C580024C026F01DC015F01EC016F01FC017F056
:109C680020C018F026507DEC58F00009D8A425D063
:109C78001BC00CF01CC00DF0020E0F6E000E0E6E15
:109C880022EC55F00009D8B409D0020E1C26210692
:109C9800D8A0220621502210D8A4EAD7120E2618DE
:109CA800D8A40BD0000E156E000E166E000E176E9F
:109CB800000E186E0C0E7DEC58F0A1EC5BF02150F4
:109CC8002210D8B402D0010E1200000E12001A0E93
:109CD8000E24106E000E0F20116E010E1024D96E86
:109CE800000E1120DA6EDF50126E1250146E136AD5
:109CF8001A0E0E24D96E000E0F20DA6EDF50156E84
:109D080015501312000E141213C01AF014C01BF0D1
:109D18001C6A1D6A0CC0D9FF0DC0DAFF030EDE18DD
:109D2800D8A42ED0140E0E24106E000E0F20116E23
:109D3800010E1024D96E000E1120DA6EDF50126E5B
:109D48001250146E136A140E0E24D96E000E0F20D2
:109D5800DA6EDF50156E15501310166E1450176E0C
:109D6800186A196A17C019F016C018F0176A166A27
:109D780016501A1217501B1218501C1219501D1287
:109D88001AC00CF01BC00DF01CC00EF01DC00FF067
:109D98001200020E1A5E000E1B5A1C5A1D5A20EEA3
:109DA80012F01850D9261950DA22FE0EDE241E6E43
:109DB800FF0EDE201F6EFF0EDE20206EFF0EDE205F
:109DC800216E1E501A5C1F501B5820501C582150E1
:109DD8001D58D8A009D0000E186E000E196E000E7E
:109DE8001A6E000E1B6E120020EE26F01850D926AF
:109DF8001950DA22DECF1EF0DECF1FF0DECF20F0C2
:109E0800DECF21F020EE02F01850D9261950DA22C0
:109E1800DF50226E22500C6E0D6A0E6A0F6A1AC04D
:109E280010F01BC011F01CC012F01DC013F007EC9D
:109E380057F01E500C24186E1F500D20196E20501C
:109E48000E201A6E21500F201B6E1200DFC0E5F0A5
:109E5800E0C0E6F0E50E0C6E000E0D6E97EC46F0D5
:109E68000CC0E7F00DC0E8F00001E8AF02D00B0E1F
:109E78001200D890E735D96EE835DA6E8A0ED92601
:109E8800010EDA22DECFE3F0DDCFE4F0E351E41196
:109E9800D8B406D0E3C0D9FFE4C0DAFF000EDF6E05
:109EA800DD51DE11D8B406D0DDC0D9FFDEC0DAFF3F
:109EB800000EDF6ED890E735D96EE835DA6E8A0E77
:109EC800D926010EDA22DDC0DEFFDEC0DDFFDD515E
:109ED800DE11D8B403D0E105D8B402D0000E1200C8
:109EE800DD0E846F000E856FDF0E866F000E876FA4
:109EF800000E886FB8EC00F00001E26FE25112002A
:109F0800000E446E20EE2AF03A50D9263B50DA2251
:109F18003C50DE180AE13D50DE1807E13E50DE18DD
:109F280004E13F50DE18D8B43CD03AC025F03BC01D
:109F380026F047EC45F0446E4450D8A432D02E0E9B
:109F48003A241B6E000E3B201C6E3CC01DF03DC029
:109F58001EF03EC01FF03FC020F0000E226E010E22
:109F6800216E20EE01F03A50D9263B50DA22DF501C
:109F780006EC4EF00009D8B406D03C683D683E684F
:109F88003F68010E446E20EE2AF03A50D9263B5025
:109F9800DA223CC0DEFF3DC0DEFF3EC0DEFF3FC030
:109FA800DEFF4450120004D00C4A0D2A0E4A0F2A34
:109FB8000EC0D9FF0FC0DAFFDF50106E0CC0F6FFDD
:109FC8000DC0F7FF000EF86E0E0EF76403D0080000
:109FD800F55005D0F6CFE9FFF7CFEAFFEF5010189C
:109FE800D8A414D00CC0F6FF0DC0F7FF000EF86E11
:109FF8000E0EF76403D00800F55005D0F6CFE9FF40
:10A00800F7CFEAFFEF500009D8A4CED70CC0F6FF6F
:10A018000DC0F7FF000EF86E0E0EF76403D00800AF
:10A02800F55005D0F6CFE9FFF7CFEAFFEF50106EF5
:10A038000EC0D9FF0FC0DAFFDF50116E1150105C4F
:10A048000C6E0D6AD8A00D061200000E866E000E6A
:10A05800846E8B688968000E0101A46F000EA96FD9
:10A06800000E916F000E906F83928394000EAB6F79
:10A07800000EAA6F200EAD6F400EAC6F000E8F6FF2
:10A08800000E8E6F0AD0000E8E25D96E040E8F2119
:10A09800DA6E000EDF6E8E4B8F2B8FBFF4D78F05D5
:10A0A800D8A0F1D7000E8F6F000E8E6F0AD0340E35
:10A0B8008E25D96E0B0E8F21DA6E000EDF6E8E4B59
:10A0C8008F2B8FBFF4D78F05D8A0F1D70F01176951
:10A0D800D6501F0B4009D66ED6980F0ED612D598BB
:10A0E8000F0ED5120E01C29BD58E12000CC014F0B3
:10A0F8000DC015F00EC016F00FC017F01006D8A04E
:10A10800110610280FE11128D8A40CD0000E0D6EEE
:10A11800000E0C6E1200144A152A164A172A100649
:10A12800D8A0110614C0F6FF15C0F7FF0800F550B7
:10A138000009D8B418D016C0D9FF17C0DAFFDF500D
:10A14800D8B411D010501110D8B40DD016C0D9FF02
:10A1580017C0DAFF14C0F6FF15C0F7FFDE5009007C
:10A16800F518D8B4D8D714C0F6FF15C0F7FF080003
:10A17800F5CF12F016C0D9FF17C0DAFFDF50136E03
:10A188001350125C0C6E0D6AD8A00D0612000F5009
:10A198001010D8B404D00F501010D8A404D00D500B
:10A1A8005EEC5BF0120020EE04F00F50D926105040
:10A1B800DA22DE50DE10D8B416D020EE04F00F50AC
:10A1C800D9261050DA2210EE02F00F50E126105076
:10A1D800E222DE50E65CE650800A156EDE50800A08
:10A1E8001558D8B0120020EE02F00F50D9261050A2
:10A1F800DA22DECF11F0DDCF12F00FC0D9FF10C088
:10A20800DAFFDECF13F0DDCF14F011501324D96E2E
:10A2180012501420DA6E0DC0DFFF20EE02F00F504E
:10A22800D9261050DA22DE2A000EDD2212000101A2
:10A238007AA10AD01FC016F020C017F01DC018F070
:10A248001EC019F0B1EC59F022BE05D021C026F08D
:10A2580022C027F004D0000E276E000E266E000ED6
:10A26800256E000E246E0CD0000E0E6E200E0D6EA4
:10A278001DC00FF01EC010F0CBEC50F0244A252A68
:10A288002650245C2550800A236E2750800A2358C4
:10A29800D8A0EAD701017AB10AD01FC016F020C0B1
:10A2A80017F01DC018F01EC019F0B1EC59F01FC00E
:10A2B80012F020C013F03AEC58F0265012241D6E0C
:10A2C800275013201E6E12000001FF51140D070EB7
:10A2D800F324D96E010EF420DA6E000EDE24CB6F63
:10A2E800010EDE20CC6F000EDE20CD6F000EDE20CA
:10A2F800CE6FFF51140D070EF324D96E010EF42012
:10A30800DA6ECBC0DEFFCCC0DEFFCDC0DEFFCEC034
:10A31800DEFFFF51140D070EF324D96E010EF42051
:10A32800DA6EDECFCFF0DDCFD0F0FF51200D140E66
:10A33800F324A46F020EF420A56FCFC0A6F0D0C0FE
:10A34800A7F0A86BA96B02EC10F00001D16FD151F6
:10A35800D8B403D0010E4D6E1200000E4D6E1200DF
:10A368000DC013F00EC014F013501410D8B43ED022
:10A3780013C0D9FF14C0DAFFDE50DE10D8B436D0CF
:10A3880013C0D9FF14C0DAFFDECF0FF0DDCF10F015
:10A398000FC0D9FF10C0DAFFDF50D8B427D020EEA5
:10A3A80002F01350D9261450DA2213C0E1FF14C06A
:10A3B800E2FF00EE06F0E650E926E550EA22DE501C
:10A3C800EE1814E1DE50EE18D8A410D013C0D9FF4F
:10A3D80014C0DAFF10EE01F0DE50E126DD50E22273
:10A3E800E75086EC5BF00F6E0FA002D0090E12004A
:10A3F800000E1200000E4C6E000E4B6E000E010196
:10A408007F6F000E7E6F020E956F8390000E946F23
:10A41800000E936F000E0001FF6F030EFF6501D061
:10A428002CD0FF51070D520EF324D96E010EF420E3
:10A43800DA6E000EDF6EFF51070D510EF324D96E50
:10A44800010EF420DA6E000EDF6EFF51070D500E7C
:10A45800F324D96E010EF420DA6E000EDF6EFF5180
:10A46800070D530EF324D96E010EF420DA6EDE6A5E
:10A47800DE6ADE6ADD6AFF2BD0D7000EFF6F12009E
:10A4880025EE04F0DE50DE10D8B4FAD700C514F07B
:10A4980001C515F0060E1424D96E050E1520DA6EC6
:10A4A800DF50126E060E1424D96E070E1520DA6ED0
:10A4B800DF50136E144A152AFF0E0E6E010E0F6E32
:10A4C80014C010F015C011F00E5010160F501116D0
:10A4D80010C000F511C001F5F29E25EE04F0DE066D
:10A4E800000EDD5AF28E0CC0D9FF0DC0DAFF13C082
:10A4F800DFFF25EE04F0010EDBBE05D0000EDE5CAA
:10A50800020EDE58D8A08982125012008380000EF5
:10A518000001B76F000EB86F000EB96F000EBA6F6A
:10A52800FF51200D140EF3248C6F020EF4208D6F52
:10A53800340E8E6F0B0E8F6F010E916F000E906FA1
:10A54800BB0E926F000E936F09EC13F05350FD0B86
:10A55800536E010E0101A46FBBC023F0BCC024F0F0
:10A568008EEC3AF023C0B5F024C0B6F0000E01011D
:10A57800A46F0001B551B725B76FB651B821B86FB0
:10A58800000EB921B96F000EBA21BA6F000E010191
:10A59800956F83901200000E146E000E156E000E5B
:10A5A800166E000E176E1050111012101310D8B43A
:10A5B8002AD0010E186E06D0D890103611361236F1
:10A5C8001336182A13AEF8D7D8901436153616361F
:10A5D800173610500C5C11500D5812500E5813506D
:10A5E8000F58D8A009D010500C5E11500D5A1250B7
:10A5F8000E5A13500F5A1480D89013321232113257
:10A608001032182EE1D714C00CF015C00DF016C08A
:10A618000EF017C00FF012005AEC59F0CC0E44ECB3
:10A628005BF0660E44EC5BF0F5EC5AF0166E1650D3
:10A63800D8A409D0000E106E000E116E000E126E16
:10A64800000E136E1200000E156E000E146E160E1C
:10A658001424D96E000E1520DA6EF5EC5AF0DF6E70
:10A66800144A152A15BEF3D7155004E1040E145CDC
:10A67800D8A0EDD719501810171004E1060E165C73
:10A68800D8A0D8D716C010F017C011F018C012F013
:10A6980019C013F01200146E0C0E1418D8B409D097
:10A6A800A1EC5BF026EC5BF00009D8A402D0FF0E09
:10A6B8001200145040097DEC5BF011507DEC5BF00A
:10A6C80010507DEC5BF00F507DEC5BF00E507DEC94
:10A6D8005BF0010E136E1450D8A402D0950E136EC1
:10A6E800080E1418D8A402D0870E136E13507DECF0
:10A6F8005BF00C0E1418D8B495EC5BF00A0E136ED0
:10A7080095EC5BF0126E12AE02D0132EF9D71250F0
:10A718001200150E126EC60EE82EFED7122EFCD7AA
:10A7280000D020D0150E126EC60EE82EFED7122EBF
:10A73800FCD700D0010E0C6E10C0F6FF11C0F7FF59
:10A74800000EF86E0E0EF76403D00800F55005D021
:10A75800F6CFE9FFF7CFEAFFEF5086EC57F0104A43
:10A76800112AD7D710C0F6FF11C0F7FF000EF86EF8
:10A778000E0EF76403D00800F55005D0F6CFE9FFB8
:10A78800F7CFEAFFEF500009D8B41200CBD711EC8D
:10A7980043F0CBC0E8F0CCC0E9F00001E851E91182
:10A7A800D8B405D0E8C0E2F0E9C0E3F012008FB4F5
:10A7B80018D0FF51200D140EF324A46F020EF420BC
:10A7C800A56F000EA66F040EA76F010EA96F000EED
:10A7D800A86FE60EAA6F000EAB6F70EC0CF00001CC
:10A7E800EA6FEA51D8B404D0EAC0E2F0E36B120091
:10A7F80068EC51F0010E0101986F000E0001E36F43
:10A80800000EE26F120011D0030E0DD0050E0E6E71
:10A81800000E0101816F000E806F2FD0010E03D052
:10A82800020E01D0000E0E6E28D080C10CF081C13E
:10A838000DF00D50000AD8B40AD0020AD8B40FD0CF
:10A848000F0AD8B411D02A0AD8B413D0EBD70C50B9
:10A858000A0AD8B4D9D71E0AD8B4D8D7E3D70C5027
:10A86800BC0AD8B4DDD7DED70C50AC0AD8B4D6D7DA
:10A87800D9D70C500F0AD8A4D5D70E501200535070
:10A88800FD0B536E340E0C6E0B0E0D6EF50E0E6E28
:10A89800020E0F6E000E116E050E106E18EC58F0B9
:10A8A800390E0C6E0B0E0D6ED50E0E6E020E0F6E5F
:10A8B800000E116E130E106E18EC58F0535002096A
:10A8C800536E4C0E0C6E0B0E0D6EE80E0E6E020ED5
:10A8D8000F6E000E116E0D0E106E18EC58F0000E73
:10A8E800246E250E236E8EEC3AF05350FD0B536EFA
:10A8F80083901200000E0001FF6F030EFF6501D068
:10A908002CD0FF51070D520EF324D96E010EF420FE
:10A91800DA6E000EDF6EFF51070D510EF324D96E6B
:10A92800010EF420DA6E000EDF6EFF51070D500E97
:10A93800F324D96E010EF420DA6E000EDF6EFF519B
:10A94800070D530EF324D96E010EF420DA6EDE6A79
:10A95800DE6ADE6ADD6AFF2BD0D7000EFF6F8390B8
:10A96800000E0101956F1200000E1B6E000E1A6E8C
:10A97800000E196E24D016EC5BF00C500D10D8B4F4
:10A9880013D0190E0C6E000E0D6E44EC52F0186EBA
:10A99800000E0101A925D96EDA6A040EDA2218C060
:10A9A800DFFFA92B1A4A1B2A19AA07D0000E1A245E
:10A9B800166E040E1B20176E12008EAC05D01BBE3F
:10A9C800DAD71B04D8A0D7D71AC016F01BC017F0C7
:10A9D8001200000E0D6E000E0C6E0001FF51140DDA
:10A9E800070EF324D96E010EF420DA6EDE6ADE6AF1
:10A9F800DE6ADD6AFF51140D130EF324D96E010EC1
:10AA0800F420DA6E000EDF6EFF51140D0F0EF324E2
:10AA1800D96E010EF420DA6EDE6ADE6ADE6ADD6A5D
:10AA28000C4A0D2A0DBED9D70D5004E1040E0C5C5A
:10AA3800D8A0D3D78390000E4D6E1200070E116E6A
:10AA4800D00E106E10D095EC5BF0126E1228D8A4C0
:10AA58000ED0E40E00D000D0E82EFCD700D000D0F5
:10AA68001006D8A0110610501110D8A4ECD7FE0E6D
:10AA78001218D8B402D0000E120095EC5BF00CC08E
:10AA8800D9FF0DC0DAFFDF6E0C4A0D2A0E06D8A0DA
:10AA98000F060E500F10D8A4F0D795EC5BF095EC8C
:10AAA8005BF0010E12000CC014F00DC015F00EC0C2
:10AAB80016F00FC017F0000E196E000E186E100673
:10AAC800D8A01106102803E11128D8B41AD014C050
:10AAD800D9FF15C0DAFF144A152ADF50126E16C0C6
:10AAE800D9FF17C0DAFF164A172ADF50136E135022
:10AAF800125C186E196AD8A0190618501910D8B423
:10AB0800DED718C00CF019C00DF01200105011104B
:10AB180012101310D8B424D0010E146E06D0D89099
:10AB28001036113612361336142A13AEF8D71050D1
:10AB38000C5C11500D5812500E5813500F58D8A0D5
:10AB480008D010500C5E11500D5A12500E5A135066
:10AB58000F5AD8901332123211321032142EE7D70E
:10AB68000CC00CF00DC00DF00EC00EF00FC00FF0B1
:10AB78001200010E0E6E000E0F6E88868782878483
:10AB8800050EE82EFED700F08794050EE82EFED7B6
:10AB980000F0000E0D6E000E0C6E8DA603D00F5047
:10ABA8000E100F6E0E500E240E6E8790050EE82EB6
:10ABB800FED700F08780050EE82EFED700F08790BC
:10ABC8000C4A0D2A0DBEE9D70D5004E1030E0C5CAA
:10ABD800D8A0E3D70F501200246EF50E256EFA0E9A
:10ABE800266E000E236E0CD025C0F6FF26C0F7FF98
:10ABF800254A262A0800F5500009D8A4F5D7232AA3
:10AC080024502318D8B409D025C0F6FF26C0F7FF72
:10AC18000800F5500009D8A4E7D7AA0E00018A6FEA
:10AC2800FE0E8B6F24C08CF08D6B25C08EF026C075
:10AC38008FF035EC5BF01200DEEC58F00009D8A478
:10AC480002D0000E120010507DEC5BF0FD0E1018C3
:10AC5800D8B420D0020E126E000E116E0EC0D9FFAD
:10AC68000FC0DAFFDF507DEC5BF00E4A0F2A1106A9
:10AC7800D8A0120611501210D8A4F0D795EC5BF0AA
:10AC880095EC5BF095EC5BF0136E13501F0B050A07
:10AC9800D8A4D7D7010E120012C018F013C019F0AB
:10ACA80014D01606D8A0170614C0D9FF15C0DAFFAD
:10ACB800144A152A18C0E1FF19C0E2FF184A192AD8
:10ACC800DFCFE7FFE750D8B40DD016501710D8B42F
:10ACD80009D0E7D718C0D9FF19C0DAFF000EDF6E18
:10ACE800184A192A1606D8A017061628F3E11728B5
:10ACF800D8B41200EFD77CC080F07DC081F0000E80
:10AD08000101756F000E746F17D07AC074F07BC0A4
:10AD180075F0800E0001766F000E776F7EC078F0B8
:10AD28007FC079F079EC41F000017451010174277A
:10AD3800000175510101752380C0F6FF81C0F7FF3E
:10AD48000800F5500009D8A4E0D774C17AF075C19D
:10AD58007BF012000FC013F010C014F011C015F0F2
:10AD680012C016F05AEC59F0CC0E44EC5BF0990E78
:10AD780044EC5BF00C0E44EC5BF0000E186E000E19
:10AD8800176E130E1724D96E000E1820DA6EDF50D6
:10AD980044EC5BF0174A182A18BEF3D7185004E1A0
:10ADA800040E175CD8A0EDD75AEC59F01200838036
:10ADB80053500209536E2BEE34F093C1DFFF000E9F
:10ADC800E8CF35FB0D0EE8CF36FB000EE8CF37FB9A
:10ADD8008FA403D0600EE8CF37FB8FA406D036CB04
:10ADE80029F0200E291229C036FB000E246E040E0D
:10ADF800236E8EEC3AF05350FD0B536E000E01019A
:10AE0800936F83901200000E146E000E156E000EE4
:10AE1800166E000E176E0CA008D010501426115094
:10AE280015221250162213501722D89010361136B8
:10AE380012361336D8900F320E320D320C320C50B7
:10AE48000D100E100F10D8A4E6D714C00CF015C0C2
:10AE58000DF016C00EF017C00FF0120015D00DC07F
:10AE6800F6FF0EC0F7FF000EF86E0E0EF76403D063
:10AE78000800F55005D0F6CFE9FFF7CFEAFFEF500D
:10AE880069EC5BF00D4A0E2A0DC0F6FF0EC0F7FF05
:10AE9800000EF86E0E0EF76403D00800F55005D0CA
:10AEA800F6CFE9FFF7CFEAFFEF500009D8B4120058
:10AEB800D6D7860E00018A6F000E8B6F82C08CF089
:10AEC80083C08DF0000E8F6F000E8E6F000E916F95
:10AED800000E906F8C0E7A6F000E7B6F84C07CF032
:10AEE80085C07DF08A0E7E6F000E7F6F7FEC56F076
:10AEF80000018E518225D96E8F518321DA6E000EA2
:10AF0800DF6E12000D6E8792050EE82EFED700F058
:10AF18000CB002D0879401D08784000E0F6E010E0A
:10AF28000E6E0DAE02D0838A01D0839A0D500D2487
:10AF38000D6E8790878087900E4A0F2A0FBEF1D733
:10AF48000F5004E1090E0E5CD8A0EBD787821200DF
:10AF58009F0E146EFF0E156E12C016F013C017F078
:10AF68001450162615501722175006E11A0E165CB3
:10AF7800D8B002D0010E01D0000E186E196A185010
:10AF88001910D8B405D05F0E1214126E136A12008D
:10AF980012C012F013C013F0120002D00C4A0D2A8E
:10AFA8000CC0F6FF0DC0F7FF0800F5500009D8B433
:10AFB8000FD00CC0F6FF0DC0F7FF0800F550106E5B
:10AFC800116A0E501018EAE10F501118D8A4E6D7EC
:10AFD8000CC0F6FF0DC0F7FF0800F5500C6E0D6AA7
:10AFE800120080004C4142454C31000000028000B4
:10AFF80000000000000E000068706469736B2E6327
:10B0080066670001091220010001001700002D11D8
:10B018009420D00F00010000000000000000000094
:10B02800099F02800102E8050EC015F00FC016F056
:10B038000CC013F00DC014F010D015C0D9FF16C005
:10B04800DAFFDF50126E154A162A13C0D9FF14C052
:10B05800DAFF12C0DFFF134A142A1006D8A011061F
:10B068001028EBE11128D8B41200E7D712C014F069
:10B0780013C015F002D0124A132A12C0F6FF13C0EB
:10B08800F7FF000EF86E0E0EF76403D00800F550B7
:10B0980005D0F6CFE9FFF7CFEAFFEF500009D8A4B3
:10B0A800EAD71450125C126E15501358136E120022
:10B0B80020EE1AF00C50D9260D50DA220EC0DFFF10
:10B0C80020EE1BF00C50D9260D50DA220F50DF6EFF
:10B0D80020EE14F00C50D9260D50DA2210C0DFFFF4
:10B0E80020EE15F00C50D9260D50DA221150DF6EE3
:10B0F8001200196E19AE12D0199E000E0E6E000EB7
:10B108000F6E000E106E000E116E370E4FEC53F0DE
:10B118001A6E010E1A6402D01A50120015C00EF0F1
:10B1280016C00FF017C010F018C011F019504FECEE
:10B1380053F0120073C047F074C048F09CEC3BF029
:10B148000001756F7551D8A413D073C00DF074C089
:10B158000EF0B4EC51F00001756F7551D8A408D009
:10B1680073C0D9FF74C0DAFF000EDE6E000EDD6E0C
:10B17800755112000CC012F00DC013F00EC014F07F
:10B188000FC015F00ED014C0D9FF15C0DAFF12C0D9
:10B19800E1FF13C0E2FFDFCFE7FF144A152A124A86
:10B1A800132A1006D8A011061028EDE11128D8B4EA
:10B1B8001200E9D7130E0D6E880E0C6E0FD095ECA9
:10B1C8005BF0FF0AD8B40ED0E40E00D000D0E82E11
:10B1D800FCD700D000D00C06D8A00D060C500D10DE
:10B1E800D8A4EDD70C500D10D8B402D0010E12001F
:10B1F800000E12000C6E0C50D8B40ED0A6EC5BF00A
:10B20800200EE82EFED7A9EC5BF0CC0E00D0E82E7D
:10B21800FDD700D000D01200A6EC5BF0C00E00D025
:10B22800E82EFDD7A9EC5BF0350EE82EFED700F02E
:10B238001200010E126E200E0C180D10D8B414D086
:10B24800F70E0E6EFF0E0F6E0CC010F00DC011F051
:10B258000E5010260F501122115004E1050E105CFB
:10B26800D8A002D0000E126E12C00CF00D6A1200A7
:10B27800340E0C6E0B0E0D6E000E0F6E000E0E6E61
:10B28800010E116E000E106ED1EC47F0010EE8CFE2
:10B2980034FB53500209536E000E246E010E236EC8
:10B2A8008EEC3AF05350FD0B536E1200A6EC5BF097
:10B2B8000A0E0D6EF80EE82EFED70D2EFCD700D024
:10B2C800A9EC5BF0E00E00D0E82EFDD774EC5BF043
:10B2D8000E6E090E0D6E840EE82EFED70D2EFCD7CD
:10B2E800A9EC5BF00E501200000EF2BE010E0F6EBC
:10B2F8000D50030B7F6E0CC07EFF0EC080FF3F0E0B
:10B3080081168184F29E550E826EAA0E826E81820B
:10B3180081B2FED781940FB002D0F29E01D0F28E96
:10B328001200340E0C6E0B0E0D6E000E0F6E000E1A
:10B338000E6E010E116E000E106ED1EC47F02BEE62
:10B3480034F095C1DFFF000E246E010E236E8EECE3
:10B358003AF0000E0101956F1200000E1C6E000EEF
:10B368001B6E0BD01AC00DF00E6A18C00FF019C072
:10B3780010F0CBEC50F01B4A1C2A1B501624D96E37
:10B388001C501720DA6EDF501A6E1A50D8B412000B
:10B39800E9D760900F0E0F01596F070E396F070E2E
:10B3A800356F4F0E936E000E8A6E8A888A828A8263
:10B3B800000E8F6E130E0E01B76F0F0EFA6F100E80
:10B3C800FC6F140EB86F12009F869E84090E0E0142
:10B3D800FD6F9F98890E9B6E000E9C6E9E989D8EA9
:10B3E8009D889D9AC599F28AF28E9E909D9C9E9A00
:10B3F8009E8A01019991000E9A6F12009F0E0E6E9F
:10B40800FF0E0F6E200E0C10106E000E0D10116E38
:10B418000E5010260F501122115006E11A0E105C22
:10B42800D8B002D0010E01D0000E0C6E0D6A1200C9
:10B438009F0E0E6EFF0E0F6E0CC010F00DC011F0B7
:10B448000E5010260F501122115006E11A0E105CF2
:10B45800D8B002D0010E01D0000E0C6E0D6A120099
:10B46800BF0E0E6EFF0E0F6E0CC010F00DC011F067
:10B478000E5010260F501122115006E11A0E105CC2
:10B48800D8B002D0010E01D0000E0C6E0D6A120069
:10B49800D00E0E6EFF0E0F6E0CC010F00DC011F026
:10B4A8000E5010260F501122115006E10A0E105CA2
:10B4B800D8B002D0010E01D0000E0C6E0D6A120039
:10B4C8000C6E0C50D8B40AD0000E966E4F0E936EC8
:10B4D8002A0E966E400E956E968A1200000E966E93
:10B4E800100E966E2A0E966EF00E936EF3D7000E1F
:10B4F800116E110E106E09D0050EE82EFED700F061
:10B50800010E0C6E200E86EC57F01006D8A011061E
:10B518001028F2E11128D8B41200EED70CC012F0AE
:10B528000DC013F008D012C0D9FF13C0DAFF0EC047
:10B53800DFFF124A132A1006D8A011061028F3E1DB
:10B548001128D8B41200EFD79150070B0C6E888AD7
:10B558008DAA03D00C50080F0C6E020E01019F1922
:10B56800D8A404D00C50FF0A0F0B0C6E0C5012001C
:10B57800000EE8CF00F5000EE8CF01F5000EE8CF89
:10B5880002F5000EE8CF03F5000EE8CF04F5000E33
:10B59800E8CF05F51200A6EC5BF0200EE82EFED7EA
:10B5A800A9EC5BF0300EE82EFED774EC5BF00D6E64
:10B5B800B00E00D0E82EFDD70D5012000C500E0230
:10B5C800F3CF10F0F4CF11F00C500F02F350112606
:10B5D8000D500E02F350112610C00CF011C00DF0E2
:10B5E8001200000E0E6E000E0F6ED8900E32CFECC9
:10B5F8005AF00009D8A40E8E0F2A070E0F64F5D74B
:10B608000E5012004D5946494C4531323334000131
:10B6180000000001000020001310120000000100CB
:10B628000000000025EE04F0010EDBBE05D0000E80
:10B63800DE5C020EDE58D8A0898204C50CF005C570
:10B648000DF01200AEEC5BF095EC5BF0DEEC58F020
:10B658000009D8B402D0010E1200A1EC5BF0000E74
:10B6680012008C0E216E000E226E8AC019F08BC05B
:10B678001AF0210E1B6E000E1C6EC7EC1FF0120094
:10B688000D6E000E0E6E0D50010BFEEC58F0D890AA
:10B698000D320E2A070E0E64F6D712000D50030B5A
:10B6A8007F6E0CC07EFF3F0E8116818000F000F097
:10B6B800805012000C6E03D0B2EC5BF004000E0157
:10B6C800CDA9FAD70CC09AFF12000C6E03D0B2ECC9
:10B6D8005BF004000E01CDA9FAD70CC09AFF120046
:10B6E80088888DA802D0010E01D0000E0C6E0C5077
:10B6F80012000C6E0CC092FF95B0FED795A0FED735
:10B70800925012000C6E0C50D8B402D0010E1200E8
:10B71800515012008380010E4D6E000E4D6E8390C5
:10B728001200926895B0FED795A0FED792501200ED
:10B738008390000E0101956F1200ACEC5BF095EC64
:10B748005BF012008398889812008398888812000A
:0EB758008F8012008F90120001E7340B120058
:10FAF400004F4B004449534B5F455252004E4F5404
:10FB04005F5245414459004E4F5F46494C45004EB3
:10FB14004F545F4F50454E4544004E4F545F454E41
:10FB240041424C4544004E4F5F46494C455F535952
:10FB34005354454D00000D0A2025325820253258D3
:10FB44002025327320253273202532732025327309
:10FB540020253273202532732025327320253273F9
:10FB640020253473202534732025347320253473E1
:10FB740020253473202534732025347320253473D1
:10FB840020000D0A48504469736B204D6B2049498D
:10FB9400202831384634364B34302920257320252B
:10FBA40073202573205374617274696E672E2E2E30
:10FBB4000D0A000D0A547269656420746F20746123
:10FBC4006C6B207768696C7374206E6F7420616449
:10FBD40064726573736564000D0A4D61782056651F
:10FBE40063746F72206469736B20256420256C64D0
:10FBF4002028256C582920000D0A2530325825303C
:10FC040032582053533830783A5374617475735BA7
:10FC140025645D20255820000D0A44736B73656CC0
:10FC24002069732025642C206E756D6265722069CD
:10FC3400732025642000466F756E6420616E205227
:10FC440054432066696C652061742025580D0A00B0
:10FC54004C6F6F6B696E6720666F7220616E205205
:10FC640054432066696C650D0A0046696E644669F2
:10FC74006C65206661696C65642073656172636894
:10FC84000D0A000D0A5365656B20746F20256C64A2
:10FC9400206661696C6564202564000D0A446973FB
:10FCA4006B2073656C656374206E756D626572207C
:10FCB4002564005365656B696E6720746F207365F6
:10FCC40063746F722025580D0A0046696E64466994
:10FCD4006C65206661696C656420726561640D0AF7
:10FCE400000D0A4F70656E696E67206578697374DC
:10FCF400696E6720257320000D0A476F7420256CF8
:10FD04007520202D20726573657474696E67000D0B
:10FD14000A57616974696E6720666F722063617245
:10FD24006420000D0A46696C6520257320697320E0
:10FD34006F70656E20000D0A57726F7465206469D8
:10FD4400736B6E6F3A202564000D0A4F70656E69FF
:10FD54006E67206E657720257320000D0A253032EA
:10FD64005825303258204578697420004E6F74202D
:10FD740061204C4946206469736B0D0A000D0A54D6
:10FD84005844415441206C656E20256420000D0ABE
:10FD940046696C6520255820697320257320000D61
:10FDA4000A4469736B202558206973202573200049
:10FDB4000D0A4873742062797465733220256400D7
:10FDC4000D0A5772697465206661696C20256400A8
:10FDD4000D0A52656164696E67205254430D0A002E
:10FDE4000D0A416D69676F2039313231440D0A00C3
:10FDF4000D0A53532F38302039313232440D0A0062
:10FE04000D0A44736B73656C2069732025642000AC
:10FE14000D0A52656164202564206279746573005B
:10FE2400566563746F722069732025580D0A002289
:10FE34002A2B2C3A3B3C3D3E3F5B5D7C7F000D0A08
:10FE44004F70656E696E672025732020000D0A448B
:10FE54006562756720697320256420000D0A50725D
:10FE64006F746F20697320256420000D0A52656148
:10FE74006420636F6E66696720000D0A46696C65CD
:10FE84006E616D6520257320002041544E206173FE
:10FE940073657274656420000D0A466F726D617437
:10FEA40074696E67200072633D25752046525F2594
:10FEB400730D0A000D0A4E6F20636172642025647D
:10FEC400002F6C6966646174612E62696E000D0AAC
:10FED40025732025582025580D0A000D0A736279D0
:10FEE400746573202564000D0A4D6F756E74696E18
:10FEF4006720004170722032312032303230004CA1
:10FF04006F6164696E672E2E2E0068706469736B6E
:10FF14002E63666700466D74206578697420005B03
:10FF2400535251206F66665D0031333A34383A31AA
:10FF340038005B2532582025645D005B5352512004
:10FF44006F6E5D0048504469736B20004E6F2063F0
:10FF54006172640072633D256420002D3E202558A3
:10FF640020005458446174610044534B53454C0081
:10FF74004E414D452558004449534B2558005B4D8F
:10FF84004C415D0044454255470050524F544F0088
:10FF94005265616479002025303258007B45525205
:10FFA4007D00302E3131004946432000454F492021
:10FFB4000052454E200041544E200053525120001F
:10FFC40044415620004E444143004E5246440052A0
:10FFD4005443002025580025325800207C2000443A
:10FFE400300044310044320044330044340044358A
:0BFFF400004436004437002563000085
:020000040020DA
:10000000FF0FFF0FFF0FFF0FFF0FFF0FFF0FFF0F80
:020000040030CA
:0C0000008CFFFFFF8EFFFFFFFFFFFFFFE4
:00000001FF
